Component: ARM Compiler 5.06 update 6 (build 750) Tool: armlink [4d35ed]

==============================================================================

Section Cross References

    debug.o(.text) refers to uart.o(.text) for uart_0_init
    debug.o(.text) refers to printfa.o(i.__0vsprintf) for __c89vsprintf
    debug.o(.text) refers to debug.o(.bss) for s_formatBuffer
    uart.o(.text) refers to gpio.o(.data) for PIN_CONFIG
    uart.o(.text) refers to uart.o(.data) for UART_0_CTRL
    gpio.o(.text) refers to gpio.o(.data) for PIN_CONFIG
    i2c.o(.text) refers to gpio.o(.text) for PIN_Set_GPIO
    i2c.o(.text) refers to memcpya.o(.text) for __aeabi_memcpy
    i2c.o(.text) refers to i2c.o(.data) for I2C_0_CTRL
    gpadc.o(.text) refers to main.o(i.__ARM_common_switch8) for __ARM_common_switch8
    gpadc.o(.text) refers to gpadc.o(.data) for GPADC
    gpadc.o(.text) refers to gpio.o(.data) for PIN_CONFIG
    timer_handler.o(.text) refers to timer.o(.text) for Timer_Evt_Creat
    timer_handler.o(.text) refers to timer.o(.data) for TIMER_EVT
    rtc_handler.o(.text) refers to rtc.o(.text) for RTC_EVT_Creat
    rtc_handler.o(.text) refers to rtc.o(.data) for RTC_EVT
    ota.o(.text) refers to memcpya.o(.text) for __aeabi_memcpy
    ota.o(.text) refers to main.o(.text) for CodeErase
    ota.o(.text) refers to segger_rtt_printf.o(.text) for SEGGER_RTT_printf
    ota.o(.text) refers to uread4.o(.text) for __aeabi_uread4
    ota.o(.text) refers to main.o(.text) for BLSetConnectionUpdate
    ota.o(.text) refers to timer.o(.text) for Timer_Evt_Start
    ota.o(.text) refers to ota.o(.data) for pevt
    ota.o(.text) refers to ota.o(.bss) for ota_w
    app_gpio.o(.text) refers to gpio.o(.text) for PIN_Set_GPIO
    app_gpio.o(.text) refers to i2c.o(.text) for i2c_Init
    app_gpio.o(.text) refers to isr.o(.text) for GPIO_callback
    app_timer.o(.text) refers to timer.o(.text) for timer_2_disable
    app_timer.o(.text) refers to isr.o(.text) for Timer_2_callback
    app_adc.o(.text) refers to main.o(.text) for GPADC_Get_Calibration
    app_adc.o(.text) refers to gpadc.o(.text) for GPADC_Init
    lis2dh.o(.text) refers to lis2dh12_reg.o(.text) for lis2dh12_read_reg
    lis2dh.o(.text) refers to delay.o(.text) for delay_ms
    lis2dh.o(.text) refers to i2c.o(.text) for i2c_1_read
    lis2dh.o(.text) refers to gpio.o(.text) for GPIO_Pin_Read
    lis2dh.o(.text) refers to segger_rtt_printf.o(.text) for SEGGER_RTT_printf
    lis2dh.o(.text) refers to lis2dh.o(.bss) for dev_ctx1
    lsm6d.o(.text) refers to delay.o(.text) for delay_ms
    lsm6d.o(.text) refers to i2c.o(.text) for i2c_0_read
    lsm6d.o(.text) refers to gpio.o(.text) for GPIO_Pin_Clear
    lsm6d.o(.text) refers to lsm6dso_reg.o(.text) for lsm6dso_device_id_get
    lsm6d.o(.text) refers to fflti.o(.text) for __aeabi_i2f
    lsm6d.o(.text) refers to fadd.o(.text) for __aeabi_frsub
    lsm6d.o(.text) refers to f2d.o(.text) for __aeabi_f2d
    lsm6d.o(.text) refers to ddiv.o(.text) for __aeabi_ddiv
    lsm6d.o(.text) refers to d2f.o(.text) for __aeabi_d2f
    lsm6d.o(.text) refers to fmul.o(.text) for __aeabi_fmul
    lsm6d.o(.text) refers to dmul.o(.text) for __aeabi_dmul
    lsm6d.o(.text) refers to dadd.o(.text) for __aeabi_dadd
    lsm6d.o(.text) refers to ffixi.o(.text) for __aeabi_f2iz
    lsm6d.o(.text) refers to fdiv.o(.text) for __aeabi_fdiv
    lsm6d.o(.text) refers to lsm6d.o(.bss) for dev_ctx
    lsm6d.o(.text) refers to lsm6d.o(.data) for cntTimes
    lis2dh12_reg.o(.text) refers to fflti.o(.text) for __aeabi_i2f
    lis2dh12_reg.o(.text) refers to fdiv.o(.text) for __aeabi_fdiv
    lis2dh12_reg.o(.text) refers to fmul.o(.text) for __aeabi_fmul
    lis2dh12_reg.o(.text) refers to fadd.o(.text) for __aeabi_fadd
    lis2dh12_reg.o(.text) refers to main.o(i.__ARM_common_switch8) for __ARM_common_switch8
    lsm6dso_reg.o(.text) refers to fflti.o(.text) for __aeabi_i2f
    lsm6dso_reg.o(.text) refers to fmul.o(.text) for __aeabi_fmul
    lsm6dso_reg.o(.text) refers to fdiv.o(.text) for __aeabi_fdiv
    lsm6dso_reg.o(.text) refers to fadd.o(.text) for __aeabi_fadd
    lsm6dso_reg.o(.text) refers to main.o(i.__ARM_common_switch8) for __ARM_common_switch8
    cjson.o(.text) refers to scanf_fp.o(.text) for _scanf_real
    cjson.o(.text) refers to printfa.o(i.__0sprintf) for __2sprintf
    cjson.o(.text) refers to tolower.o(.text) for tolower
    cjson.o(.text) refers to strlen.o(.text) for strlen
    cjson.o(.text) refers to memcpya.o(.text) for __aeabi_memcpy
    cjson.o(.text) refers to memseta.o(.text) for __aeabi_memclr4
    cjson.o(.text) refers to main.o(i.__ARM_common_switch8) for __ARM_common_switch8
    cjson.o(.text) refers to strtod.o(i.strtod) for strtod
    cjson.o(.text) refers to cdrcmple.o(.text) for __aeabi_cdrcmple
    cjson.o(.text) refers to cdcmple.o(.text) for __aeabi_cdcmple
    cjson.o(.text) refers to dfixi.o(.text) for __aeabi_d2iz
    cjson.o(.text) refers to strcpy.o(.text) for strcpy
    cjson.o(.text) refers to cjson.o(.data) for global_error
    cjson.o(.text) refers to cjson.o(.bss) for version
    cjson.o(.text) refers to mallocr.o(i.__malloc$realloc) for malloc
    cjson.o(.text) refers to mallocr.o(i.__free$realloc) for free
    cjson.o(.text) refers to mallocr.o(i.realloc) for realloc
    cjson.o(.text) refers to dmul.o(.text) for __aeabi_dmul
    cjson.o(.text) refers to dadd.o(.text) for __aeabi_dsub
    cjson.o(.text) refers to __0sscanf.o(.text) for __0sscanf
    cjson.o(.text) refers to strncmp.o(.text) for strncmp
    cjson.o(.text) refers to strcmp.o(.text) for strcmp
    cjson.o(.text) refers to dflti.o(.text) for __aeabi_i2d
    cjson.o(.text) refers to f2d.o(.text) for __aeabi_f2d
    cjson.o(.data) refers to mallocr.o(i.__malloc$realloc) for malloc
    cjson.o(.data) refers to mallocr.o(i.__free$realloc) for free
    cjson.o(.data) refers to mallocr.o(i.realloc) for realloc
    crc16.o(.text) refers to crc16.o(.constdata) for crc16tab
    main.o(.text) refers to gpio.o(.text) for GPIO_Pin_Clear
    main.o(.text) refers to delay.o(.text) for delay_ms
    main.o(.text) refers to lsm6d.o(.text) for Lsm6dso_Disable
    main.o(.text) refers to uwrite4.o(.text) for __aeabi_uwrite4
    main.o(.text) refers to main.o(.text) for WakeupConfig
    main.o(.text) refers to timer.o(.text) for timer_1_disable
    main.o(.text) refers to app_timer.o(.text) for Timer2_Disable
    main.o(.text) refers to segger_rtt_printf.o(.text) for SEGGER_RTT_printf
    main.o(.text) refers to ota.o(.text) for CmdFwErase
    main.o(.text) refers to lsm6d.o(.bss) for PAS
    main.o(.text) refers to main.o(.data) for start_tx
    main.o(.text) refers to main.o(.bss) for dtts_tx_buffer
    main.o(.text) refers to ota.o(.data) for ota_state
    main.o(.text) refers to timer.o(.data) for TIMER_EVT
    main.o(.text) refers to gpio.o(.data) for PIN_CONFIG
    main.o(.text) refers to common.o(.text) for str_cmp
    main.o(.text) refers to uread4.o(.text) for __aeabi_uread4
    main.o(.text) refers to memcpya.o(.text) for __aeabi_memcpy
    main.o(.text) refers to main.o(i.__ARM_common_switch8) for __ARM_common_switch8
    main.o(.text) refers to segger_rtt.o(.text) for SEGGER_RTT_Init
    main.o(.text) refers to timer_handler.o(.text) for Timer_Evt_List
    main.o(.text) refers to mcu_bsp.o(.text) for BSP_MCU_Config
    main.o(.text) refers to lis2dh.o(.text) for Lis2dh_Init
    main.o(.text) refers to ffltui.o(.text) for __aeabi_ui2f
    main.o(.text) refers to f2d.o(.text) for __aeabi_f2d
    main.o(.text) refers to dmul.o(.text) for __aeabi_dmul
    main.o(.text) refers to ddiv.o(.text) for __aeabi_ddiv
    main.o(.text) refers to d2f.o(.text) for __aeabi_d2f
    main.o(.text) refers to fmul.o(.text) for __aeabi_fmul
    main.o(.text) refers to fdiv.o(.text) for __aeabi_fdiv
    main.o(.text) refers to dadd.o(.text) for __aeabi_dadd
    main.o(.text) refers to fadd.o(.text) for __aeabi_fsub
    main.o(.text) refers to dfixi.o(.text) for __aeabi_d2iz
    main.o(.text) refers to gpadc.o(.text) for GPADC_channel_sel
    main.o(.text) refers to rtc.o(.text) for RTC_EVT_Clr
    main.o(.text) refers to cjson.o(.text) for cJSON_CreateObject
    main.o(.text) refers to dflti.o(.text) for __aeabi_i2d
    main.o(.text) refers to timer_handler.o(.bss) for syd_sysTimer
    main.o(.text) refers to rtc.o(.data) for RTC_EVT
    main.o(.text) refers to mallocr.o(i.__malloc$realloc) for malloc
    main.o(.text) refers to crc16.o(.text) for crc16_ccitt
    main.o(.text) refers to mallocr.o(i.__free$realloc) for free
    mcu_bsp.o(.text) refers to app_timer.o(.text) for Timer_Config
    mcu_bsp.o(.text) refers to app_gpio.o(.text) for LED_IO_Config
    mcu_bsp.o(.text) refers to app_adc.o(.text) for ADC_Config
    isr.o(.text) refers to lsm6d.o(.text) for Lsm6dso_RPM_Cal
    isr.o(.text) refers to main.o(.text) for pack_timer_event
    isr.o(.text) refers to gpio.o(.text) for GPIO_Pin_Read
    isr.o(.text) refers to lsm6d.o(.bss) for PAS
    isr.o(.text) refers to gpio.o(.data) for GPIO_IRQ_CTRL
    segger_rtt.o(.text) refers to strcpy.o(.text) for strcpy
    segger_rtt.o(.text) refers to memcpya.o(.text) for __aeabi_memcpy
    segger_rtt.o(.text) refers to segger_rtt.o(.bss) for _SEGGER_RTT
    segger_rtt.o(.text) refers to segger_rtt.o(.data) for _aTerminalId
    segger_rtt.o(.text) refers to strlen.o(.text) for strlen
    segger_rtt_printf.o(.text) refers to segger_rtt.o(.text) for SEGGER_RTT_Write
    segger_rtt_printf.o(.text) refers to uidiv.o(.text) for __aeabi_uidivmod
    segger_rtt_printf.o(.text) refers to idiv.o(.text) for __aeabi_idivmod
    segger_rtt_printf.o(.text) refers to printfa.o(i.__0sprintf) for __2sprintf
    segger_rtt_printf.o(.text) refers to segger_rtt_printf.o(.constdata) for _aV2C
    segger_rtt_syscalls_keil.o(.text) refers to fputc.o(i.fputc) for fputc
    segger_rtt_syscalls_keil.o(.text) refers to strcmp.o(.text) for strcmp
    segger_rtt_syscalls_keil.o(.text) refers to segger_rtt.o(.text) for SEGGER_RTT_Write
    segger_rtt_syscalls_keil.o(.text) refers to stdout.o(.data) for __stdout
    segger_rtt_syscalls_keil.o(.text) refers to segger_rtt_syscalls_keil.o(.constdata) for __stdout_name
    startup_armcm0.o(RESET) refers to startup_armcm0.o(STACK) for __initial_sp
    startup_armcm0.o(RESET) refers to startup_armcm0.o(.text) for Reset_Handler
    startup_armcm0.o(RESET) refers to rtc.o(.text) for RTC_IRQHandler
    startup_armcm0.o(RESET) refers to uart.o(.text) for UART0_IRQHandler
    startup_armcm0.o(RESET) refers to timer.o(.text) for TIMER0_IRQHandler
    startup_armcm0.o(RESET) refers to gpio.o(.text) for GPIO_IRQHandler
    startup_armcm0.o(RESET) refers to gpadc.o(.text) for GPADC_IRQHandler
    startup_armcm0.o(.text) refers to system_armcm0.o(.text) for SystemInit
    startup_armcm0.o(.text) refers to entry.o(.ARM.Collect$$$$00000000) for __main
    system_armcm0.o(.text) refers to system_armcm0.o(.data) for SystemCoreClock
    main.o(.text) refers to uread4.o(.text) for __aeabi_uread4
    main.o(.text) refers to uwrite4.o(.text) for __aeabi_uwrite4
    main.o(.text) refers to memcpya.o(.text) for __aeabi_memcpy
    main.o(.text) refers to memseta.o(.text) for __aeabi_memclr
    main.o(.text) refers to main.o(.data) for .data
    main.o(.text) refers to dfltui.o(.text) for __aeabi_ui2d
    main.o(.text) refers to dmul.o(.text) for __aeabi_dmul
    main.o(.text) refers to dfixui.o(.text) for __aeabi_d2uiz
    main.o(.text) refers to idiv.o(.text) for __aeabi_idivmod
    main.o(.text) refers to main.o(.bss) for .bss
    main.o(.text) refers to uidiv.o(.text) for __aeabi_uidivmod
    main.o(.text) refers to memcmp.o(.text) for memcmp
    main.o(.text) refers to dflti.o(.text) for __aeabi_i2d
    main.o(.text) refers to dadd.o(.text) for __aeabi_dadd
    main.o(.text) refers to ffltui.o(.text) for __aeabi_ui2f
    main.o(.text) refers to fadd.o(.text) for __aeabi_fadd
    main.o(.text) refers to f2d.o(.text) for __aeabi_f2d
    main.o(.text) refers to ddiv.o(.text) for __aeabi_ddiv
    main.o(.text) refers to main.o(.constdata) for .constdata
    main.o(.text) refers to main.o(i.__ARM_common_switch8) for __ARM_common_switch8
    timer.o(.text) refers to dfltui.o(.text) for __aeabi_ui2d
    timer.o(.text) refers to dmul.o(.text) for __aeabi_dmul
    timer.o(.text) refers to dfixui.o(.text) for __aeabi_d2uiz
    timer.o(.text) refers to main.o(.text) for syd52832_chip_confirm
    timer.o(.text) refers to timer.o(.data) for .data
    timer.o(.text) refers to timer.o(.bss) for .bss
    rtc.o(.text) refers to uidiv.o(.text) for __aeabi_uidivmod
    rtc.o(.text) refers to uread4.o(.text) for __aeabi_uread4
    rtc.o(.text) refers to timer.o(.text) for TimerDelayUS
    rtc.o(.text) refers to rtc.o(.data) for .data
    rtc.o(.text) refers to rtc_handler.o(.data) for syd_history_setting_str
    rtc.o(.text) refers to main.o(.text) for syd52832_chip_confirm
    strtod.o(i.__softfp_strtod) refers (Special) to iusefp.o(.text) for __I$use$fp
    strtod.o(i.__softfp_strtod) refers to strtod.o(.text) for __strtod_int
    strtod.o(i.strtod) refers (Special) to iusefp.o(.text) for __I$use$fp
    strtod.o(i.strtod) refers to strtod.o(.text) for __strtod_int
    entry.o(.ARM.Collect$$$$00000000) refers (Special) to entry10a.o(.ARM.Collect$$$$0000000D) for __rt_final_cpp
    entry.o(.ARM.Collect$$$$00000000) refers (Special) to entry11a.o(.ARM.Collect$$$$0000000F) for __rt_final_exit
    entry.o(.ARM.Collect$$$$00000000) refers (Special) to entry7b.o(.ARM.Collect$$$$00000008) for _main_clock
    entry.o(.ARM.Collect$$$$00000000) refers (Special) to entry8b.o(.ARM.Collect$$$$0000000A) for _main_cpp_init
    entry.o(.ARM.Collect$$$$00000000) refers (Special) to entry9a.o(.ARM.Collect$$$$0000000B) for _main_init
    entry.o(.ARM.Collect$$$$00000000) refers (Special) to entry5.o(.ARM.Collect$$$$00000004) for _main_scatterload
    entry.o(.ARM.Collect$$$$00000000) refers (Special) to entry2.o(.ARM.Collect$$$$00000001) for _main_stk
    fputc.o(i.fputc) refers (Special) to iusesemip.o(.text) for __I$use$semihosting$fputc
    fputc.o(i.fputc) refers (Special) to semi.o(.text) for __semihosting_library_function
    idiv.o(.text) refers to uidiv.o(.text) for __aeabi_uidivmod
    printfb.o(i.__0fprintf$bare) refers to printfb.o(i._printf_core) for _printf_core
    printfb.o(i.__0fprintf$bare) refers to fputc.o(i.fputc) for fputc
    printfb.o(i.__0printf$bare) refers to printfb.o(i._printf_core) for _printf_core
    printfb.o(i.__0printf$bare) refers to fputc.o(i.fputc) for fputc
    printfb.o(i.__0printf$bare) refers to stdout.o(.data) for __stdout
    printfb.o(i.__0snprintf$bare) refers to printfb.o(i._printf_core) for _printf_core
    printfb.o(i.__0snprintf$bare) refers to printfb.o(i._snputc) for _snputc
    printfb.o(i.__0sprintf$bare) refers to printfb.o(i._printf_core) for _printf_core
    printfb.o(i.__0sprintf$bare) refers to printfb.o(i._sputc) for _sputc
    printfb.o(i.__0vfprintf$bare) refers to printfb.o(i._printf_core) for _printf_core
    printfb.o(i.__0vfprintf$bare) refers to fputc.o(i.fputc) for fputc
    printfb.o(i.__0vprintf$bare) refers to printfb.o(i._printf_core) for _printf_core
    printfb.o(i.__0vprintf$bare) refers to fputc.o(i.fputc) for fputc
    printfb.o(i.__0vprintf$bare) refers to stdout.o(.data) for __stdout
    printfb.o(i.__0vsnprintf$bare) refers to printfb.o(i._printf_core) for _printf_core
    printfb.o(i.__0vsnprintf$bare) refers to printfb.o(i._snputc) for _snputc
    printfb.o(i.__0vsprintf$bare) refers to printfb.o(i._printf_core) for _printf_core
    printfb.o(i.__0vsprintf$bare) refers to printfb.o(i._sputc) for _sputc
    printf0.o(i.__0fprintf$0) refers to printf0.o(i._printf_core) for _printf_core
    printf0.o(i.__0fprintf$0) refers to fputc.o(i.fputc) for fputc
    printf0.o(i.__0printf$0) refers to printf0.o(i._printf_core) for _printf_core
    printf0.o(i.__0printf$0) refers to fputc.o(i.fputc) for fputc
    printf0.o(i.__0printf$0) refers to stdout.o(.data) for __stdout
    printf0.o(i.__0snprintf$0) refers to printf0.o(i._printf_core) for _printf_core
    printf0.o(i.__0snprintf$0) refers to printf0.o(i._snputc) for _snputc
    printf0.o(i.__0sprintf$0) refers to printf0.o(i._printf_core) for _printf_core
    printf0.o(i.__0sprintf$0) refers to printf0.o(i._sputc) for _sputc
    printf0.o(i.__0vfprintf$0) refers to printf0.o(i._printf_core) for _printf_core
    printf0.o(i.__0vfprintf$0) refers to fputc.o(i.fputc) for fputc
    printf0.o(i.__0vprintf$0) refers to printf0.o(i._printf_core) for _printf_core
    printf0.o(i.__0vprintf$0) refers to fputc.o(i.fputc) for fputc
    printf0.o(i.__0vprintf$0) refers to stdout.o(.data) for __stdout
    printf0.o(i.__0vsnprintf$0) refers to printf0.o(i._printf_core) for _printf_core
    printf0.o(i.__0vsnprintf$0) refers to printf0.o(i._snputc) for _snputc
    printf0.o(i.__0vsprintf$0) refers to printf0.o(i._printf_core) for _printf_core
    printf0.o(i.__0vsprintf$0) refers to printf0.o(i._sputc) for _sputc
    printf1.o(i.__0fprintf$1) refers to printf1.o(i._printf_core) for _printf_core
    printf1.o(i.__0fprintf$1) refers to fputc.o(i.fputc) for fputc
    printf1.o(i.__0printf$1) refers to printf1.o(i._printf_core) for _printf_core
    printf1.o(i.__0printf$1) refers to fputc.o(i.fputc) for fputc
    printf1.o(i.__0printf$1) refers to stdout.o(.data) for __stdout
    printf1.o(i.__0snprintf$1) refers to printf1.o(i._printf_core) for _printf_core
    printf1.o(i.__0snprintf$1) refers to printf1.o(i._snputc) for _snputc
    printf1.o(i.__0sprintf$1) refers to printf1.o(i._printf_core) for _printf_core
    printf1.o(i.__0sprintf$1) refers to printf1.o(i._sputc) for _sputc
    printf1.o(i.__0vfprintf$1) refers to printf1.o(i._printf_core) for _printf_core
    printf1.o(i.__0vfprintf$1) refers to fputc.o(i.fputc) for fputc
    printf1.o(i.__0vprintf$1) refers to printf1.o(i._printf_core) for _printf_core
    printf1.o(i.__0vprintf$1) refers to fputc.o(i.fputc) for fputc
    printf1.o(i.__0vprintf$1) refers to stdout.o(.data) for __stdout
    printf1.o(i.__0vsnprintf$1) refers to printf1.o(i._printf_core) for _printf_core
    printf1.o(i.__0vsnprintf$1) refers to printf1.o(i._snputc) for _snputc
    printf1.o(i.__0vsprintf$1) refers to printf1.o(i._printf_core) for _printf_core
    printf1.o(i.__0vsprintf$1) refers to printf1.o(i._sputc) for _sputc
    printf1.o(i._printf_core) refers to uidiv.o(.text) for __aeabi_uidivmod
    printf2.o(i.__0fprintf$2) refers to printf2.o(i._printf_core) for _printf_core
    printf2.o(i.__0fprintf$2) refers to fputc.o(i.fputc) for fputc
    printf2.o(i.__0printf$2) refers to printf2.o(i._printf_core) for _printf_core
    printf2.o(i.__0printf$2) refers to fputc.o(i.fputc) for fputc
    printf2.o(i.__0printf$2) refers to stdout.o(.data) for __stdout
    printf2.o(i.__0snprintf$2) refers to printf2.o(i._printf_core) for _printf_core
    printf2.o(i.__0snprintf$2) refers to printf2.o(i._snputc) for _snputc
    printf2.o(i.__0sprintf$2) refers to printf2.o(i._printf_core) for _printf_core
    printf2.o(i.__0sprintf$2) refers to printf2.o(i._sputc) for _sputc
    printf2.o(i.__0vfprintf$2) refers to printf2.o(i._printf_core) for _printf_core
    printf2.o(i.__0vfprintf$2) refers to fputc.o(i.fputc) for fputc
    printf2.o(i.__0vprintf$2) refers to printf2.o(i._printf_core) for _printf_core
    printf2.o(i.__0vprintf$2) refers to fputc.o(i.fputc) for fputc
    printf2.o(i.__0vprintf$2) refers to stdout.o(.data) for __stdout
    printf2.o(i.__0vsnprintf$2) refers to printf2.o(i._printf_core) for _printf_core
    printf2.o(i.__0vsnprintf$2) refers to printf2.o(i._snputc) for _snputc
    printf2.o(i.__0vsprintf$2) refers to printf2.o(i._printf_core) for _printf_core
    printf2.o(i.__0vsprintf$2) refers to printf2.o(i._sputc) for _sputc
    printf3.o(i.__0fprintf$3) refers to printf3.o(i._printf_core) for _printf_core
    printf3.o(i.__0fprintf$3) refers to fputc.o(i.fputc) for fputc
    printf3.o(i.__0printf$3) refers to printf3.o(i._printf_core) for _printf_core
    printf3.o(i.__0printf$3) refers to fputc.o(i.fputc) for fputc
    printf3.o(i.__0printf$3) refers to stdout.o(.data) for __stdout
    printf3.o(i.__0snprintf$3) refers to printf3.o(i._printf_core) for _printf_core
    printf3.o(i.__0snprintf$3) refers to printf3.o(i._snputc) for _snputc
    printf3.o(i.__0sprintf$3) refers to printf3.o(i._printf_core) for _printf_core
    printf3.o(i.__0sprintf$3) refers to printf3.o(i._sputc) for _sputc
    printf3.o(i.__0vfprintf$3) refers to printf3.o(i._printf_core) for _printf_core
    printf3.o(i.__0vfprintf$3) refers to fputc.o(i.fputc) for fputc
    printf3.o(i.__0vprintf$3) refers to printf3.o(i._printf_core) for _printf_core
    printf3.o(i.__0vprintf$3) refers to fputc.o(i.fputc) for fputc
    printf3.o(i.__0vprintf$3) refers to stdout.o(.data) for __stdout
    printf3.o(i.__0vsnprintf$3) refers to printf3.o(i._printf_core) for _printf_core
    printf3.o(i.__0vsnprintf$3) refers to printf3.o(i._snputc) for _snputc
    printf3.o(i.__0vsprintf$3) refers to printf3.o(i._printf_core) for _printf_core
    printf3.o(i.__0vsprintf$3) refers to printf3.o(i._sputc) for _sputc
    printf3.o(i._printf_core) refers to uidiv.o(.text) for __aeabi_uidivmod
    printf4.o(i.__0fprintf$4) refers to printf4.o(i._printf_core) for _printf_core
    printf4.o(i.__0fprintf$4) refers to fputc.o(i.fputc) for fputc
    printf4.o(i.__0printf$4) refers to printf4.o(i._printf_core) for _printf_core
    printf4.o(i.__0printf$4) refers to fputc.o(i.fputc) for fputc
    printf4.o(i.__0printf$4) refers to stdout.o(.data) for __stdout
    printf4.o(i.__0snprintf$4) refers to printf4.o(i._printf_core) for _printf_core
    printf4.o(i.__0snprintf$4) refers to printf4.o(i._snputc) for _snputc
    printf4.o(i.__0sprintf$4) refers to printf4.o(i._printf_core) for _printf_core
    printf4.o(i.__0sprintf$4) refers to printf4.o(i._sputc) for _sputc
    printf4.o(i.__0vfprintf$4) refers to printf4.o(i._printf_core) for _printf_core
    printf4.o(i.__0vfprintf$4) refers to fputc.o(i.fputc) for fputc
    printf4.o(i.__0vprintf$4) refers to printf4.o(i._printf_core) for _printf_core
    printf4.o(i.__0vprintf$4) refers to fputc.o(i.fputc) for fputc
    printf4.o(i.__0vprintf$4) refers to stdout.o(.data) for __stdout
    printf4.o(i.__0vsnprintf$4) refers to printf4.o(i._printf_core) for _printf_core
    printf4.o(i.__0vsnprintf$4) refers to printf4.o(i._snputc) for _snputc
    printf4.o(i.__0vsprintf$4) refers to printf4.o(i._printf_core) for _printf_core
    printf4.o(i.__0vsprintf$4) refers to printf4.o(i._sputc) for _sputc
    printf4.o(i._printf_core) refers to uldiv.o(.text) for __aeabi_uldivmod
    printf5.o(i.__0fprintf$5) refers to printf5.o(i._printf_core) for _printf_core
    printf5.o(i.__0fprintf$5) refers to fputc.o(i.fputc) for fputc
    printf5.o(i.__0printf$5) refers to printf5.o(i._printf_core) for _printf_core
    printf5.o(i.__0printf$5) refers to fputc.o(i.fputc) for fputc
    printf5.o(i.__0printf$5) refers to stdout.o(.data) for __stdout
    printf5.o(i.__0snprintf$5) refers to printf5.o(i._printf_core) for _printf_core
    printf5.o(i.__0snprintf$5) refers to printf5.o(i._snputc) for _snputc
    printf5.o(i.__0sprintf$5) refers to printf5.o(i._printf_core) for _printf_core
    printf5.o(i.__0sprintf$5) refers to printf5.o(i._sputc) for _sputc
    printf5.o(i.__0vfprintf$5) refers to printf5.o(i._printf_core) for _printf_core
    printf5.o(i.__0vfprintf$5) refers to fputc.o(i.fputc) for fputc
    printf5.o(i.__0vprintf$5) refers to printf5.o(i._printf_core) for _printf_core
    printf5.o(i.__0vprintf$5) refers to fputc.o(i.fputc) for fputc
    printf5.o(i.__0vprintf$5) refers to stdout.o(.data) for __stdout
    printf5.o(i.__0vsnprintf$5) refers to printf5.o(i._printf_core) for _printf_core
    printf5.o(i.__0vsnprintf$5) refers to printf5.o(i._snputc) for _snputc
    printf5.o(i.__0vsprintf$5) refers to printf5.o(i._printf_core) for _printf_core
    printf5.o(i.__0vsprintf$5) refers to printf5.o(i._sputc) for _sputc
    printf5.o(i._printf_core) refers to uldiv.o(.text) for __aeabi_uldivmod
    printf6.o(i.__0fprintf$6) refers to printf6.o(i._printf_core) for _printf_core
    printf6.o(i.__0fprintf$6) refers to fputc.o(i.fputc) for fputc
    printf6.o(i.__0printf$6) refers to printf6.o(i._printf_core) for _printf_core
    printf6.o(i.__0printf$6) refers to fputc.o(i.fputc) for fputc
    printf6.o(i.__0printf$6) refers to stdout.o(.data) for __stdout
    printf6.o(i.__0snprintf$6) refers to printf6.o(i._printf_core) for _printf_core
    printf6.o(i.__0snprintf$6) refers to printf6.o(i._snputc) for _snputc
    printf6.o(i.__0sprintf$6) refers to printf6.o(i._printf_core) for _printf_core
    printf6.o(i.__0sprintf$6) refers to printf6.o(i._sputc) for _sputc
    printf6.o(i.__0vfprintf$6) refers to printf6.o(i._printf_core) for _printf_core
    printf6.o(i.__0vfprintf$6) refers to fputc.o(i.fputc) for fputc
    printf6.o(i.__0vprintf$6) refers to printf6.o(i._printf_core) for _printf_core
    printf6.o(i.__0vprintf$6) refers to fputc.o(i.fputc) for fputc
    printf6.o(i.__0vprintf$6) refers to stdout.o(.data) for __stdout
    printf6.o(i.__0vsnprintf$6) refers to printf6.o(i._printf_core) for _printf_core
    printf6.o(i.__0vsnprintf$6) refers to printf6.o(i._snputc) for _snputc
    printf6.o(i.__0vsprintf$6) refers to printf6.o(i._printf_core) for _printf_core
    printf6.o(i.__0vsprintf$6) refers to printf6.o(i._sputc) for _sputc
    printf6.o(i._printf_core) refers to printf6.o(i._printf_pre_padding) for _printf_pre_padding
    printf6.o(i._printf_core) refers to printf6.o(i._printf_post_padding) for _printf_post_padding
    printf6.o(i._printf_core) refers to uidiv.o(.text) for __aeabi_uidivmod
    printf7.o(i.__0fprintf$7) refers to printf7.o(i._printf_core) for _printf_core
    printf7.o(i.__0fprintf$7) refers to fputc.o(i.fputc) for fputc
    printf7.o(i.__0printf$7) refers to printf7.o(i._printf_core) for _printf_core
    printf7.o(i.__0printf$7) refers to fputc.o(i.fputc) for fputc
    printf7.o(i.__0printf$7) refers to stdout.o(.data) for __stdout
    printf7.o(i.__0snprintf$7) refers to printf7.o(i._printf_core) for _printf_core
    printf7.o(i.__0snprintf$7) refers to printf7.o(i._snputc) for _snputc
    printf7.o(i.__0sprintf$7) refers to printf7.o(i._printf_core) for _printf_core
    printf7.o(i.__0sprintf$7) refers to printf7.o(i._sputc) for _sputc
    printf7.o(i.__0vfprintf$7) refers to printf7.o(i._printf_core) for _printf_core
    printf7.o(i.__0vfprintf$7) refers to fputc.o(i.fputc) for fputc
    printf7.o(i.__0vprintf$7) refers to printf7.o(i._printf_core) for _printf_core
    printf7.o(i.__0vprintf$7) refers to fputc.o(i.fputc) for fputc
    printf7.o(i.__0vprintf$7) refers to stdout.o(.data) for __stdout
    printf7.o(i.__0vsnprintf$7) refers to printf7.o(i._printf_core) for _printf_core
    printf7.o(i.__0vsnprintf$7) refers to printf7.o(i._snputc) for _snputc
    printf7.o(i.__0vsprintf$7) refers to printf7.o(i._printf_core) for _printf_core
    printf7.o(i.__0vsprintf$7) refers to printf7.o(i._sputc) for _sputc
    printf7.o(i._printf_core) refers to printf7.o(i._printf_pre_padding) for _printf_pre_padding
    printf7.o(i._printf_core) refers to printf7.o(i._printf_post_padding) for _printf_post_padding
    printf7.o(i._printf_core) refers to uldiv.o(.text) for __aeabi_uldivmod
    printf8.o(i.__0fprintf$8) refers to printf8.o(i._printf_core) for _printf_core
    printf8.o(i.__0fprintf$8) refers to fputc.o(i.fputc) for fputc
    printf8.o(i.__0printf$8) refers to printf8.o(i._printf_core) for _printf_core
    printf8.o(i.__0printf$8) refers to fputc.o(i.fputc) for fputc
    printf8.o(i.__0printf$8) refers to stdout.o(.data) for __stdout
    printf8.o(i.__0snprintf$8) refers to printf8.o(i._printf_core) for _printf_core
    printf8.o(i.__0snprintf$8) refers to printf8.o(i._snputc) for _snputc
    printf8.o(i.__0sprintf$8) refers to printf8.o(i._printf_core) for _printf_core
    printf8.o(i.__0sprintf$8) refers to printf8.o(i._sputc) for _sputc
    printf8.o(i.__0vfprintf$8) refers to printf8.o(i._printf_core) for _printf_core
    printf8.o(i.__0vfprintf$8) refers to fputc.o(i.fputc) for fputc
    printf8.o(i.__0vprintf$8) refers to printf8.o(i._printf_core) for _printf_core
    printf8.o(i.__0vprintf$8) refers to fputc.o(i.fputc) for fputc
    printf8.o(i.__0vprintf$8) refers to stdout.o(.data) for __stdout
    printf8.o(i.__0vsnprintf$8) refers to printf8.o(i._printf_core) for _printf_core
    printf8.o(i.__0vsnprintf$8) refers to printf8.o(i._snputc) for _snputc
    printf8.o(i.__0vsprintf$8) refers to printf8.o(i._printf_core) for _printf_core
    printf8.o(i.__0vsprintf$8) refers to printf8.o(i._sputc) for _sputc
    printf8.o(i._printf_core) refers to printf8.o(i._printf_pre_padding) for _printf_pre_padding
    printf8.o(i._printf_core) refers to printf8.o(i._printf_post_padding) for _printf_post_padding
    printf8.o(i._printf_core) refers to uldiv.o(.text) for __aeabi_uldivmod
    printfa.o(i.__0fprintf) refers (Special) to iusefp.o(.text) for __I$use$fp
    printfa.o(i.__0fprintf) refers to printfa.o(i._printf_core) for _printf_core
    printfa.o(i.__0fprintf) refers to fputc.o(i.fputc) for fputc
    printfa.o(i.__0printf) refers (Special) to iusefp.o(.text) for __I$use$fp
    printfa.o(i.__0printf) refers to printfa.o(i._printf_core) for _printf_core
    printfa.o(i.__0printf) refers to fputc.o(i.fputc) for fputc
    printfa.o(i.__0printf) refers to stdout.o(.data) for __stdout
    printfa.o(i.__0snprintf) refers (Special) to iusefp.o(.text) for __I$use$fp
    printfa.o(i.__0snprintf) refers to printfa.o(i._printf_core) for _printf_core
    printfa.o(i.__0snprintf) refers to printfa.o(i._snputc) for _snputc
    printfa.o(i.__0sprintf) refers (Special) to iusefp.o(.text) for __I$use$fp
    printfa.o(i.__0sprintf) refers to printfa.o(i._printf_core) for _printf_core
    printfa.o(i.__0sprintf) refers to printfa.o(i._sputc) for _sputc
    printfa.o(i.__0vfprintf) refers (Special) to iusefp.o(.text) for __I$use$fp
    printfa.o(i.__0vfprintf) refers to printfa.o(i._printf_core) for _printf_core
    printfa.o(i.__0vfprintf) refers to fputc.o(i.fputc) for fputc
    printfa.o(i.__0vprintf) refers (Special) to iusefp.o(.text) for __I$use$fp
    printfa.o(i.__0vprintf) refers to printfa.o(i._printf_core) for _printf_core
    printfa.o(i.__0vprintf) refers to fputc.o(i.fputc) for fputc
    printfa.o(i.__0vprintf) refers to stdout.o(.data) for __stdout
    printfa.o(i.__0vsnprintf) refers (Special) to iusefp.o(.text) for __I$use$fp
    printfa.o(i.__0vsnprintf) refers to printfa.o(i._printf_core) for _printf_core
    printfa.o(i.__0vsnprintf) refers to printfa.o(i._snputc) for _snputc
    printfa.o(i.__0vsprintf) refers (Special) to iusefp.o(.text) for __I$use$fp
    printfa.o(i.__0vsprintf) refers to printfa.o(i._printf_core) for _printf_core
    printfa.o(i.__0vsprintf) refers to printfa.o(i._sputc) for _sputc
    printfa.o(i._fp_digits) refers (Special) to iusefp.o(.text) for __I$use$fp
    printfa.o(i._fp_digits) refers to dmul.o(.text) for __aeabi_dmul
    printfa.o(i._fp_digits) refers to ddiv.o(.text) for __aeabi_ddiv
    printfa.o(i._fp_digits) refers to cdrcmple.o(.text) for __aeabi_cdrcmple
    printfa.o(i._fp_digits) refers to dadd.o(.text) for __aeabi_dadd
    printfa.o(i._fp_digits) refers to dfixul.o(.text) for __aeabi_d2ulz
    printfa.o(i._fp_digits) refers to uldiv.o(.text) for __aeabi_uldivmod
    printfa.o(i._printf_core) refers (Special) to iusefp.o(.text) for __I$use$fp
    printfa.o(i._printf_core) refers to printfa.o(i._printf_pre_padding) for _printf_pre_padding
    printfa.o(i._printf_core) refers to uldiv.o(.text) for __aeabi_uldivmod
    printfa.o(i._printf_core) refers to printfa.o(i._printf_post_padding) for _printf_post_padding
    printfa.o(i._printf_core) refers to printfa.o(i._fp_digits) for _fp_digits
    printfa.o(i._printf_core) refers to uidiv.o(.text) for __aeabi_uidivmod
    printfa.o(i._printf_post_padding) refers (Special) to iusefp.o(.text) for __I$use$fp
    printfa.o(i._printf_pre_padding) refers (Special) to iusefp.o(.text) for __I$use$fp
    printfa.o(i._snputc) refers (Special) to iusefp.o(.text) for __I$use$fp
    printfa.o(i._sputc) refers (Special) to iusefp.o(.text) for __I$use$fp
    malloc.o(i.free) refers to mvars.o(.data) for __microlib_freelist
    malloc.o(i.malloc) refers to mvars.o(.data) for __microlib_freelist_initialised
    malloc.o(i.malloc) refers to mvars.o(.data) for __microlib_freelist
    malloc.o(i.malloc) refers to startup_armcm0.o(HEAP) for __heap_base
    mallocr.o(i.__free$realloc) refers to mvars.o(.data) for __microlib_freelist
    mallocr.o(i.__malloc$realloc) refers to mallocr.o(i.internal_alloc) for internal_alloc
    mallocr.o(i.__malloc$realloc) refers to mvars.o(.data) for __microlib_freelist_initialised
    mallocr.o(i.__malloc$realloc) refers to startup_armcm0.o(HEAP) for __heap_base
    mallocr.o(i.__malloc$realloc) refers to mvars.o(.data) for __microlib_freelist
    mallocr.o(i.internal_alloc) refers to memcpya.o(.text) for __aeabi_memcpy
    mallocr.o(i.internal_alloc) refers to mvars.o(.data) for __microlib_freelist
    mallocr.o(i.realloc) refers to mallocr.o(i.__free$realloc) for free
    mallocr.o(i.realloc) refers to mallocr.o(i.internal_alloc) for internal_alloc
    mallocr.o(i.realloc) refers to mallocr.o(i.__malloc$realloc) for malloc
    mallocr.o(i.realloc) refers to mvars.o(.data) for __microlib_freelist
    malloca.o(i.__aligned_malloc) refers to mvars.o(.data) for __microlib_freelist
    malloca.o(i.__aligned_malloc) refers to mvars.o(.data) for __microlib_freelist_initialised
    malloca.o(i.__aligned_malloc) refers to startup_armcm0.o(HEAP) for __heap_base
    malloca.o(i.__free$memalign) refers to mvars.o(.data) for __microlib_freelist
    malloca.o(i.__malloc$memalign) refers to malloca.o(i.__aligned_malloc) for __aligned_malloc
    mallocra.o(i.__aligned_malloc$realloc) refers to mallocra.o(i.internal_alloc) for internal_alloc
    mallocra.o(i.__aligned_malloc$realloc) refers to startup_armcm0.o(HEAP) for __heap_base
    mallocra.o(i.__aligned_malloc$realloc) refers to mvars.o(.data) for __microlib_freelist
    mallocra.o(i.__aligned_malloc$realloc) refers to mvars.o(.data) for __microlib_freelist_initialised
    mallocra.o(i.__free$realloc$memalign) refers to mvars.o(.data) for __microlib_freelist
    mallocra.o(i.__malloc$realloc$memalign) refers to mallocra.o(i.__aligned_malloc$realloc) for __aligned_malloc$realloc
    mallocra.o(i.__realloc$memalign) refers to mallocra.o(i.__free$realloc$memalign) for __free$realloc$memalign
    mallocra.o(i.__realloc$memalign) refers to mallocra.o(i.internal_alloc) for internal_alloc
    mallocra.o(i.__realloc$memalign) refers to mallocra.o(i.__malloc$realloc$memalign) for __malloc$realloc$memalign
    mallocra.o(i.__realloc$memalign) refers to mvars.o(.data) for __microlib_freelist
    mallocra.o(i.internal_alloc) refers to memcpya.o(.text) for __aeabi_memcpy
    mallocra.o(i.internal_alloc) refers to mvars.o(.data) for __microlib_freelist
    __0sscanf.o(.text) refers to scanf_char.o(.text) for __vfscanf_char
    __0sscanf.o(.text) refers to _sgetc.o(.text) for _sgetc
    scanf_fp.o(.text) refers (Special) to iusefp.o(.text) for __I$use$fp
    scanf_fp.o(.text) refers to llmul.o(.text) for __aeabi_lmul
    scanf_fp.o(.text) refers to dfltul.o(.text) for __aeabi_ul2d
    scanf_fp.o(.text) refers to dmul.o(.text) for __aeabi_dmul
    scanf_fp.o(.text) refers to ddiv.o(.text) for __aeabi_ddiv
    scanf_fp.o(.text) refers to scanf_fp.o(i._is_digit) for _is_digit
    scanf_fp.o(.text) refers to d2f.o(.text) for __aeabi_d2f
    fadd.o(.text) refers (Special) to iusefp.o(.text) for __I$use$fp
    fadd.o(.text) refers to fepilogue.o(.text) for _float_epilogue
    fmul.o(.text) refers (Special) to iusefp.o(.text) for __I$use$fp
    fdiv.o(.text) refers (Special) to iusefp.o(.text) for __I$use$fp
    fdiv.o(.text) refers to fepilogue.o(.text) for _float_round
    dadd.o(.text) refers (Special) to iusefp.o(.text) for __I$use$fp
    dadd.o(.text) refers to llshl.o(.text) for __aeabi_llsl
    dadd.o(.text) refers to llsshr.o(.text) for __aeabi_lasr
    dadd.o(.text) refers to depilogue.o(.text) for _double_epilogue
    dmul.o(.text) refers (Special) to iusefp.o(.text) for __I$use$fp
    dmul.o(.text) refers to depilogue.o(.text) for _double_epilogue
    ddiv.o(.text) refers (Special) to iusefp.o(.text) for __I$use$fp
    ddiv.o(.text) refers to depilogue.o(.text) for _double_round
    fflti.o(.text) refers (Special) to iusefp.o(.text) for __I$use$fp
    fflti.o(.text) refers to fepilogue.o(.text) for _float_epilogue
    ffltui.o(.text) refers (Special) to iusefp.o(.text) for __I$use$fp
    ffltui.o(.text) refers to fepilogue.o(.text) for _float_epilogue
    dflti.o(.text) refers (Special) to iusefp.o(.text) for __I$use$fp
    dflti.o(.text) refers to depilogue.o(.text) for _double_epilogue
    dfltui.o(.text) refers (Special) to iusefp.o(.text) for __I$use$fp
    dfltui.o(.text) refers to depilogue.o(.text) for _double_epilogue
    ffixi.o(.text) refers (Special) to iusefp.o(.text) for __I$use$fp
    dfixi.o(.text) refers (Special) to iusefp.o(.text) for __I$use$fp
    dfixi.o(.text) refers to llushr.o(.text) for __aeabi_llsr
    dfixui.o(.text) refers (Special) to iusefp.o(.text) for __I$use$fp
    dfixui.o(.text) refers to llushr.o(.text) for __aeabi_llsr
    f2d.o(.text) refers (Special) to iusefp.o(.text) for __I$use$fp
    cdcmple.o(.text) refers (Special) to iusefp.o(.text) for __I$use$fp
    cdrcmple.o(.text) refers (Special) to iusefp.o(.text) for __I$use$fp
    d2f.o(.text) refers (Special) to iusefp.o(.text) for __I$use$fp
    d2f.o(.text) refers to fepilogue.o(.text) for _float_round
    entry2.o(.ARM.Collect$$$$00000001) refers to entry2.o(.ARM.Collect$$$$00002712) for __lit__00000000
    entry2.o(.ARM.Collect$$$$00002712) refers to startup_armcm0.o(STACK) for __initial_sp
    entry2.o(__vectab_stack_and_reset_area) refers to startup_armcm0.o(STACK) for __initial_sp
    entry2.o(__vectab_stack_and_reset_area) refers to entry.o(.ARM.Collect$$$$00000000) for __main
    entry5.o(.ARM.Collect$$$$00000004) refers to init.o(.text) for __scatterload
    entry9a.o(.ARM.Collect$$$$0000000B) refers to main.o(.text) for main
    entry9b.o(.ARM.Collect$$$$0000000C) refers to main.o(.text) for main
    uldiv.o(.text) refers to llushr.o(.text) for __aeabi_llsr
    uldiv.o(.text) refers to llshl.o(.text) for __aeabi_llsl
    llmul.o(.text) refers to llshl.o(.text) for __aeabi_llsl
    scanf_char.o(.text) refers to _scanf.o(.text) for __vfscanf
    scanf_char.o(.text) refers to isspace_c.o(.text) for isspace
    strtod.o(.text) refers to scanf_fp.o(.text) for _scanf_real
    strtod.o(.text) refers to _sgetc.o(.text) for _sgetc
    strtod.o(.text) refers to isspace_c.o(.text) for isspace
    depilogue.o(.text) refers to depilogue.o(i.__ARM_clz) for __ARM_clz
    depilogue.o(.text) refers to llshl.o(.text) for __aeabi_llsl
    depilogue.o(.text) refers to llushr.o(.text) for __aeabi_llsr
    dfltul.o(.text) refers to depilogue.o(.text) for _double_epilogue
    dfixul.o(.text) refers to llushr.o(.text) for __aeabi_llsr
    dfixul.o(.text) refers to llshl.o(.text) for __aeabi_llsl
    init.o(.text) refers to entry5.o(.ARM.Collect$$$$00000004) for __main_after_scatterload
    isspace_c.o(.text) refers to ctype_c.o(.text) for __ctype_lookup
    _scanf.o(.text) refers (Weak) to scanf_fp.o(.text) for _scanf_real
    ctype_c.o(.text) refers to ctype_c.o(.constdata) for .constdata
    scanf_fp.o(i._is_digit) refers (Special) to iusefp.o(.text) for __I$use$fp


==============================================================================

Removing Unused input sections from the image.

    Removing debug.o(.rev16_text), (4 bytes).
    Removing debug.o(.revsh_text), (4 bytes).
    Removing debug.o(.text), (144 bytes).
    Removing debug.o(.bss), (128 bytes).
    Removing uart.o(.rev16_text), (4 bytes).
    Removing uart.o(.revsh_text), (4 bytes).
    Removing delay.o(.rev16_text), (4 bytes).
    Removing delay.o(.revsh_text), (4 bytes).
    Removing gpio.o(.rev16_text), (4 bytes).
    Removing gpio.o(.revsh_text), (4 bytes).
    Removing i2c.o(.rev16_text), (4 bytes).
    Removing i2c.o(.revsh_text), (4 bytes).
    Removing gpadc.o(.rev16_text), (4 bytes).
    Removing gpadc.o(.revsh_text), (4 bytes).
    Removing wdt.o(.rev16_text), (4 bytes).
    Removing wdt.o(.revsh_text), (4 bytes).
    Removing timer_handler.o(.rev16_text), (4 bytes).
    Removing timer_handler.o(.revsh_text), (4 bytes).
    Removing rtc_handler.o(.rev16_text), (4 bytes).
    Removing rtc_handler.o(.revsh_text), (4 bytes).
    Removing rtc_handler.o(.text), (44 bytes).
    Removing rtc_handler.o(.bss), (24 bytes).
    Removing ota.o(.rev16_text), (4 bytes).
    Removing ota.o(.revsh_text), (4 bytes).
    Removing app_gpio.o(.rev16_text), (4 bytes).
    Removing app_gpio.o(.revsh_text), (4 bytes).
    Removing app_timer.o(.rev16_text), (4 bytes).
    Removing app_timer.o(.revsh_text), (4 bytes).
    Removing app_adc.o(.rev16_text), (4 bytes).
    Removing app_adc.o(.revsh_text), (4 bytes).
    Removing lis2dh.o(.rev16_text), (4 bytes).
    Removing lis2dh.o(.revsh_text), (4 bytes).
    Removing lsm6d.o(.rev16_text), (4 bytes).
    Removing lsm6d.o(.revsh_text), (4 bytes).
    Removing main.o(.rev16_text), (4 bytes).
    Removing main.o(.revsh_text), (4 bytes).
    Removing mcu_bsp.o(.rev16_text), (4 bytes).
    Removing mcu_bsp.o(.revsh_text), (4 bytes).
    Removing isr.o(.rev16_text), (4 bytes).
    Removing isr.o(.revsh_text), (4 bytes).
    Removing segger_rtt.o(.rev16_text), (4 bytes).
    Removing segger_rtt.o(.revsh_text), (4 bytes).
    Removing segger_rtt_printf.o(.rev16_text), (4 bytes).
    Removing segger_rtt_printf.o(.revsh_text), (4 bytes).
    Removing segger_rtt_syscalls_keil.o(.rev16_text), (4 bytes).
    Removing segger_rtt_syscalls_keil.o(.revsh_text), (4 bytes).
    Removing segger_rtt_syscalls_keil.o(.text), (180 bytes).
    Removing segger_rtt_syscalls_keil.o(.constdata), (20 bytes).
    Removing system_armcm0.o(.rev16_text), (4 bytes).
    Removing system_armcm0.o(.revsh_text), (4 bytes).
    Removing main.o(.rev16_text), (4 bytes).
    Removing main.o(.revsh_text), (4 bytes).
    Removing timer.o(.rev16_text), (4 bytes).
    Removing timer.o(.revsh_text), (4 bytes).
    Removing rtc.o(.rev16_text), (4 bytes).
    Removing rtc.o(.revsh_text), (4 bytes).

56 unused section(s) (total 740 bytes) removed from the image.

==============================================================================

Image Symbol Table

    Local Symbols

    Symbol Name                              Value     Ov Type        Size  Object(Section)

    ../clib/../cmprslib/zerorunl2.c          0x00000000   Number         0  __dczerorl2.o ABSOLUTE
    ../clib/microlib/ctype/ctype.c           0x00000000   Number         0  ctype_c.o ABSOLUTE
    ../clib/microlib/ctype/ctype.c           0x00000000   Number         0  isspace_c.o ABSOLUTE
    ../clib/microlib/ctype/tolower.c         0x00000000   Number         0  tolower.o ABSOLUTE
    ../clib/microlib/division.c              0x00000000   Number         0  uldiv.o ABSOLUTE
    ../clib/microlib/division.c              0x00000000   Number         0  uidiv.o ABSOLUTE
    ../clib/microlib/division.c              0x00000000   Number         0  idiv.o ABSOLUTE
    ../clib/microlib/init/entry.s            0x00000000   Number         0  entry9b.o ABSOLUTE
    ../clib/microlib/init/entry.s            0x00000000   Number         0  entry11b.o ABSOLUTE
    ../clib/microlib/init/entry.s            0x00000000   Number         0  entry8a.o ABSOLUTE
    ../clib/microlib/init/entry.s            0x00000000   Number         0  entry7b.o ABSOLUTE
    ../clib/microlib/init/entry.s            0x00000000   Number         0  entry5.o ABSOLUTE
    ../clib/microlib/init/entry.s            0x00000000   Number         0  entry10b.o ABSOLUTE
    ../clib/microlib/init/entry.s            0x00000000   Number         0  entry11a.o ABSOLUTE
    ../clib/microlib/init/entry.s            0x00000000   Number         0  entry2.o ABSOLUTE
    ../clib/microlib/init/entry.s            0x00000000   Number         0  entry10a.o ABSOLUTE
    ../clib/microlib/init/entry.s            0x00000000   Number         0  entry7a.o ABSOLUTE
    ../clib/microlib/init/entry.s            0x00000000   Number         0  entry9a.o ABSOLUTE
    ../clib/microlib/init/entry.s            0x00000000   Number         0  entry8b.o ABSOLUTE
    ../clib/microlib/init/entry.s            0x00000000   Number         0  entry.o ABSOLUTE
    ../clib/microlib/longlong.c              0x00000000   Number         0  llushr.o ABSOLUTE
    ../clib/microlib/longlong.c              0x00000000   Number         0  llshl.o ABSOLUTE
    ../clib/microlib/longlong.c              0x00000000   Number         0  llmul.o ABSOLUTE
    ../clib/microlib/longlong.c              0x00000000   Number         0  llsshr.o ABSOLUTE
    ../clib/microlib/malloc/malloc.c         0x00000000   Number         0  malloc.o ABSOLUTE
    ../clib/microlib/malloc/malloc.c         0x00000000   Number         0  mallocra.o ABSOLUTE
    ../clib/microlib/malloc/malloc.c         0x00000000   Number         0  malloca.o ABSOLUTE
    ../clib/microlib/malloc/malloc.c         0x00000000   Number         0  mallocr.o ABSOLUTE
    ../clib/microlib/malloc/mvars.c          0x00000000   Number         0  mvars.o ABSOLUTE
    ../clib/microlib/printf/printf.c         0x00000000   Number         0  printf2.o ABSOLUTE
    ../clib/microlib/printf/printf.c         0x00000000   Number         0  printf3.o ABSOLUTE
    ../clib/microlib/printf/printf.c         0x00000000   Number         0  printf4.o ABSOLUTE
    ../clib/microlib/printf/printf.c         0x00000000   Number         0  printf6.o ABSOLUTE
    ../clib/microlib/printf/printf.c         0x00000000   Number         0  printf7.o ABSOLUTE
    ../clib/microlib/printf/printf.c         0x00000000   Number         0  printf8.o ABSOLUTE
    ../clib/microlib/printf/printf.c         0x00000000   Number         0  printfa.o ABSOLUTE
    ../clib/microlib/printf/printf.c         0x00000000   Number         0  printfb.o ABSOLUTE
    ../clib/microlib/printf/printf.c         0x00000000   Number         0  printf0.o ABSOLUTE
    ../clib/microlib/printf/printf.c         0x00000000   Number         0  printf1.o ABSOLUTE
    ../clib/microlib/printf/printf.c         0x00000000   Number         0  printf5.o ABSOLUTE
    ../clib/microlib/printf/stubs.s          0x00000000   Number         0  stubs.o ABSOLUTE
    ../clib/microlib/stdio/fflush.c          0x00000000   Number         0  fflush.o ABSOLUTE
    ../clib/microlib/stdio/fputc.c           0x00000000   Number         0  fputc.o ABSOLUTE
    ../clib/microlib/stdio/semi.s            0x00000000   Number         0  semi.o ABSOLUTE
    ../clib/microlib/stdio/streams.c         0x00000000   Number         0  stdout.o ABSOLUTE
    ../clib/microlib/string/memcmp.c         0x00000000   Number         0  memcmp.o ABSOLUTE
    ../clib/microlib/string/memcpy.c         0x00000000   Number         0  memcpya.o ABSOLUTE
    ../clib/microlib/string/memcpy.c         0x00000000   Number         0  memcpyb.o ABSOLUTE
    ../clib/microlib/string/memset.c         0x00000000   Number         0  memseta.o ABSOLUTE
    ../clib/microlib/string/strcmp.c         0x00000000   Number         0  strcmp.o ABSOLUTE
    ../clib/microlib/string/strcpy.c         0x00000000   Number         0  strcpy.o ABSOLUTE
    ../clib/microlib/string/strlen.c         0x00000000   Number         0  strlen.o ABSOLUTE
    ../clib/microlib/string/strncmp.c        0x00000000   Number         0  strncmp.o ABSOLUTE
    ../clib/microlib/stubs.s                 0x00000000   Number         0  useno.o ABSOLUTE
    ../clib/microlib/stubs.s                 0x00000000   Number         0  iusesemip.o ABSOLUTE
    ../clib/microlib/stubs.s                 0x00000000   Number         0  iusefp.o ABSOLUTE
    ../clib/microlib/unhosted.c              0x00000000   Number         0  uread4.o ABSOLUTE
    ../clib/microlib/unhosted.c              0x00000000   Number         0  uwrite4.o ABSOLUTE
    ../clib/scanf.c                          0x00000000   Number         0  __0sscanf.o ABSOLUTE
    ../clib/scanf.c                          0x00000000   Number         0  scanf_fp.o ABSOLUTE
    ../clib/scanf.c                          0x00000000   Number         0  _scanf.o ABSOLUTE
    ../clib/scanf.c                          0x00000000   Number         0  strtod.o ABSOLUTE
    ../clib/scanf.c                          0x00000000   Number         0  _sgetc.o ABSOLUTE
    ../clib/scanf.c                          0x00000000   Number         0  scanf_char.o ABSOLUTE
    ../fplib/microlib/d2f.c                  0x00000000   Number         0  d2f.o ABSOLUTE
    ../fplib/microlib/f2d.c                  0x00000000   Number         0  f2d.o ABSOLUTE
    ../fplib/microlib/fpadd.c                0x00000000   Number         0  fadd.o ABSOLUTE
    ../fplib/microlib/fpadd.c                0x00000000   Number         0  dadd.o ABSOLUTE
    ../fplib/microlib/fpdiv.c                0x00000000   Number         0  fdiv.o ABSOLUTE
    ../fplib/microlib/fpdiv.c                0x00000000   Number         0  ddiv.o ABSOLUTE
    ../fplib/microlib/fpepilogue.c           0x00000000   Number         0  depilogue.o ABSOLUTE
    ../fplib/microlib/fpepilogue.c           0x00000000   Number         0  fepilogue.o ABSOLUTE
    ../fplib/microlib/fpfix.c                0x00000000   Number         0  dfixui.o ABSOLUTE
    ../fplib/microlib/fpfix.c                0x00000000   Number         0  dfixi.o ABSOLUTE
    ../fplib/microlib/fpfix.c                0x00000000   Number         0  dfixul.o ABSOLUTE
    ../fplib/microlib/fpfix.c                0x00000000   Number         0  ffixi.o ABSOLUTE
    ../fplib/microlib/fpflt.c                0x00000000   Number         0  dflti.o ABSOLUTE
    ../fplib/microlib/fpflt.c                0x00000000   Number         0  fflti.o ABSOLUTE
    ../fplib/microlib/fpflt.c                0x00000000   Number         0  dfltul.o ABSOLUTE
    ../fplib/microlib/fpflt.c                0x00000000   Number         0  ffltui.o ABSOLUTE
    ../fplib/microlib/fpflt.c                0x00000000   Number         0  dfltui.o ABSOLUTE
    ../fplib/microlib/fpmul.c                0x00000000   Number         0  fmul.o ABSOLUTE
    ../fplib/microlib/fpmul.c                0x00000000   Number         0  dmul.o ABSOLUTE
    ../mathlib/strtod.c                      0x00000000   Number         0  strtod.o ABSOLUTE
    ..\..\App\app_adc.c                      0x00000000   Number         0  app_adc.o ABSOLUTE
    ..\..\App\app_gpio.c                     0x00000000   Number         0  app_gpio.o ABSOLUTE
    ..\..\App\app_timer.c                    0x00000000   Number         0  app_timer.o ABSOLUTE
    ..\..\Driver\debug.c                     0x00000000   Number         0  debug.o ABSOLUTE
    ..\..\Driver\delay.c                     0x00000000   Number         0  delay.o ABSOLUTE
    ..\..\Driver\gpadc.c                     0x00000000   Number         0  gpadc.o ABSOLUTE
    ..\..\Driver\gpio.c                      0x00000000   Number         0  gpio.o ABSOLUTE
    ..\..\Driver\i2c.c                       0x00000000   Number         0  i2c.o ABSOLUTE
    ..\..\Driver\ota.c                       0x00000000   Number         0  ota.o ABSOLUTE
    ..\..\Driver\rtc_handler.c               0x00000000   Number         0  rtc_handler.o ABSOLUTE
    ..\..\Driver\timer_handler.c             0x00000000   Number         0  timer_handler.o ABSOLUTE
    ..\..\Driver\uart.c                      0x00000000   Number         0  uart.o ABSOLUTE
    ..\..\Driver\wdt.c                       0x00000000   Number         0  wdt.o ABSOLUTE
    ..\..\Hardware\cJSON.c                   0x00000000   Number         0  cjson.o ABSOLUTE
    ..\..\Hardware\common.c                  0x00000000   Number         0  common.o ABSOLUTE
    ..\..\Hardware\crc16.c                   0x00000000   Number         0  crc16.o ABSOLUTE
    ..\..\Hardware\lis2dh.c                  0x00000000   Number         0  lis2dh.o ABSOLUTE
    ..\..\Hardware\lis2dh12_reg.c            0x00000000   Number         0  lis2dh12_reg.o ABSOLUTE
    ..\..\Hardware\lsm6d.c                   0x00000000   Number         0  lsm6d.o ABSOLUTE
    ..\..\Hardware\lsm6dso_reg.c             0x00000000   Number         0  lsm6dso_reg.o ABSOLUTE
    ..\..\Rtt\SEGGER_RTT.c                   0x00000000   Number         0  segger_rtt.o ABSOLUTE
    ..\..\Rtt\SEGGER_RTT_Syscalls_KEIL.c     0x00000000   Number         0  segger_rtt_syscalls_keil.o ABSOLUTE
    ..\..\Rtt\SEGGER_RTT_printf.c            0x00000000   Number         0  segger_rtt_printf.o ABSOLUTE
    ..\\..\\App\\app_adc.c                   0x00000000   Number         0  app_adc.o ABSOLUTE
    ..\\..\\App\\app_gpio.c                  0x00000000   Number         0  app_gpio.o ABSOLUTE
    ..\\..\\App\\app_timer.c                 0x00000000   Number         0  app_timer.o ABSOLUTE
    ..\\..\\Driver\\debug.c                  0x00000000   Number         0  debug.o ABSOLUTE
    ..\\..\\Driver\\delay.c                  0x00000000   Number         0  delay.o ABSOLUTE
    ..\\..\\Driver\\gpadc.c                  0x00000000   Number         0  gpadc.o ABSOLUTE
    ..\\..\\Driver\\gpio.c                   0x00000000   Number         0  gpio.o ABSOLUTE
    ..\\..\\Driver\\i2c.c                    0x00000000   Number         0  i2c.o ABSOLUTE
    ..\\..\\Driver\\ota.c                    0x00000000   Number         0  ota.o ABSOLUTE
    ..\\..\\Driver\\rtc_handler.c            0x00000000   Number         0  rtc_handler.o ABSOLUTE
    ..\\..\\Driver\\timer_handler.c          0x00000000   Number         0  timer_handler.o ABSOLUTE
    ..\\..\\Driver\\uart.c                   0x00000000   Number         0  uart.o ABSOLUTE
    ..\\..\\Driver\\wdt.c                    0x00000000   Number         0  wdt.o ABSOLUTE
    ..\\..\\Hardware\\lis2dh.c               0x00000000   Number         0  lis2dh.o ABSOLUTE
    ..\\..\\Hardware\\lsm6d.c                0x00000000   Number         0  lsm6d.o ABSOLUTE
    ..\\..\\Rtt\\SEGGER_RTT.c                0x00000000   Number         0  segger_rtt.o ABSOLUTE
    ..\\..\\Rtt\\SEGGER_RTT_Syscalls_KEIL.c  0x00000000   Number         0  segger_rtt_syscalls_keil.o ABSOLUTE
    ..\\..\\Rtt\\SEGGER_RTT_printf.c         0x00000000   Number         0  segger_rtt_printf.o ABSOLUTE
    ..\\isr.c                                0x00000000   Number         0  isr.o ABSOLUTE
    ..\\main.c                               0x00000000   Number         0  main.o ABSOLUTE
    ..\\mcu_bsp.c                            0x00000000   Number         0  mcu_bsp.o ABSOLUTE
    ..\isr.c                                 0x00000000   Number         0  isr.o ABSOLUTE
    ..\main.c                                0x00000000   Number         0  main.o ABSOLUTE
    ..\mcu_bsp.c                             0x00000000   Number         0  mcu_bsp.o ABSOLUTE
    Driver\\rtc.c                            0x00000000   Number         0  rtc.o ABSOLUTE
    Driver\\timer.c                          0x00000000   Number         0  timer.o ABSOLUTE
    Driver\rtc.c                             0x00000000   Number         0  rtc.o ABSOLUTE
    Driver\timer.c                           0x00000000   Number         0  timer.o ABSOLUTE
    Main\\main.c                             0x00000000   Number         0  main.o ABSOLUTE
    Main\main.c                              0x00000000   Number         0  main.o ABSOLUTE
    RTE\Device\ARMCM0\startup_ARMCM0.s       0x00000000   Number         0  startup_armcm0.o ABSOLUTE
    RTE\Device\ARMCM0\system_ARMCM0.c        0x00000000   Number         0  system_armcm0.o ABSOLUTE
    RTE\\Device\\ARMCM0\\system_ARMCM0.c     0x00000000   Number         0  system_armcm0.o ABSOLUTE
    cdcmple.s                                0x00000000   Number         0  cdcmple.o ABSOLUTE
    cdrcmple.s                               0x00000000   Number         0  cdrcmple.o ABSOLUTE
    dc.s                                     0x00000000   Number         0  dc.o ABSOLUTE
    handlers.s                               0x00000000   Number         0  handlers.o ABSOLUTE
    init.s                                   0x00000000   Number         0  init.o ABSOLUTE
    RESET                                    0x10000000   Section      192  startup_armcm0.o(RESET)
    .ARM.Collect$$$$00000000                 0x100000c0   Section        0  entry.o(.ARM.Collect$$$$00000000)
    .ARM.Collect$$$$00000001                 0x100000c0   Section        4  entry2.o(.ARM.Collect$$$$00000001)
    .ARM.Collect$$$$00000004                 0x100000c4   Section        4  entry5.o(.ARM.Collect$$$$00000004)
    .ARM.Collect$$$$00000008                 0x100000c8   Section        0  entry7b.o(.ARM.Collect$$$$00000008)
    .ARM.Collect$$$$0000000A                 0x100000c8   Section        0  entry8b.o(.ARM.Collect$$$$0000000A)
    .ARM.Collect$$$$0000000B                 0x100000c8   Section        8  entry9a.o(.ARM.Collect$$$$0000000B)
    .ARM.Collect$$$$0000000D                 0x100000d0   Section        0  entry10a.o(.ARM.Collect$$$$0000000D)
    .ARM.Collect$$$$0000000F                 0x100000d0   Section        0  entry11a.o(.ARM.Collect$$$$0000000F)
    .ARM.Collect$$$$00002712                 0x100000d0   Section        4  entry2.o(.ARM.Collect$$$$00002712)
    __lit__00000000                          0x100000d0   Data           4  entry2.o(.ARM.Collect$$$$00002712)
    .text                                    0x100000d4   Section        0  uart.o(.text)
    __NVIC_EnableIRQ                         0x10000559   Thumb Code    26  uart.o(.text)
    __NVIC_DisableIRQ                        0x10000573   Thumb Code    28  uart.o(.text)
    .text                                    0x10000598   Section        0  delay.o(.text)
    .text                                    0x100005d0   Section        0  gpio.o(.text)
    .text                                    0x10000b44   Section        0  i2c.o(.text)
    .text                                    0x10000f84   Section        0  gpadc.o(.text)
    .text                                    0x1000150c   Section        0  timer_handler.o(.text)
    .text                                    0x100015b8   Section        0  ota.o(.text)
    EvtCommandComplete                       0x100015b9   Thumb Code    46  ota.o(.text)
    Cmd4KSETTINGWrite                        0x100015fd   Thumb Code   120  ota.o(.text)
    CmdFwWriteStart                          0x10001675   Thumb Code    36  ota.o(.text)
    Cmd4KSETTINGUpgrade                      0x10001699   Thumb Code    80  ota.o(.text)
    CmdFwUpgradev20                          0x100016e9   Thumb Code   134  ota.o(.text)
    CmdFlashdataUpgradev30                   0x1000176f   Thumb Code   104  ota.o(.text)
    .text                                    0x10001ca8   Section        0  app_gpio.o(.text)
    .text                                    0x10001dc4   Section        0  app_timer.o(.text)
    .text                                    0x10001de8   Section        0  app_adc.o(.text)
    .text                                    0x10001e10   Section        0  lis2dh.o(.text)
    lis2dh12_xyz_axis_enable_set             0x10001e11   Thumb Code    94  lis2dh.o(.text)
    platform1_delay                          0x10001e6f   Thumb Code    12  lis2dh.o(.text)
    platform1_read                           0x10001e7b   Thumb Code    42  lis2dh.o(.text)
    platform1_write                          0x10001ea5   Thumb Code    42  lis2dh.o(.text)
    .text                                    0x10001fa4   Section        0  lsm6d.o(.text)
    platform0_delay                          0x10001fa5   Thumb Code    12  lsm6d.o(.text)
    platform0_read                           0x10001fb1   Thumb Code    42  lsm6d.o(.text)
    platform0_write                          0x10001fdb   Thumb Code    42  lsm6d.o(.text)
    Cadence_Stop_Judge                       0x10002095   Thumb Code    86  lsm6d.o(.text)
    .text                                    0x1000223c   Section        0  lis2dh12_reg.o(.text)
    .text                                    0x10003688   Section        0  lsm6dso_reg.o(.text)
    bytecpy                                  0x100036d5   Thumb Code    14  lsm6dso_reg.o(.text)
    .text                                    0x1000bc94   Section        0  cjson.o(.text)
    case_insensitive_strcmp                  0x1000bd0f   Thumb Code    76  cjson.o(.text)
    cJSON_strdup                             0x1000bd5b   Thumb Code    52  cjson.o(.text)
    cJSON_New_Item                           0x1000bde7   Thumb Code    28  cjson.o(.text)
    get_decimal_point                        0x1000be69   Thumb Code     4  cjson.o(.text)
    parse_number                             0x1000be6d   Thumb Code   298  cjson.o(.text)
    ensure                                   0x1000c04b   Thumb Code   248  cjson.o(.text)
    update_offset                            0x1000c143   Thumb Code    40  cjson.o(.text)
    compare_double                           0x1000c16b   Thumb Code   116  cjson.o(.text)
    print_number                             0x1000c1df   Thumb Code   278  cjson.o(.text)
    parse_hex4                               0x1000c2f5   Thumb Code    90  cjson.o(.text)
    utf16_literal_to_utf8                    0x1000c34f   Thumb Code   370  cjson.o(.text)
    parse_string                             0x1000c4c1   Thumb Code   406  cjson.o(.text)
    print_string_ptr                         0x1000c657   Thumb Code   370  cjson.o(.text)
    print_string                             0x1000c7c9   Thumb Code    16  cjson.o(.text)
    buffer_skip_whitespace                   0x1000c7d9   Thumb Code    80  cjson.o(.text)
    skip_utf8_bom                            0x1000c829   Thumb Code    66  cjson.o(.text)
    parse_object                             0x1000c86b   Thumb Code   340  cjson.o(.text)
    parse_array                              0x1000c9bf   Thumb Code   282  cjson.o(.text)
    parse_value                              0x1000cad9   Thumb Code   314  cjson.o(.text)
    print_object                             0x1000cd35   Thumb Code   396  cjson.o(.text)
    print_array                              0x1000cec1   Thumb Code   212  cjson.o(.text)
    print_value                              0x1000cf95   Thumb Code   238  cjson.o(.text)
    print                                    0x1000d083   Thumb Code   192  cjson.o(.text)
    get_array_item                           0x1000d21d   Thumb Code    32  cjson.o(.text)
    get_object_item                          0x1000d255   Thumb Code    94  cjson.o(.text)
    suffix_object                            0x1000d2f1   Thumb Code     6  cjson.o(.text)
    create_reference                         0x1000d2f7   Thumb Code    62  cjson.o(.text)
    add_item_to_array                        0x1000d335   Thumb Code    62  cjson.o(.text)
    cast_away_const                          0x1000d383   Thumb Code     2  cjson.o(.text)
    add_item_to_object                       0x1000d385   Thumb Code   146  cjson.o(.text)
    replace_item_in_object                   0x1000d95b   Thumb Code    90  cjson.o(.text)
    skip_oneline_comment                     0x1000dcf5   Thumb Code    42  cjson.o(.text)
    skip_multiline_comment                   0x1000dd1f   Thumb Code    50  cjson.o(.text)
    minify_string                            0x1000dd51   Thumb Code   122  cjson.o(.text)
    .text                                    0x1000e0b4   Section        0  crc16.o(.text)
    .text                                    0x1000e15c   Section        0  common.o(.text)
    .text                                    0x1000e190   Section        0  main.o(.text)
    __NVIC_SetPriority                       0x1000e191   Thumb Code   110  main.o(.text)
    PowerDown                                0x1000e1ff   Thumb Code   104  main.o(.text)
    timer_1_callback                         0x1000e29f   Thumb Code    44  main.o(.text)
    send_to_master                           0x1000e2cb   Thumb Code   202  main.o(.text)
    work_timer_event                         0x1000e3fd   Thumb Code   162  main.o(.text)
    timer_event_handler                      0x1000e65f   Thumb Code   118  main.o(.text)
    setup_adv_data                           0x1000e883   Thumb Code   174  main.o(.text)
    rf_stop                                  0x1000e931   Thumb Code     8  main.o(.text)
    ble_gatt_read                            0x1000e939   Thumb Code   192  main.o(.text)
    ble_gatt_write                           0x1000eaa9   Thumb Code   252  main.o(.text)
    ble_init                                 0x1000f099   Thumb Code   132  main.o(.text)
    .text                                    0x1000f6b8   Section        0  mcu_bsp.o(.text)
    BSP_TimerConfig                          0x1000f6b9   Thumb Code     8  mcu_bsp.o(.text)
    BSP_GPIOConfig                           0x1000f6c1   Thumb Code    24  mcu_bsp.o(.text)
    BSP_ADCConfig                            0x1000f6e5   Thumb Code     8  mcu_bsp.o(.text)
    .text                                    0x1000f6ec   Section        0  isr.o(.text)
    .text                                    0x1000f748   Section        0  segger_rtt.o(.text)
    _DoInit                                  0x1000f749   Thumb Code    74  segger_rtt.o(.text)
    _WriteBlocking                           0x1000f793   Thumb Code   122  segger_rtt.o(.text)
    _WriteNoCheck                            0x1000f80d   Thumb Code    74  segger_rtt.o(.text)
    _PostTerminalSwitch                      0x1000f857   Thumb Code    32  segger_rtt.o(.text)
    _GetAvailWriteSpace                      0x1000f877   Thumb Code    28  segger_rtt.o(.text)
    .text                                    0x10010274   Section        0  segger_rtt_printf.o(.text)
    _StoreChar                               0x10010275   Thumb Code    68  segger_rtt_printf.o(.text)
    _PrintUnsigned                           0x100102b9   Thumb Code   280  segger_rtt_printf.o(.text)
    _PrintInt                                0x100103d1   Thumb Code   270  segger_rtt_printf.o(.text)
    .text                                    0x10010818   Section       28  startup_armcm0.o(.text)
    .text                                    0x10010834   Section        0  system_armcm0.o(.text)
    .text                                    0x1001084c   Section        0  main.o(.text)
    _LCDisConnect                            0x1001084d   Thumb Code    46  main.o(.text)
    _LCTimer_Handler                         0x1001087b   Thumb Code   248  main.o(.text)
    _LCRxPkt_Handler                         0x1001098d   Thumb Code   280  main.o(.text)
    _LCTxPkt_Handler                         0x10010aa5   Thumb Code   316  main.o(.text)
    _LLENCReq                                0x10011375   Thumb Code   244  main.o(.text)
    _GAPStartAdv                             0x100119e3   Thumb Code   558  main.o(.text)
    WaitLLCOverSlpth                         0x10012d9d   Thumb Code    38  main.o(.text)
    _BBRXFIFORead                            0x10012dc3   Thumb Code   166  main.o(.text)
    _rom_rx_sweyntooth_protect               0x10012e69   Thumb Code   150  main.o(.text)
    STKSetRand                               0x10012eff   Thumb Code    30  main.o(.text)
    AttWriteFlash                            0x10012f1d   Thumb Code   110  main.o(.text)
    GetOverSlpth                             0x10012f8b   Thumb Code    26  main.o(.text)
    .text                                    0x10012fb4   Section        0  timer.o(.text)
    Timer_Evt_Trigger                        0x100130b1   Thumb Code   110  timer.o(.text)
    __NVIC_EnableIRQ                         0x100135bf   Thumb Code    18  timer.o(.text)
    __NVIC_DisableIRQ                        0x100135d1   Thumb Code    28  timer.o(.text)
    .text                                    0x100135f8   Section        0  rtc.o(.text)
    Timer_RTCEVT_Trigger                     0x10013787   Thumb Code   150  rtc.o(.text)
    .text                                    0x10013bc0   Section        0  uidiv.o(.text)
    .text                                    0x10013bec   Section        0  idiv.o(.text)
    .text                                    0x10013c14   Section        0  tolower.o(.text)
    .text                                    0x10013c20   Section        0  memcpya.o(.text)
    .text                                    0x10013c44   Section        0  memseta.o(.text)
    .text                                    0x10013c68   Section        0  strlen.o(.text)
    .text                                    0x10013c76   Section        0  strcmp.o(.text)
    .text                                    0x10013c92   Section        0  memcmp.o(.text)
    .text                                    0x10013cac   Section        0  strcpy.o(.text)
    .text                                    0x10013cbe   Section        0  strncmp.o(.text)
    .text                                    0x10013cdc   Section        0  uread4.o(.text)
    .text                                    0x10013cf0   Section        0  uwrite4.o(.text)
    .text                                    0x10013d04   Section        0  __0sscanf.o(.text)
    .text                                    0x10013d40   Section        0  scanf_fp.o(.text)
    _fp_value                                0x10013d41   Thumb Code   286  scanf_fp.o(.text)
    .text                                    0x100140b4   Section        0  fadd.o(.text)
    .text                                    0x10014166   Section        0  fmul.o(.text)
    .text                                    0x100141e0   Section        0  fdiv.o(.text)
    .text                                    0x1001425c   Section        0  dadd.o(.text)
    .text                                    0x100143c0   Section        0  dmul.o(.text)
    .text                                    0x10014490   Section        0  ddiv.o(.text)
    .text                                    0x10014580   Section        0  fflti.o(.text)
    .text                                    0x10014596   Section        0  ffltui.o(.text)
    .text                                    0x100145a4   Section        0  dflti.o(.text)
    .text                                    0x100145cc   Section        0  dfltui.o(.text)
    .text                                    0x100145e8   Section        0  ffixi.o(.text)
    .text                                    0x1001461c   Section        0  dfixi.o(.text)
    .text                                    0x10014664   Section        0  dfixui.o(.text)
    .text                                    0x100146a0   Section        0  f2d.o(.text)
    .text                                    0x100146c8   Section       40  cdcmple.o(.text)
    .text                                    0x100146f0   Section       40  cdrcmple.o(.text)
    .text                                    0x10014718   Section        0  d2f.o(.text)
    .text                                    0x10014750   Section        0  uldiv.o(.text)
    .text                                    0x100147b0   Section        0  llmul.o(.text)
    .text                                    0x1001482a   Section        0  llshl.o(.text)
    .text                                    0x1001484a   Section        0  llushr.o(.text)
    .text                                    0x1001486c   Section        0  llsshr.o(.text)
    .text                                    0x10014894   Section        0  scanf_char.o(.text)
    _scanf_char_input                        0x10014895   Thumb Code    12  scanf_char.o(.text)
    .text                                    0x100148c0   Section        0  _sgetc.o(.text)
    .text                                    0x10014904   Section        0  strtod.o(.text)
    _local_sscanf                            0x10014905   Thumb Code    54  strtod.o(.text)
    .text                                    0x100149a8   Section        0  iusefp.o(.text)
    .text                                    0x100149a8   Section        0  fepilogue.o(.text)
    .text                                    0x10014a2a   Section        0  depilogue.o(.text)
    .text                                    0x10014ae8   Section        0  dfltul.o(.text)
    .text                                    0x10014b04   Section        0  dfixul.o(.text)
    .text                                    0x10014b44   Section       36  init.o(.text)
    .text                                    0x10014b68   Section        0  isspace_c.o(.text)
    .text                                    0x10014b78   Section        0  _scanf.o(.text)
    .text                                    0x10014eb0   Section        0  ctype_c.o(.text)
    .text                                    0x10014ed4   Section        0  __dczerorl2.o(.text)
    i.__0sprintf                             0x10014f2c   Section        0  printfa.o(i.__0sprintf)
    i.__ARM_clz                              0x10014f54   Section        0  depilogue.o(i.__ARM_clz)
    i.__ARM_common_switch8                   0x10014f82   Section        0  main.o(i.__ARM_common_switch8)
    i.__free$realloc                         0x10014f9c   Section        0  mallocr.o(i.__free$realloc)
    i.__malloc$realloc                       0x10015000   Section        0  mallocr.o(i.__malloc$realloc)
    i.__scatterload_copy                     0x10015048   Section       14  handlers.o(i.__scatterload_copy)
    i.__scatterload_null                     0x10015056   Section        2  handlers.o(i.__scatterload_null)
    i.__scatterload_zeroinit                 0x10015058   Section       14  handlers.o(i.__scatterload_zeroinit)
    i._fp_digits                             0x10015068   Section        0  printfa.o(i._fp_digits)
    _fp_digits                               0x10015069   Thumb Code   344  printfa.o(i._fp_digits)
    i._is_digit                              0x100151dc   Section        0  scanf_fp.o(i._is_digit)
    i._printf_core                           0x100151ec   Section        0  printfa.o(i._printf_core)
    _printf_core                             0x100151ed   Thumb Code  1754  printfa.o(i._printf_core)
    i._printf_post_padding                   0x100158d8   Section        0  printfa.o(i._printf_post_padding)
    _printf_post_padding                     0x100158d9   Thumb Code    32  printfa.o(i._printf_post_padding)
    i._printf_pre_padding                    0x100158f8   Section        0  printfa.o(i._printf_pre_padding)
    _printf_pre_padding                      0x100158f9   Thumb Code    44  printfa.o(i._printf_pre_padding)
    i._sputc                                 0x10015924   Section        0  printfa.o(i._sputc)
    _sputc                                   0x10015925   Thumb Code    10  printfa.o(i._sputc)
    i.internal_alloc                         0x10015930   Section        0  mallocr.o(i.internal_alloc)
    internal_alloc                           0x10015931   Thumb Code    74  mallocr.o(i.internal_alloc)
    i.realloc                                0x10015980   Section        0  mallocr.o(i.realloc)
    i.strtod                                 0x100159f4   Section        0  strtod.o(i.strtod)
    .constdata                               0x10015a10   Section      512  crc16.o(.constdata)
    crc16tab                                 0x10015a10   Data         512  crc16.o(.constdata)
    .constdata                               0x10015c10   Section       16  segger_rtt_printf.o(.constdata)
    _aV2C                                    0x10015c10   Data          16  segger_rtt_printf.o(.constdata)
    .constdata                               0x10015c20   Section       40  main.o(.constdata)
    _ll_packet_length                        0x10015c23   Data          15  main.o(.constdata)
    _smp_packet_lenght                       0x10015c32   Data          22  main.o(.constdata)
    .constdata                               0x10015c48   Section       64  ctype_c.o(.constdata)
    .data                                    0x20003000   Section        8  uart.o(.data)
    UART_0_CTRL                              0x20003000   Data           4  uart.o(.data)
    UART_1_CTRL                              0x20003004   Data           4  uart.o(.data)
    .data                                    0x20003008   Section       72  gpio.o(.data)
    gpio_callback                            0x2000301c   Data           4  gpio.o(.data)
    pinmuxtab48                              0x20003020   Data          24  gpio.o(.data)
    pinmuxtab32                              0x20003038   Data          24  gpio.o(.data)
    .data                                    0x20003050   Section       24  i2c.o(.data)
    I2C_0_CTRL                               0x20003050   Data           4  i2c.o(.data)
    I2C_0_TXD                                0x20003054   Data           4  i2c.o(.data)
    I2C_0_RXD                                0x20003058   Data           4  i2c.o(.data)
    I2C_1_CTRL                               0x2000305c   Data           4  i2c.o(.data)
    I2C_1_TXD                                0x20003060   Data           4  i2c.o(.data)
    I2C_1_RXD                                0x20003064   Data           4  i2c.o(.data)
    .data                                    0x20003068   Section       12  gpadc.o(.data)
    adc_callback                             0x20003070   Data           4  gpadc.o(.data)
    .data                                    0x20003074   Section        4  rtc_handler.o(.data)
    .data                                    0x20003078   Section       28  ota.o(.data)
    EvtBuf                                   0x20003088   Data           8  ota.o(.data)
    .data                                    0x20003094   Section       39  lsm6d.o(.data)
    data_raw_acc                             0x20003098   Data           6  lsm6d.o(.data)
    data_raw_ang                             0x2000309e   Data           6  lsm6d.o(.data)
    data_acc_offset                          0x200030a4   Data           6  lsm6d.o(.data)
    data_ang_offset                          0x200030aa   Data           6  lsm6d.o(.data)
    gyro_z                                   0x200030b0   Data           4  lsm6d.o(.data)
    cntTimes                                 0x200030b4   Data           1  lsm6d.o(.data)
    Last_theta                               0x200030b6   Data           2  lsm6d.o(.data)
    temp                                     0x200030b8   Data           2  lsm6d.o(.data)
    ActFlag                                  0x200030ba   Data           1  lsm6d.o(.data)
    .data                                    0x200030bc   Section       20  cjson.o(.data)
    global_error                             0x200030bc   Data           8  cjson.o(.data)
    global_hooks                             0x200030c4   Data          12  cjson.o(.data)
    .data                                    0x200030d0   Section      103  main.o(.data)
    dev_addr                                 0x200030d0   Data           7  main.o(.data)
    work_led_count                           0x200030d7   Data           1  main.o(.data)
    Device_Name_Array                        0x200030d8   Data          12  main.o(.data)
    hex                                      0x200030e4   Data          17  main.o(.data)
    g_report                                 0x200030f8   Data           4  main.o(.data)
    latency_state                            0x200030fe   Data           1  main.o(.data)
    spp_delay_cnt                            0x20003100   Data           2  main.o(.data)
    count                                    0x20003134   Data           1  main.o(.data)
    batteryPercenttemp                       0x20003135   Data           2  main.o(.data)
    .data                                    0x20003137   Section       17  segger_rtt.o(.data)
    _aTerminalId                             0x20003137   Data          16  segger_rtt.o(.data)
    _ActiveTerminal                          0x20003147   Data           1  segger_rtt.o(.data)
    .data                                    0x20003148   Section        4  system_armcm0.o(.data)
    .data                                    0x2000314c   Section       64  main.o(.data)
    syd_confirm                              0x2000314c   Data           1  main.o(.data)
    ww_minus_cnt                             0x2000314d   Data           1  main.o(.data)
    ext_uart_en                              0x2000314e   Data           1  main.o(.data)
    get_bond_device_idx                      0x2000314f   Data           1  main.o(.data)
    _valid_l2cap_lenght                      0x20003150   Data           1  main.o(.data)
    rssi_rx                                  0x20003152   Data           1  main.o(.data)
    p_flash_hdr                              0x20003154   Data           4  main.o(.data)
    p_lclink                                 0x20003158   Data           4  main.o(.data)
    p_txpdu                                  0x2000315c   Data           4  main.o(.data)
    p_rxbuf                                  0x20003160   Data           4  main.o(.data)
    p_flash                                  0x20003164   Data           4  main.o(.data)
    p_dump_key                               0x2000316c   Data           4  main.o(.data)
    EFUSE_CTRL                               0x20003170   Data           4  main.o(.data)
    BB_CTRL                                  0x20003174   Data           4  main.o(.data)
    PW_CTRL                                  0x20003178   Data           4  main.o(.data)
    PIN_CONFIG                               0x2000317c   Data           4  main.o(.data)
    CONFIG_FLASH_SIZE                        0x20003180   Data           4  main.o(.data)
    g_evt                                    0x20003184   Data           8  main.o(.data)
    .data                                    0x2000318c   Section       28  timer.o(.data)
    TIMER_CTRL                               0x20003190   Data           4  timer.o(.data)
    .data                                    0x200031a8   Section       40  rtc.o(.data)
    enabled                                  0x200031a8   Data           1  rtc.o(.data)
    irq_cb                                   0x200031c8   Data           4  rtc.o(.data)
    .data                                    0x200031d0   Section        4  mvars.o(.data)
    .data                                    0x200031d4   Section        4  mvars.o(.data)
    .bss                                     0x200031d8   Section      120  timer_handler.o(.bss)
    .bss                                     0x20003250   Section       40  ota.o(.bss)
    .bss                                     0x20003278   Section       16  lis2dh.o(.bss)
    .bss                                     0x20003288   Section       42  lsm6d.o(.bss)
    .bss                                     0x200032b2   Section       15  cjson.o(.bss)
    version                                  0x200032b2   Data          15  cjson.o(.bss)
    .bss                                     0x200032c4   Section     1032  main.o(.bss)
    .bss                                     0x200036cc   Section     1112  segger_rtt.o(.bss)
    _acUpBuffer                              0x20003714   Data        1024  segger_rtt.o(.bss)
    _acDownBuffer                            0x20003b14   Data          16  segger_rtt.o(.bss)
    .bss                                     0x20003b24   Section      104  main.o(.bss)
    code_hdr                                 0x20003b24   Data          87  main.o(.bss)
    smart_update_ctrol                       0x20003b7b   Data          17  main.o(.bss)
    .bss                                     0x20003b8c   Section       12  timer.o(.bss)
    timer_callback                           0x20003b8c   Data          12  timer.o(.bss)
    HEAP                                     0x20003b98   Section     3072  startup_armcm0.o(HEAP)
    STACK                                    0x20004798   Section     1024  startup_armcm0.o(STACK)

    Global Symbols

    Symbol Name                              Value     Ov Type        Size  Object(Section)

    BuildAttributes$$THM_ISAv3M$S$PE$A:L22$X:L11$S22$IEEE1$IW$USESV6$~STKCKD$USESV7$~SHL$OTIME$ROPI$IEEEJ$EBA8$MICROLIB$REQ8$PRES8$EABIv2 0x00000000   Number         0  anon$$obj.o ABSOLUTE
    __ARM_use_no_argv                        0x00000000   Number         0  main.o ABSOLUTE
    __use_no_errno                           0x00000000   Number         0  useno.o ABSOLUTE
    __use_no_exception_handling              0x00000000   Number         0  useno.o ABSOLUTE
    __use_no_fp                              0x00000000   Number         0  useno.o ABSOLUTE
    __use_no_heap                            0x00000000   Number         0  useno.o ABSOLUTE
    __use_no_heap_region                     0x00000000   Number         0  useno.o ABSOLUTE
    __use_no_semihosting                     0x00000000   Number         0  useno.o ABSOLUTE
    __use_no_semihosting_swi                 0x00000000   Number         0  useno.o ABSOLUTE
    __use_no_signal_handling                 0x00000000   Number         0  useno.o ABSOLUTE
    _printf_a                                0x00000000   Number         0  stubs.o ABSOLUTE
    _printf_c                                0x00000000   Number         0  stubs.o ABSOLUTE
    _printf_charcount                        0x00000000   Number         0  stubs.o ABSOLUTE
    _printf_d                                0x00000000   Number         0  stubs.o ABSOLUTE
    _printf_e                                0x00000000   Number         0  stubs.o ABSOLUTE
    _printf_f                                0x00000000   Number         0  stubs.o ABSOLUTE
    _printf_flags                            0x00000000   Number         0  stubs.o ABSOLUTE
    _printf_fp_dec                           0x00000000   Number         0  stubs.o ABSOLUTE
    _printf_fp_hex                           0x00000000   Number         0  stubs.o ABSOLUTE
    _printf_g                                0x00000000   Number         0  stubs.o ABSOLUTE
    _printf_i                                0x00000000   Number         0  stubs.o ABSOLUTE
    _printf_int_dec                          0x00000000   Number         0  stubs.o ABSOLUTE
    _printf_l                                0x00000000   Number         0  stubs.o ABSOLUTE
    _printf_lc                               0x00000000   Number         0  stubs.o ABSOLUTE
    _printf_ll                               0x00000000   Number         0  stubs.o ABSOLUTE
    _printf_lld                              0x00000000   Number         0  stubs.o ABSOLUTE
    _printf_lli                              0x00000000   Number         0  stubs.o ABSOLUTE
    _printf_llo                              0x00000000   Number         0  stubs.o ABSOLUTE
    _printf_llu                              0x00000000   Number         0  stubs.o ABSOLUTE
    _printf_llx                              0x00000000   Number         0  stubs.o ABSOLUTE
    _printf_longlong_dec                     0x00000000   Number         0  stubs.o ABSOLUTE
    _printf_longlong_hex                     0x00000000   Number         0  stubs.o ABSOLUTE
    _printf_longlong_oct                     0x00000000   Number         0  stubs.o ABSOLUTE
    _printf_ls                               0x00000000   Number         0  stubs.o ABSOLUTE
    _printf_mbtowc                           0x00000000   Number         0  stubs.o ABSOLUTE
    _printf_n                                0x00000000   Number         0  stubs.o ABSOLUTE
    _printf_o                                0x00000000   Number         0  stubs.o ABSOLUTE
    _printf_p                                0x00000000   Number         0  stubs.o ABSOLUTE
    _printf_percent                          0x00000000   Number         0  stubs.o ABSOLUTE
    _printf_pre_padding                      0x00000000   Number         0  stubs.o ABSOLUTE
    _printf_return_value                     0x00000000   Number         0  stubs.o ABSOLUTE
    _printf_s                                0x00000000   Number         0  stubs.o ABSOLUTE
    _printf_sizespec                         0x00000000   Number         0  stubs.o ABSOLUTE
    _printf_str                              0x00000000   Number         0  stubs.o ABSOLUTE
    _printf_truncate_signed                  0x00000000   Number         0  stubs.o ABSOLUTE
    _printf_truncate_unsigned                0x00000000   Number         0  stubs.o ABSOLUTE
    _printf_u                                0x00000000   Number         0  stubs.o ABSOLUTE
    _printf_wc                               0x00000000   Number         0  stubs.o ABSOLUTE
    _printf_wctomb                           0x00000000   Number         0  stubs.o ABSOLUTE
    _printf_widthprec                        0x00000000   Number         0  stubs.o ABSOLUTE
    _printf_x                                0x00000000   Number         0  stubs.o ABSOLUTE
    __cpp_initialize__aeabi_                  - Undefined Weak Reference
    __cxa_finalize                            - Undefined Weak Reference
    _clock_init                               - Undefined Weak Reference
    _microlib_exit                            - Undefined Weak Reference
    _scanf_int                                - Undefined Weak Reference
    _scanf_longlong                           - Undefined Weak Reference
    _scanf_string                             - Undefined Weak Reference
    __Vectors_Size                           0x000000c0   Number         0  startup_armcm0.o ABSOLUTE
    __Vectors                                0x10000000   Data           4  startup_armcm0.o(RESET)
    __Vectors_End                            0x100000c0   Data           0  startup_armcm0.o(RESET)
    __main                                   0x100000c1   Thumb Code     0  entry.o(.ARM.Collect$$$$00000000)
    _main_stk                                0x100000c1   Thumb Code     0  entry2.o(.ARM.Collect$$$$00000001)
    _main_scatterload                        0x100000c5   Thumb Code     0  entry5.o(.ARM.Collect$$$$00000004)
    __main_after_scatterload                 0x100000c9   Thumb Code     0  entry5.o(.ARM.Collect$$$$00000004)
    _main_clock                              0x100000c9   Thumb Code     0  entry7b.o(.ARM.Collect$$$$00000008)
    _main_cpp_init                           0x100000c9   Thumb Code     0  entry8b.o(.ARM.Collect$$$$0000000A)
    _main_init                               0x100000c9   Thumb Code     0  entry9a.o(.ARM.Collect$$$$0000000B)
    __rt_final_cpp                           0x100000d1   Thumb Code     0  entry10a.o(.ARM.Collect$$$$0000000D)
    __rt_final_exit                          0x100000d1   Thumb Code     0  entry11a.o(.ARM.Collect$$$$0000000F)
    uart_0_init                              0x100000d5   Thumb Code   340  uart.o(.text)
    uart_0_write                             0x10000229   Thumb Code    40  uart.o(.text)
    uart_0_read                              0x10000251   Thumb Code    72  uart.o(.text)
    uart_0_close                             0x10000299   Thumb Code    26  uart.o(.text)
    UART0_IRQHandler                         0x100002b3   Thumb Code   106  uart.o(.text)
    uart_1_init                              0x1000031d   Thumb Code   338  uart.o(.text)
    uart_1_write                             0x1000046f   Thumb Code    40  uart.o(.text)
    uart_1_read                              0x10000497   Thumb Code    86  uart.o(.text)
    uart_1_close                             0x100004ed   Thumb Code    26  uart.o(.text)
    uartRx_callback                          0x10000507   Thumb Code    12  uart.o(.text)
    UART1_IRQHandler                         0x10000513   Thumb Code    70  uart.o(.text)
    delay_ms                                 0x10000599   Thumb Code    30  delay.o(.text)
    delay_us                                 0x100005b7   Thumb Code    26  delay.o(.text)
    PIN_Set_GPIO                             0x100005d1   Thumb Code    50  gpio.o(.text)
    PIN_Pullup_Enable                        0x10000603   Thumb Code   150  gpio.o(.text)
    PIN_Pullup_Disable                       0x10000699   Thumb Code   148  gpio.o(.text)
    GPIO_Set_Output                          0x1000072d   Thumb Code    50  gpio.o(.text)
    GPIO_Set_Input                           0x1000075f   Thumb Code   200  gpio.o(.text)
    GPIO_Set_Input_DIR                       0x10000827   Thumb Code    50  gpio.o(.text)
    GPIO_Input_Enable                        0x10000859   Thumb Code    50  gpio.o(.text)
    GPIO_Input_Disable                       0x1000088b   Thumb Code    50  gpio.o(.text)
    GPIO_Pin_Set                             0x100008bd   Thumb Code    50  gpio.o(.text)
    GPIO_Pin_Clear                           0x100008ef   Thumb Code    50  gpio.o(.text)
    GPIO_Pin_Turn                            0x10000921   Thumb Code    50  gpio.o(.text)
    GPIO_Pin_Read                            0x10000953   Thumb Code    34  gpio.o(.text)
    io_irq_enable                            0x10000975   Thumb Code   192  gpio.o(.text)
    io_irq_disable                           0x10000a35   Thumb Code    52  gpio.o(.text)
    io_irq_disable_all                       0x10000a69   Thumb Code    76  gpio.o(.text)
    GPIO_IRQHandler                          0x10000ab5   Thumb Code   132  gpio.o(.text)
    i2c_Init                                 0x10000b45   Thumb Code   132  i2c.o(.text)
    i2c_0_write                              0x10000bc9   Thumb Code   232  i2c.o(.text)
    i2c_0_read                               0x10000cb1   Thumb Code   234  i2c.o(.text)
    i2c_1_write                              0x10000d9b   Thumb Code   232  i2c.o(.text)
    i2c_1_read                               0x10000e83   Thumb Code   258  i2c.o(.text)
    GPADC_channel_sel                        0x10000f85   Thumb Code    48  gpadc.o(.text)
    GPADC_Init                               0x10000fb5   Thumb Code  1064  gpadc.o(.text)
    GPADC_start                              0x100013dd   Thumb Code    50  gpadc.o(.text)
    GPADC_stop                               0x1000140f   Thumb Code   142  gpadc.o(.text)
    GPADC_get_value                          0x1000149d   Thumb Code    20  gpadc.o(.text)
    GPADC_IRQHandler                         0x100014b1   Thumb Code    78  gpadc.o(.text)
    Timer_Evt_2s                             0x1000150d   Thumb Code    14  timer_handler.o(.text)
    Timer_EVT_1S_OTA                         0x1000151b   Thumb Code    14  timer_handler.o(.text)
    Timer_EVT_1S_WORK                        0x10001529   Thumb Code    14  timer_handler.o(.text)
    Timer_EVT_300MS_PCAK                     0x10001537   Thumb Code    14  timer_handler.o(.text)
    Timer_EVT_20S_BATTERY                    0x10001545   Thumb Code    14  timer_handler.o(.text)
    Timer_Evt_List                           0x10001553   Thumb Code    72  timer_handler.o(.text)
    CmdFwErase                               0x100015e7   Thumb Code    22  ota.o(.text)
    ota_variable_clear                       0x100017d7   Thumb Code    38  ota.o(.text)
    ota_cmd                                  0x100017fd   Thumb Code  1042  ota.o(.text)
    ota_rsp                                  0x10001c0f   Thumb Code    42  ota.o(.text)
    LED_IO_Config                            0x10001ca9   Thumb Code    24  app_gpio.o(.text)
    State_IO_Config                          0x10001cc1   Thumb Code    42  app_gpio.o(.text)
    IIC_IO_Config                            0x10001ceb   Thumb Code    26  app_gpio.o(.text)
    Ctr_IO_Config                            0x10001d05   Thumb Code   108  app_gpio.o(.text)
    INT_IO_Config                            0x10001d71   Thumb Code    78  app_gpio.o(.text)
    Timer_Config                             0x10001dc5   Thumb Code     8  app_timer.o(.text)
    Timer2_Enable                            0x10001dcd   Thumb Code    12  app_timer.o(.text)
    Timer2_Disable                           0x10001dd9   Thumb Code     8  app_timer.o(.text)
    ADC_Config                               0x10001de9   Thumb Code    38  app_adc.o(.text)
    Lis2dh_Init                              0x10001ecf   Thumb Code   126  lis2dh.o(.text)
    Lis2dh_Act_State_Judge                   0x10001f4d   Thumb Code    42  lis2dh.o(.text)
    Lsm6dso_Init                             0x10002005   Thumb Code   144  lsm6d.o(.text)
    Lsm6dso_RPM_Cal                          0x100020eb   Thumb Code   248  lsm6d.o(.text)
    Lsm6dso_Disable                          0x100021e3   Thumb Code    12  lsm6d.o(.text)
    lis2dh12_read_reg                        0x1000223d   Thumb Code    38  lis2dh12_reg.o(.text)
    lis2dh12_write_reg                       0x10002263   Thumb Code    38  lis2dh12_reg.o(.text)
    lis2dh12_from_fs2_hr_to_mg               0x10002289   Thumb Code    32  lis2dh12_reg.o(.text)
    lis2dh12_from_fs4_hr_to_mg               0x100022a9   Thumb Code    32  lis2dh12_reg.o(.text)
    lis2dh12_from_fs8_hr_to_mg               0x100022c9   Thumb Code    32  lis2dh12_reg.o(.text)
    lis2dh12_from_fs16_hr_to_mg              0x100022e9   Thumb Code    30  lis2dh12_reg.o(.text)
    lis2dh12_from_lsb_hr_to_celsius          0x10002307   Thumb Code    40  lis2dh12_reg.o(.text)
    lis2dh12_from_fs2_nm_to_mg               0x1000232f   Thumb Code    32  lis2dh12_reg.o(.text)
    lis2dh12_from_fs4_nm_to_mg               0x1000234f   Thumb Code    32  lis2dh12_reg.o(.text)
    lis2dh12_from_fs8_nm_to_mg               0x1000236f   Thumb Code    32  lis2dh12_reg.o(.text)
    lis2dh12_from_fs16_nm_to_mg              0x1000238f   Thumb Code    30  lis2dh12_reg.o(.text)
    lis2dh12_from_lsb_nm_to_celsius          0x100023ad   Thumb Code    40  lis2dh12_reg.o(.text)
    lis2dh12_from_fs2_lp_to_mg               0x100023d5   Thumb Code    32  lis2dh12_reg.o(.text)
    lis2dh12_from_fs4_lp_to_mg               0x100023f5   Thumb Code    32  lis2dh12_reg.o(.text)
    lis2dh12_from_fs8_lp_to_mg               0x10002415   Thumb Code    32  lis2dh12_reg.o(.text)
    lis2dh12_from_fs16_lp_to_mg              0x10002435   Thumb Code    30  lis2dh12_reg.o(.text)
    lis2dh12_from_lsb_lp_to_celsius          0x10002453   Thumb Code    40  lis2dh12_reg.o(.text)
    lis2dh12_temp_status_reg_get             0x1000247b   Thumb Code    24  lis2dh12_reg.o(.text)
    lis2dh12_temp_data_ready_get             0x10002493   Thumb Code    34  lis2dh12_reg.o(.text)
    lis2dh12_temp_data_ovr_get               0x100024b5   Thumb Code    34  lis2dh12_reg.o(.text)
    lis2dh12_temperature_raw_get             0x100024d7   Thumb Code    44  lis2dh12_reg.o(.text)
    lis2dh12_temperature_meas_set            0x10002503   Thumb Code    60  lis2dh12_reg.o(.text)
    lis2dh12_temperature_meas_get            0x1000253f   Thumb Code    60  lis2dh12_reg.o(.text)
    lis2dh12_operating_mode_set              0x1000257b   Thumb Code   150  lis2dh12_reg.o(.text)
    lis2dh12_operating_mode_get              0x10002611   Thumb Code    82  lis2dh12_reg.o(.text)
    lis2dh12_data_rate_set                   0x10002663   Thumb Code    60  lis2dh12_reg.o(.text)
    lis2dh12_data_rate_get                   0x1000269f   Thumb Code   132  lis2dh12_reg.o(.text)
    lis2dh12_high_pass_on_outputs_set        0x10002723   Thumb Code    60  lis2dh12_reg.o(.text)
    lis2dh12_high_pass_on_outputs_get        0x1000275f   Thumb Code    34  lis2dh12_reg.o(.text)
    lis2dh12_high_pass_bandwidth_set         0x10002781   Thumb Code    60  lis2dh12_reg.o(.text)
    lis2dh12_high_pass_bandwidth_get         0x100027bd   Thumb Code    82  lis2dh12_reg.o(.text)
    lis2dh12_high_pass_mode_set              0x1000280f   Thumb Code    60  lis2dh12_reg.o(.text)
    lis2dh12_high_pass_mode_get              0x1000284b   Thumb Code    80  lis2dh12_reg.o(.text)
    lis2dh12_full_scale_set                  0x1000289b   Thumb Code    60  lis2dh12_reg.o(.text)
    lis2dh12_full_scale_get                  0x100028d7   Thumb Code    82  lis2dh12_reg.o(.text)
    lis2dh12_block_data_update_set           0x10002929   Thumb Code    60  lis2dh12_reg.o(.text)
    lis2dh12_block_data_update_get           0x10002965   Thumb Code    32  lis2dh12_reg.o(.text)
    lis2dh12_filter_reference_set            0x10002985   Thumb Code    24  lis2dh12_reg.o(.text)
    lis2dh12_filter_reference_get            0x1000299d   Thumb Code    24  lis2dh12_reg.o(.text)
    lis2dh12_xl_data_ready_get               0x100029b5   Thumb Code    34  lis2dh12_reg.o(.text)
    lis2dh12_xl_data_ovr_get                 0x100029d7   Thumb Code    32  lis2dh12_reg.o(.text)
    lis2dh12_acceleration_raw_get            0x100029f7   Thumb Code    84  lis2dh12_reg.o(.text)
    lis2dh12_device_id_get                   0x10002a4b   Thumb Code    24  lis2dh12_reg.o(.text)
    lis2dh12_self_test_set                   0x10002a63   Thumb Code    60  lis2dh12_reg.o(.text)
    lis2dh12_self_test_get                   0x10002a9f   Thumb Code    72  lis2dh12_reg.o(.text)
    lis2dh12_data_format_set                 0x10002ae7   Thumb Code    60  lis2dh12_reg.o(.text)
    lis2dh12_data_format_get                 0x10002b23   Thumb Code    62  lis2dh12_reg.o(.text)
    lis2dh12_boot_set                        0x10002b61   Thumb Code    60  lis2dh12_reg.o(.text)
    lis2dh12_boot_get                        0x10002b9d   Thumb Code    32  lis2dh12_reg.o(.text)
    lis2dh12_status_get                      0x10002bbd   Thumb Code    24  lis2dh12_reg.o(.text)
    lis2dh12_int1_gen_conf_set               0x10002bd5   Thumb Code    24  lis2dh12_reg.o(.text)
    lis2dh12_int1_gen_conf_get               0x10002bed   Thumb Code    24  lis2dh12_reg.o(.text)
    lis2dh12_int1_gen_source_get             0x10002c05   Thumb Code    24  lis2dh12_reg.o(.text)
    lis2dh12_int1_gen_threshold_set          0x10002c1d   Thumb Code    58  lis2dh12_reg.o(.text)
    lis2dh12_int1_gen_threshold_get          0x10002c57   Thumb Code    34  lis2dh12_reg.o(.text)
    lis2dh12_int1_gen_duration_set           0x10002c79   Thumb Code    58  lis2dh12_reg.o(.text)
    lis2dh12_int1_gen_duration_get           0x10002cb3   Thumb Code    34  lis2dh12_reg.o(.text)
    lis2dh12_int2_gen_conf_set               0x10002cd5   Thumb Code    24  lis2dh12_reg.o(.text)
    lis2dh12_int2_gen_conf_get               0x10002ced   Thumb Code    24  lis2dh12_reg.o(.text)
    lis2dh12_int2_gen_source_get             0x10002d05   Thumb Code    24  lis2dh12_reg.o(.text)
    lis2dh12_int2_gen_threshold_set          0x10002d1d   Thumb Code    58  lis2dh12_reg.o(.text)
    lis2dh12_int2_gen_threshold_get          0x10002d57   Thumb Code    34  lis2dh12_reg.o(.text)
    lis2dh12_int2_gen_duration_set           0x10002d79   Thumb Code    58  lis2dh12_reg.o(.text)
    lis2dh12_int2_gen_duration_get           0x10002db3   Thumb Code    34  lis2dh12_reg.o(.text)
    lis2dh12_high_pass_int_conf_set          0x10002dd5   Thumb Code    58  lis2dh12_reg.o(.text)
    lis2dh12_high_pass_int_conf_get          0x10002e0f   Thumb Code   104  lis2dh12_reg.o(.text)
    lis2dh12_pin_int1_config_set             0x10002e77   Thumb Code    24  lis2dh12_reg.o(.text)
    lis2dh12_pin_int1_config_get             0x10002e8f   Thumb Code    24  lis2dh12_reg.o(.text)
    lis2dh12_int2_pin_detect_4d_set          0x10002ea7   Thumb Code    58  lis2dh12_reg.o(.text)
    lis2dh12_int2_pin_detect_4d_get          0x10002ee1   Thumb Code    34  lis2dh12_reg.o(.text)
    lis2dh12_int2_pin_notification_mode_set  0x10002f03   Thumb Code    60  lis2dh12_reg.o(.text)
    lis2dh12_int2_pin_notification_mode_get  0x10002f3f   Thumb Code    62  lis2dh12_reg.o(.text)
    lis2dh12_int1_pin_detect_4d_set          0x10002f7d   Thumb Code    60  lis2dh12_reg.o(.text)
    lis2dh12_int1_pin_detect_4d_get          0x10002fb9   Thumb Code    34  lis2dh12_reg.o(.text)
    lis2dh12_int1_pin_notification_mode_set  0x10002fdb   Thumb Code    60  lis2dh12_reg.o(.text)
    lis2dh12_int1_pin_notification_mode_get  0x10003017   Thumb Code    62  lis2dh12_reg.o(.text)
    lis2dh12_pin_int2_config_set             0x10003055   Thumb Code    24  lis2dh12_reg.o(.text)
    lis2dh12_pin_int2_config_get             0x1000306d   Thumb Code    24  lis2dh12_reg.o(.text)
    lis2dh12_fifo_set                        0x10003085   Thumb Code    60  lis2dh12_reg.o(.text)
    lis2dh12_fifo_get                        0x100030c1   Thumb Code    34  lis2dh12_reg.o(.text)
    lis2dh12_fifo_watermark_set              0x100030e3   Thumb Code    58  lis2dh12_reg.o(.text)
    lis2dh12_fifo_watermark_get              0x1000311d   Thumb Code    34  lis2dh12_reg.o(.text)
    lis2dh12_fifo_trigger_event_set          0x1000313f   Thumb Code    60  lis2dh12_reg.o(.text)
    lis2dh12_fifo_trigger_event_get          0x1000317b   Thumb Code    62  lis2dh12_reg.o(.text)
    lis2dh12_fifo_mode_set                   0x100031b9   Thumb Code    60  lis2dh12_reg.o(.text)
    lis2dh12_fifo_mode_get                   0x100031f5   Thumb Code    80  lis2dh12_reg.o(.text)
    lis2dh12_fifo_status_get                 0x10003245   Thumb Code    24  lis2dh12_reg.o(.text)
    lis2dh12_fifo_data_level_get             0x1000325d   Thumb Code    34  lis2dh12_reg.o(.text)
    lis2dh12_fifo_empty_flag_get             0x1000327f   Thumb Code    34  lis2dh12_reg.o(.text)
    lis2dh12_fifo_ovr_flag_get               0x100032a1   Thumb Code    34  lis2dh12_reg.o(.text)
    lis2dh12_fifo_fth_flag_get               0x100032c3   Thumb Code    32  lis2dh12_reg.o(.text)
    lis2dh12_tap_conf_set                    0x100032e3   Thumb Code    24  lis2dh12_reg.o(.text)
    lis2dh12_tap_conf_get                    0x100032fb   Thumb Code    24  lis2dh12_reg.o(.text)
    lis2dh12_tap_source_get                  0x10003313   Thumb Code    24  lis2dh12_reg.o(.text)
    lis2dh12_tap_threshold_set               0x1000332b   Thumb Code    58  lis2dh12_reg.o(.text)
    lis2dh12_tap_threshold_get               0x10003365   Thumb Code    34  lis2dh12_reg.o(.text)
    lis2dh12_tap_notification_mode_set       0x10003387   Thumb Code    60  lis2dh12_reg.o(.text)
    lis2dh12_tap_notification_mode_get       0x100033c3   Thumb Code    60  lis2dh12_reg.o(.text)
    lis2dh12_shock_dur_set                   0x100033ff   Thumb Code    58  lis2dh12_reg.o(.text)
    lis2dh12_shock_dur_get                   0x10003439   Thumb Code    34  lis2dh12_reg.o(.text)
    lis2dh12_quiet_dur_set                   0x1000345b   Thumb Code    46  lis2dh12_reg.o(.text)
    lis2dh12_quiet_dur_get                   0x10003489   Thumb Code    30  lis2dh12_reg.o(.text)
    lis2dh12_double_tap_timeout_set          0x100034a7   Thumb Code    46  lis2dh12_reg.o(.text)
    lis2dh12_double_tap_timeout_get          0x100034d5   Thumb Code    30  lis2dh12_reg.o(.text)
    lis2dh12_act_threshold_set               0x100034f3   Thumb Code    58  lis2dh12_reg.o(.text)
    lis2dh12_act_threshold_get               0x1000352d   Thumb Code    34  lis2dh12_reg.o(.text)
    lis2dh12_act_timeout_set                 0x1000354f   Thumb Code    46  lis2dh12_reg.o(.text)
    lis2dh12_act_timeout_get                 0x1000357d   Thumb Code    30  lis2dh12_reg.o(.text)
    lis2dh12_pin_sdo_sa0_mode_set            0x1000359b   Thumb Code    60  lis2dh12_reg.o(.text)
    lis2dh12_pin_sdo_sa0_mode_get            0x100035d7   Thumb Code    56  lis2dh12_reg.o(.text)
    lis2dh12_spi_mode_set                    0x1000360f   Thumb Code    58  lis2dh12_reg.o(.text)
    lis2dh12_spi_mode_get                    0x10003649   Thumb Code    62  lis2dh12_reg.o(.text)
    lsm6dso_read_reg                         0x10003689   Thumb Code    38  lsm6dso_reg.o(.text)
    lsm6dso_write_reg                        0x100036af   Thumb Code    38  lsm6dso_reg.o(.text)
    lsm6dso_from_fs2_to_mg                   0x100036e3   Thumb Code    20  lsm6dso_reg.o(.text)
    lsm6dso_from_fs4_to_mg                   0x100036f7   Thumb Code    20  lsm6dso_reg.o(.text)
    lsm6dso_from_fs8_to_mg                   0x1000370b   Thumb Code    20  lsm6dso_reg.o(.text)
    lsm6dso_from_fs16_to_mg                  0x1000371f   Thumb Code    20  lsm6dso_reg.o(.text)
    lsm6dso_from_fs125_to_mdps               0x10003733   Thumb Code    20  lsm6dso_reg.o(.text)
    lsm6dso_from_fs500_to_mdps               0x10003747   Thumb Code    20  lsm6dso_reg.o(.text)
    lsm6dso_from_fs250_to_mdps               0x1000375b   Thumb Code    20  lsm6dso_reg.o(.text)
    lsm6dso_from_fs1000_to_mdps              0x1000376f   Thumb Code    20  lsm6dso_reg.o(.text)
    lsm6dso_from_fs2000_to_mdps              0x10003783   Thumb Code    20  lsm6dso_reg.o(.text)
    lsm6dso_from_lsb_to_celsius              0x10003797   Thumb Code    30  lsm6dso_reg.o(.text)
    lsm6dso_from_lsb_to_nsec                 0x100037b5   Thumb Code    20  lsm6dso_reg.o(.text)
    lsm6dso_xl_full_scale_set                0x100037c9   Thumb Code    60  lsm6dso_reg.o(.text)
    lsm6dso_xl_full_scale_get                0x10003805   Thumb Code    82  lsm6dso_reg.o(.text)
    lsm6dso_mem_bank_set                     0x10003857   Thumb Code    46  lsm6dso_reg.o(.text)
    lsm6dso_fsm_data_rate_get                0x10003885   Thumb Code   118  lsm6dso_reg.o(.text)
    lsm6dso_fsm_enable_get                   0x100038fb   Thumb Code    44  lsm6dso_reg.o(.text)
    lsm6dso_xl_data_rate_set                 0x10003927   Thumb Code   374  lsm6dso_reg.o(.text)
    lsm6dso_xl_data_rate_get                 0x10003a9d   Thumb Code   174  lsm6dso_reg.o(.text)
    lsm6dso_gy_full_scale_set                0x10003b4b   Thumb Code    60  lsm6dso_reg.o(.text)
    lsm6dso_gy_full_scale_get                0x10003b87   Thumb Code    86  lsm6dso_reg.o(.text)
    lsm6dso_gy_data_rate_set                 0x10003bdd   Thumb Code   374  lsm6dso_reg.o(.text)
    lsm6dso_gy_data_rate_get                 0x10003d53   Thumb Code   124  lsm6dso_reg.o(.text)
    lsm6dso_block_data_update_set            0x10003dcf   Thumb Code    60  lsm6dso_reg.o(.text)
    lsm6dso_block_data_update_get            0x10003e0b   Thumb Code    34  lsm6dso_reg.o(.text)
    lsm6dso_xl_offset_weight_set             0x10003e2d   Thumb Code    60  lsm6dso_reg.o(.text)
    lsm6dso_xl_offset_weight_get             0x10003e69   Thumb Code    62  lsm6dso_reg.o(.text)
    lsm6dso_xl_power_mode_set                0x10003ea7   Thumb Code   132  lsm6dso_reg.o(.text)
    lsm6dso_xl_power_mode_get                0x10003f2b   Thumb Code    98  lsm6dso_reg.o(.text)
    lsm6dso_gy_power_mode_set                0x10003f8d   Thumb Code    60  lsm6dso_reg.o(.text)
    lsm6dso_gy_power_mode_get                0x10003fc9   Thumb Code    60  lsm6dso_reg.o(.text)
    lsm6dso_status_reg_get                   0x10004005   Thumb Code    24  lsm6dso_reg.o(.text)
    lsm6dso_xl_flag_data_ready_get           0x1000401d   Thumb Code    34  lsm6dso_reg.o(.text)
    lsm6dso_gy_flag_data_ready_get           0x1000403f   Thumb Code    34  lsm6dso_reg.o(.text)
    lsm6dso_temp_flag_data_ready_get         0x10004061   Thumb Code    34  lsm6dso_reg.o(.text)
    lsm6dso_xl_usr_offset_x_set              0x10004083   Thumb Code    24  lsm6dso_reg.o(.text)
    lsm6dso_xl_usr_offset_x_get              0x1000409b   Thumb Code    24  lsm6dso_reg.o(.text)
    lsm6dso_xl_usr_offset_y_set              0x100040b3   Thumb Code    24  lsm6dso_reg.o(.text)
    lsm6dso_xl_usr_offset_y_get              0x100040cb   Thumb Code    24  lsm6dso_reg.o(.text)
    lsm6dso_xl_usr_offset_z_set              0x100040e3   Thumb Code    24  lsm6dso_reg.o(.text)
    lsm6dso_xl_usr_offset_z_get              0x100040fb   Thumb Code    24  lsm6dso_reg.o(.text)
    lsm6dso_xl_usr_offset_set                0x10004113   Thumb Code    60  lsm6dso_reg.o(.text)
    lsm6dso_xl_usr_offset_get                0x1000414f   Thumb Code    34  lsm6dso_reg.o(.text)
    lsm6dso_timestamp_rst                    0x10004171   Thumb Code    22  lsm6dso_reg.o(.text)
    lsm6dso_timestamp_set                    0x10004187   Thumb Code    60  lsm6dso_reg.o(.text)
    lsm6dso_timestamp_get                    0x100041c3   Thumb Code    34  lsm6dso_reg.o(.text)
    lsm6dso_timestamp_raw_get                0x100041e5   Thumb Code    66  lsm6dso_reg.o(.text)
    lsm6dso_rounding_mode_set                0x10004227   Thumb Code    60  lsm6dso_reg.o(.text)
    lsm6dso_rounding_mode_get                0x10004263   Thumb Code    82  lsm6dso_reg.o(.text)
    lsm6dso_temperature_raw_get              0x100042b5   Thumb Code    44  lsm6dso_reg.o(.text)
    lsm6dso_angular_rate_raw_get             0x100042e1   Thumb Code    84  lsm6dso_reg.o(.text)
    lsm6dso_acceleration_raw_get             0x10004335   Thumb Code    84  lsm6dso_reg.o(.text)
    lsm6dso_fifo_out_raw_get                 0x10004389   Thumb Code    24  lsm6dso_reg.o(.text)
    lsm6dso_number_of_steps_get              0x100043a1   Thumb Code    78  lsm6dso_reg.o(.text)
    lsm6dso_steps_reset                      0x100043ef   Thumb Code    84  lsm6dso_reg.o(.text)
    lsm6dso_odr_cal_reg_set                  0x10004443   Thumb Code    46  lsm6dso_reg.o(.text)
    lsm6dso_odr_cal_reg_get                  0x10004471   Thumb Code    30  lsm6dso_reg.o(.text)
    lsm6dso_mem_bank_get                     0x1000448f   Thumb Code    70  lsm6dso_reg.o(.text)
    lsm6dso_ln_pg_write                      0x100044d5   Thumb Code   398  lsm6dso_reg.o(.text)
    lsm6dso_ln_pg_write_byte                 0x10004663   Thumb Code    22  lsm6dso_reg.o(.text)
    lsm6dso_ln_pg_read                       0x10004679   Thumb Code   398  lsm6dso_reg.o(.text)
    lsm6dso_ln_pg_read_byte                  0x10004807   Thumb Code    22  lsm6dso_reg.o(.text)
    lsm6dso_data_ready_mode_set              0x1000481d   Thumb Code    60  lsm6dso_reg.o(.text)
    lsm6dso_data_ready_mode_get              0x10004859   Thumb Code    60  lsm6dso_reg.o(.text)
    lsm6dso_device_id_get                    0x10004895   Thumb Code    24  lsm6dso_reg.o(.text)
    lsm6dso_reset_set                        0x100048ad   Thumb Code    58  lsm6dso_reg.o(.text)
    lsm6dso_reset_get                        0x100048e7   Thumb Code    34  lsm6dso_reg.o(.text)
    lsm6dso_auto_increment_set               0x10004909   Thumb Code    60  lsm6dso_reg.o(.text)
    lsm6dso_auto_increment_get               0x10004945   Thumb Code    34  lsm6dso_reg.o(.text)
    lsm6dso_boot_set                         0x10004967   Thumb Code    60  lsm6dso_reg.o(.text)
    lsm6dso_boot_get                         0x100049a3   Thumb Code    32  lsm6dso_reg.o(.text)
    lsm6dso_xl_self_test_set                 0x100049c3   Thumb Code    58  lsm6dso_reg.o(.text)
    lsm6dso_xl_self_test_get                 0x100049fd   Thumb Code    72  lsm6dso_reg.o(.text)
    lsm6dso_gy_self_test_set                 0x10004a45   Thumb Code    60  lsm6dso_reg.o(.text)
    lsm6dso_gy_self_test_get                 0x10004a81   Thumb Code    72  lsm6dso_reg.o(.text)
    lsm6dso_xl_filter_lp2_set                0x10004ac9   Thumb Code    60  lsm6dso_reg.o(.text)
    lsm6dso_xl_filter_lp2_get                0x10004b05   Thumb Code    34  lsm6dso_reg.o(.text)
    lsm6dso_gy_filter_lp1_set                0x10004b27   Thumb Code    60  lsm6dso_reg.o(.text)
    lsm6dso_gy_filter_lp1_get                0x10004b63   Thumb Code    34  lsm6dso_reg.o(.text)
    lsm6dso_filter_settling_mask_set         0x10004b85   Thumb Code    60  lsm6dso_reg.o(.text)
    lsm6dso_filter_settling_mask_get         0x10004bc1   Thumb Code    34  lsm6dso_reg.o(.text)
    lsm6dso_gy_lp1_bandwidth_set             0x10004be3   Thumb Code    58  lsm6dso_reg.o(.text)
    lsm6dso_gy_lp1_bandwidth_get             0x10004c1d   Thumb Code   104  lsm6dso_reg.o(.text)
    lsm6dso_xl_lp2_on_6d_set                 0x10004c85   Thumb Code    58  lsm6dso_reg.o(.text)
    lsm6dso_xl_lp2_on_6d_get                 0x10004cbf   Thumb Code    34  lsm6dso_reg.o(.text)
    lsm6dso_xl_hp_path_on_out_set            0x10004ce1   Thumb Code   108  lsm6dso_reg.o(.text)
    lsm6dso_xl_hp_path_on_out_get            0x10004d4d   Thumb Code   282  lsm6dso_reg.o(.text)
    lsm6dso_xl_fast_settling_set             0x10004e67   Thumb Code    60  lsm6dso_reg.o(.text)
    lsm6dso_xl_fast_settling_get             0x10004ea3   Thumb Code    34  lsm6dso_reg.o(.text)
    lsm6dso_xl_hp_path_internal_set          0x10004ec5   Thumb Code    60  lsm6dso_reg.o(.text)
    lsm6dso_xl_hp_path_internal_get          0x10004f01   Thumb Code    62  lsm6dso_reg.o(.text)
    lsm6dso_gy_hp_path_internal_set          0x10004f3f   Thumb Code    84  lsm6dso_reg.o(.text)
    lsm6dso_gy_hp_path_internal_get          0x10004f93   Thumb Code   108  lsm6dso_reg.o(.text)
    lsm6dso_aux_sdo_ocs_mode_set             0x10004fff   Thumb Code    60  lsm6dso_reg.o(.text)
    lsm6dso_aux_sdo_ocs_mode_get             0x1000503b   Thumb Code    60  lsm6dso_reg.o(.text)
    lsm6dso_aux_pw_on_ctrl_set               0x10005077   Thumb Code    76  lsm6dso_reg.o(.text)
    lsm6dso_aux_pw_on_ctrl_get               0x100050c3   Thumb Code    58  lsm6dso_reg.o(.text)
    lsm6dso_aux_xl_fs_mode_set               0x100050fd   Thumb Code    60  lsm6dso_reg.o(.text)
    lsm6dso_aux_xl_fs_mode_get               0x10005139   Thumb Code    62  lsm6dso_reg.o(.text)
    lsm6dso_aux_status_reg_get               0x10005177   Thumb Code    24  lsm6dso_reg.o(.text)
    lsm6dso_aux_xl_flag_data_ready_get       0x1000518f   Thumb Code    34  lsm6dso_reg.o(.text)
    lsm6dso_aux_gy_flag_data_ready_get       0x100051b1   Thumb Code    34  lsm6dso_reg.o(.text)
    lsm6dso_aux_gy_flag_settling_get         0x100051d3   Thumb Code    34  lsm6dso_reg.o(.text)
    lsm6dso_aux_xl_self_test_set             0x100051f5   Thumb Code    58  lsm6dso_reg.o(.text)
    lsm6dso_aux_xl_self_test_get             0x1000522f   Thumb Code    72  lsm6dso_reg.o(.text)
    lsm6dso_aux_den_polarity_set             0x10005277   Thumb Code    60  lsm6dso_reg.o(.text)
    lsm6dso_aux_den_polarity_get             0x100052b3   Thumb Code    62  lsm6dso_reg.o(.text)
    lsm6dso_aux_den_mode_set                 0x100052f1   Thumb Code   116  lsm6dso_reg.o(.text)
    lsm6dso_aux_den_mode_get                 0x10005365   Thumb Code   114  lsm6dso_reg.o(.text)
    lsm6dso_aux_drdy_on_int2_set             0x100053d7   Thumb Code    60  lsm6dso_reg.o(.text)
    lsm6dso_aux_drdy_on_int2_get             0x10005413   Thumb Code    32  lsm6dso_reg.o(.text)
    lsm6dso_aux_mode_set                     0x10005433   Thumb Code    82  lsm6dso_reg.o(.text)
    lsm6dso_aux_mode_get                     0x10005485   Thumb Code    82  lsm6dso_reg.o(.text)
    lsm6dso_aux_gy_full_scale_set            0x100054d7   Thumb Code    60  lsm6dso_reg.o(.text)
    lsm6dso_aux_gy_full_scale_get            0x10005513   Thumb Code    86  lsm6dso_reg.o(.text)
    lsm6dso_aux_spi_mode_set                 0x10005569   Thumb Code    60  lsm6dso_reg.o(.text)
    lsm6dso_aux_spi_mode_get                 0x100055a5   Thumb Code    62  lsm6dso_reg.o(.text)
    lsm6dso_aux_gy_lp1_bandwidth_set         0x100055e3   Thumb Code    60  lsm6dso_reg.o(.text)
    lsm6dso_aux_gy_lp1_bandwidth_get         0x1000561f   Thumb Code    82  lsm6dso_reg.o(.text)
    lsm6dso_aux_gy_hp_bandwidth_set          0x10005671   Thumb Code    78  lsm6dso_reg.o(.text)
    lsm6dso_aux_gy_hp_bandwidth_get          0x100056bf   Thumb Code   104  lsm6dso_reg.o(.text)
    lsm6dso_aux_gy_clamp_set                 0x10005727   Thumb Code    58  lsm6dso_reg.o(.text)
    lsm6dso_aux_gy_clamp_get                 0x10005761   Thumb Code    62  lsm6dso_reg.o(.text)
    lsm6dso_aux_gy_self_test_set             0x1000579f   Thumb Code    60  lsm6dso_reg.o(.text)
    lsm6dso_aux_gy_self_test_get             0x100057db   Thumb Code    72  lsm6dso_reg.o(.text)
    lsm6dso_aux_xl_bandwidth_set             0x10005823   Thumb Code    60  lsm6dso_reg.o(.text)
    lsm6dso_aux_xl_bandwidth_get             0x1000585f   Thumb Code   104  lsm6dso_reg.o(.text)
    lsm6dso_aux_xl_full_scale_set            0x100058c7   Thumb Code    60  lsm6dso_reg.o(.text)
    lsm6dso_aux_xl_full_scale_get            0x10005903   Thumb Code    80  lsm6dso_reg.o(.text)
    lsm6dso_sdo_sa0_mode_set                 0x10005953   Thumb Code    60  lsm6dso_reg.o(.text)
    lsm6dso_sdo_sa0_mode_get                 0x1000598f   Thumb Code    62  lsm6dso_reg.o(.text)
    lsm6dso_spi_mode_set                     0x100059cd   Thumb Code    60  lsm6dso_reg.o(.text)
    lsm6dso_spi_mode_get                     0x10005a09   Thumb Code    62  lsm6dso_reg.o(.text)
    lsm6dso_i2c_interface_set                0x10005a47   Thumb Code    60  lsm6dso_reg.o(.text)
    lsm6dso_i2c_interface_get                0x10005a83   Thumb Code    62  lsm6dso_reg.o(.text)
    lsm6dso_i3c_disable_set                  0x10005ac1   Thumb Code   116  lsm6dso_reg.o(.text)
    lsm6dso_i3c_disable_get                  0x10005b35   Thumb Code   124  lsm6dso_reg.o(.text)
    lsm6dso_int1_mode_set                    0x10005bb1   Thumb Code    58  lsm6dso_reg.o(.text)
    lsm6dso_int1_mode_get                    0x10005beb   Thumb Code    62  lsm6dso_reg.o(.text)
    lsm6dso_pin_mode_set                     0x10005c29   Thumb Code    60  lsm6dso_reg.o(.text)
    lsm6dso_pin_mode_get                     0x10005c65   Thumb Code    62  lsm6dso_reg.o(.text)
    lsm6dso_pin_polarity_set                 0x10005ca3   Thumb Code    60  lsm6dso_reg.o(.text)
    lsm6dso_pin_polarity_get                 0x10005cdf   Thumb Code    62  lsm6dso_reg.o(.text)
    lsm6dso_all_on_int1_set                  0x10005d1d   Thumb Code    60  lsm6dso_reg.o(.text)
    lsm6dso_all_on_int1_get                  0x10005d59   Thumb Code    34  lsm6dso_reg.o(.text)
    lsm6dso_int_notification_set             0x10005d7b   Thumb Code   160  lsm6dso_reg.o(.text)
    lsm6dso_int_notification_get             0x10005e1b   Thumb Code   154  lsm6dso_reg.o(.text)
    lsm6dso_wkup_ths_weight_set              0x10005eb5   Thumb Code    60  lsm6dso_reg.o(.text)
    lsm6dso_wkup_ths_weight_get              0x10005ef1   Thumb Code    62  lsm6dso_reg.o(.text)
    lsm6dso_wkup_threshold_set               0x10005f2f   Thumb Code    58  lsm6dso_reg.o(.text)
    lsm6dso_wkup_threshold_get               0x10005f69   Thumb Code    34  lsm6dso_reg.o(.text)
    lsm6dso_xl_usr_offset_on_wkup_set        0x10005f8b   Thumb Code    60  lsm6dso_reg.o(.text)
    lsm6dso_xl_usr_offset_on_wkup_get        0x10005fc7   Thumb Code    34  lsm6dso_reg.o(.text)
    lsm6dso_wkup_dur_set                     0x10005fe9   Thumb Code    60  lsm6dso_reg.o(.text)
    lsm6dso_wkup_dur_get                     0x10006025   Thumb Code    34  lsm6dso_reg.o(.text)
    lsm6dso_gy_sleep_mode_set                0x10006047   Thumb Code    60  lsm6dso_reg.o(.text)
    lsm6dso_gy_sleep_mode_get                0x10006083   Thumb Code    34  lsm6dso_reg.o(.text)
    lsm6dso_act_pin_notification_set         0x100060a5   Thumb Code    60  lsm6dso_reg.o(.text)
    lsm6dso_act_pin_notification_get         0x100060e1   Thumb Code    62  lsm6dso_reg.o(.text)
    lsm6dso_act_mode_set                     0x1000611f   Thumb Code    60  lsm6dso_reg.o(.text)
    lsm6dso_act_mode_get                     0x1000615b   Thumb Code    82  lsm6dso_reg.o(.text)
    lsm6dso_act_sleep_dur_set                0x100061ad   Thumb Code    58  lsm6dso_reg.o(.text)
    lsm6dso_act_sleep_dur_get                0x100061e7   Thumb Code    34  lsm6dso_reg.o(.text)
    lsm6dso_tap_detection_on_z_set           0x10006209   Thumb Code    60  lsm6dso_reg.o(.text)
    lsm6dso_tap_detection_on_z_get           0x10006245   Thumb Code    34  lsm6dso_reg.o(.text)
    lsm6dso_tap_detection_on_y_set           0x10006267   Thumb Code    60  lsm6dso_reg.o(.text)
    lsm6dso_tap_detection_on_y_get           0x100062a3   Thumb Code    34  lsm6dso_reg.o(.text)
    lsm6dso_tap_detection_on_x_set           0x100062c5   Thumb Code    60  lsm6dso_reg.o(.text)
    lsm6dso_tap_detection_on_x_get           0x10006301   Thumb Code    34  lsm6dso_reg.o(.text)
    lsm6dso_tap_threshold_x_set              0x10006323   Thumb Code    58  lsm6dso_reg.o(.text)
    lsm6dso_tap_threshold_x_get              0x1000635d   Thumb Code    34  lsm6dso_reg.o(.text)
    lsm6dso_tap_axis_priority_set            0x1000637f   Thumb Code    60  lsm6dso_reg.o(.text)
    lsm6dso_tap_axis_priority_get            0x100063bb   Thumb Code    90  lsm6dso_reg.o(.text)
    lsm6dso_tap_threshold_y_set              0x10006415   Thumb Code    58  lsm6dso_reg.o(.text)
    lsm6dso_tap_threshold_y_get              0x1000644f   Thumb Code    34  lsm6dso_reg.o(.text)
    lsm6dso_tap_threshold_z_set              0x10006471   Thumb Code    58  lsm6dso_reg.o(.text)
    lsm6dso_tap_threshold_z_get              0x100064ab   Thumb Code    34  lsm6dso_reg.o(.text)
    lsm6dso_tap_shock_set                    0x100064cd   Thumb Code    58  lsm6dso_reg.o(.text)
    lsm6dso_tap_shock_get                    0x10006507   Thumb Code    34  lsm6dso_reg.o(.text)
    lsm6dso_tap_quiet_set                    0x10006529   Thumb Code    60  lsm6dso_reg.o(.text)
    lsm6dso_tap_quiet_get                    0x10006565   Thumb Code    34  lsm6dso_reg.o(.text)
    lsm6dso_tap_dur_set                      0x10006587   Thumb Code    60  lsm6dso_reg.o(.text)
    lsm6dso_tap_dur_get                      0x100065c3   Thumb Code    32  lsm6dso_reg.o(.text)
    lsm6dso_tap_mode_set                     0x100065e3   Thumb Code    60  lsm6dso_reg.o(.text)
    lsm6dso_tap_mode_get                     0x1000661f   Thumb Code    60  lsm6dso_reg.o(.text)
    lsm6dso_6d_threshold_set                 0x1000665b   Thumb Code    60  lsm6dso_reg.o(.text)
    lsm6dso_6d_threshold_get                 0x10006697   Thumb Code    82  lsm6dso_reg.o(.text)
    lsm6dso_4d_mode_set                      0x100066e9   Thumb Code    60  lsm6dso_reg.o(.text)
    lsm6dso_4d_mode_get                      0x10006725   Thumb Code    32  lsm6dso_reg.o(.text)
    lsm6dso_ff_threshold_set                 0x10006745   Thumb Code    58  lsm6dso_reg.o(.text)
    lsm6dso_ff_threshold_get                 0x1000677f   Thumb Code   104  lsm6dso_reg.o(.text)
    lsm6dso_ff_dur_set                       0x100067e7   Thumb Code   116  lsm6dso_reg.o(.text)
    lsm6dso_ff_dur_get                       0x1000685b   Thumb Code    60  lsm6dso_reg.o(.text)
    lsm6dso_fifo_watermark_set               0x10006897   Thumb Code    84  lsm6dso_reg.o(.text)
    lsm6dso_fifo_watermark_get               0x100068eb   Thumb Code    58  lsm6dso_reg.o(.text)
    lsm6dso_compression_algo_init_set        0x10006925   Thumb Code    84  lsm6dso_reg.o(.text)
    lsm6dso_compression_algo_init_get        0x10006979   Thumb Code    54  lsm6dso_reg.o(.text)
    lsm6dso_compression_algo_set             0x100069af   Thumb Code    84  lsm6dso_reg.o(.text)
    lsm6dso_compression_algo_get             0x10006a03   Thumb Code    96  lsm6dso_reg.o(.text)
    lsm6dso_fifo_virtual_sens_odr_chg_set    0x10006a63   Thumb Code    60  lsm6dso_reg.o(.text)
    lsm6dso_fifo_virtual_sens_odr_chg_get    0x10006a9f   Thumb Code    34  lsm6dso_reg.o(.text)
    lsm6dso_compression_algo_real_time_set   0x10006ac1   Thumb Code    60  lsm6dso_reg.o(.text)
    lsm6dso_compression_algo_real_time_get   0x10006afd   Thumb Code    34  lsm6dso_reg.o(.text)
    lsm6dso_fifo_stop_on_wtm_set             0x10006b1f   Thumb Code    60  lsm6dso_reg.o(.text)
    lsm6dso_fifo_stop_on_wtm_get             0x10006b5b   Thumb Code    32  lsm6dso_reg.o(.text)
    lsm6dso_fifo_xl_batch_set                0x10006b7b   Thumb Code    58  lsm6dso_reg.o(.text)
    lsm6dso_fifo_xl_batch_get                0x10006bb5   Thumb Code   132  lsm6dso_reg.o(.text)
    lsm6dso_fifo_gy_batch_set                0x10006c39   Thumb Code    60  lsm6dso_reg.o(.text)
    lsm6dso_fifo_gy_batch_get                0x10006c75   Thumb Code   130  lsm6dso_reg.o(.text)
    lsm6dso_fifo_mode_set                    0x10006cf7   Thumb Code    58  lsm6dso_reg.o(.text)
    lsm6dso_fifo_mode_get                    0x10006d31   Thumb Code    92  lsm6dso_reg.o(.text)
    lsm6dso_fifo_temp_batch_set              0x10006d8d   Thumb Code    60  lsm6dso_reg.o(.text)
    lsm6dso_fifo_temp_batch_get              0x10006dc9   Thumb Code    82  lsm6dso_reg.o(.text)
    lsm6dso_fifo_timestamp_decimation_set    0x10006e1b   Thumb Code    60  lsm6dso_reg.o(.text)
    lsm6dso_fifo_timestamp_decimation_get    0x10006e57   Thumb Code    80  lsm6dso_reg.o(.text)
    lsm6dso_fifo_cnt_event_batch_set         0x10006ea7   Thumb Code    60  lsm6dso_reg.o(.text)
    lsm6dso_fifo_cnt_event_batch_get         0x10006ee3   Thumb Code    62  lsm6dso_reg.o(.text)
    lsm6dso_rst_batch_counter_set            0x10006f21   Thumb Code    60  lsm6dso_reg.o(.text)
    lsm6dso_rst_batch_counter_get            0x10006f5d   Thumb Code    34  lsm6dso_reg.o(.text)
    lsm6dso_batch_counter_threshold_set      0x10006f7f   Thumb Code    86  lsm6dso_reg.o(.text)
    lsm6dso_batch_counter_threshold_get      0x10006fd5   Thumb Code    58  lsm6dso_reg.o(.text)
    lsm6dso_fifo_data_level_get              0x1000700f   Thumb Code    50  lsm6dso_reg.o(.text)
    lsm6dso_fifo_status_get                  0x10007041   Thumb Code    36  lsm6dso_reg.o(.text)
    lsm6dso_fifo_full_flag_get               0x10007065   Thumb Code    40  lsm6dso_reg.o(.text)
    lsm6dso_fifo_ovr_flag_get                0x1000708d   Thumb Code    40  lsm6dso_reg.o(.text)
    lsm6dso_fifo_wtm_flag_get                0x100070b5   Thumb Code    38  lsm6dso_reg.o(.text)
    lsm6dso_fifo_sensor_tag_get              0x100070db   Thumb Code   204  lsm6dso_reg.o(.text)
    lsm6dso_fifo_pedo_batch_set              0x100071a7   Thumb Code    84  lsm6dso_reg.o(.text)
    lsm6dso_fifo_pedo_batch_get              0x100071fb   Thumb Code    62  lsm6dso_reg.o(.text)
    lsm6dso_sh_batch_slave_set               0x10007239   Thumb Code    98  lsm6dso_reg.o(.text)
    lsm6dso_sh_batch_slave_get               0x1000729b   Thumb Code    70  lsm6dso_reg.o(.text)
    lsm6dso_den_mode_set                     0x100072e1   Thumb Code    60  lsm6dso_reg.o(.text)
    lsm6dso_den_mode_get                     0x1000731d   Thumb Code    84  lsm6dso_reg.o(.text)
    lsm6dso_den_polarity_set                 0x10007371   Thumb Code    60  lsm6dso_reg.o(.text)
    lsm6dso_den_polarity_get                 0x100073ad   Thumb Code    62  lsm6dso_reg.o(.text)
    lsm6dso_den_enable_set                   0x100073eb   Thumb Code    60  lsm6dso_reg.o(.text)
    lsm6dso_den_enable_get                   0x10007427   Thumb Code    72  lsm6dso_reg.o(.text)
    lsm6dso_den_mark_axis_x_set              0x1000746f   Thumb Code    60  lsm6dso_reg.o(.text)
    lsm6dso_den_mark_axis_x_get              0x100074ab   Thumb Code    34  lsm6dso_reg.o(.text)
    lsm6dso_den_mark_axis_y_set              0x100074cd   Thumb Code    60  lsm6dso_reg.o(.text)
    lsm6dso_den_mark_axis_y_get              0x10007509   Thumb Code    34  lsm6dso_reg.o(.text)
    lsm6dso_den_mark_axis_z_set              0x1000752b   Thumb Code    60  lsm6dso_reg.o(.text)
    lsm6dso_den_mark_axis_z_get              0x10007567   Thumb Code    32  lsm6dso_reg.o(.text)
    lsm6dso_pedo_sens_set                    0x10007587   Thumb Code    84  lsm6dso_reg.o(.text)
    lsm6dso_pedo_sens_get                    0x100075db   Thumb Code    82  lsm6dso_reg.o(.text)
    lsm6dso_pedo_step_detect_get             0x1000762d   Thumb Code    62  lsm6dso_reg.o(.text)
    lsm6dso_pedo_debounce_steps_set          0x1000766b   Thumb Code    24  lsm6dso_reg.o(.text)
    lsm6dso_pedo_debounce_steps_get          0x10007683   Thumb Code    24  lsm6dso_reg.o(.text)
    lsm6dso_pedo_steps_period_set            0x1000769b   Thumb Code    60  lsm6dso_reg.o(.text)
    lsm6dso_pedo_steps_period_get            0x100076d7   Thumb Code    58  lsm6dso_reg.o(.text)
    lsm6dso_pedo_int_mode_set                0x10007711   Thumb Code    60  lsm6dso_reg.o(.text)
    lsm6dso_pedo_int_mode_get                0x1000774d   Thumb Code    62  lsm6dso_reg.o(.text)
    lsm6dso_motion_flag_data_ready_get       0x1000778b   Thumb Code    62  lsm6dso_reg.o(.text)
    lsm6dso_tilt_flag_data_ready_get         0x100077c9   Thumb Code    62  lsm6dso_reg.o(.text)
    lsm6dso_mag_sensitivity_set              0x10007807   Thumb Code    56  lsm6dso_reg.o(.text)
    lsm6dso_mag_sensitivity_get              0x1000783f   Thumb Code    54  lsm6dso_reg.o(.text)
    lsm6dso_mag_offset_set                   0x10007875   Thumb Code    92  lsm6dso_reg.o(.text)
    lsm6dso_mag_offset_get                   0x100078d1   Thumb Code    84  lsm6dso_reg.o(.text)
    lsm6dso_mag_soft_iron_set                0x10007925   Thumb Code   164  lsm6dso_reg.o(.text)
    lsm6dso_mag_soft_iron_get                0x100079c9   Thumb Code   144  lsm6dso_reg.o(.text)
    lsm6dso_mag_z_orient_set                 0x10007a59   Thumb Code    54  lsm6dso_reg.o(.text)
    lsm6dso_mag_z_orient_get                 0x10007a8f   Thumb Code    88  lsm6dso_reg.o(.text)
    lsm6dso_mag_y_orient_set                 0x10007ae7   Thumb Code    56  lsm6dso_reg.o(.text)
    lsm6dso_mag_y_orient_get                 0x10007b1f   Thumb Code    88  lsm6dso_reg.o(.text)
    lsm6dso_mag_x_orient_set                 0x10007b77   Thumb Code    54  lsm6dso_reg.o(.text)
    lsm6dso_mag_x_orient_get                 0x10007bad   Thumb Code    88  lsm6dso_reg.o(.text)
    lsm6dso_long_cnt_flag_data_ready_get     0x10007c05   Thumb Code    60  lsm6dso_reg.o(.text)
    lsm6dso_fsm_enable_set                   0x10007c41   Thumb Code    66  lsm6dso_reg.o(.text)
    lsm6dso_long_cnt_set                     0x10007c83   Thumb Code    64  lsm6dso_reg.o(.text)
    lsm6dso_long_cnt_get                     0x10007cc3   Thumb Code    62  lsm6dso_reg.o(.text)
    lsm6dso_long_clr_set                     0x10007d01   Thumb Code    82  lsm6dso_reg.o(.text)
    lsm6dso_long_clr_get                     0x10007d53   Thumb Code   108  lsm6dso_reg.o(.text)
    lsm6dso_fsm_out_get                      0x10007dbf   Thumb Code    44  lsm6dso_reg.o(.text)
    lsm6dso_fsm_data_rate_set                0x10007deb   Thumb Code   118  lsm6dso_reg.o(.text)
    lsm6dso_fsm_init_set                     0x10007e61   Thumb Code    90  lsm6dso_reg.o(.text)
    lsm6dso_fsm_init_get                     0x10007ebb   Thumb Code    62  lsm6dso_reg.o(.text)
    lsm6dso_long_cnt_int_value_set           0x10007ef9   Thumb Code    60  lsm6dso_reg.o(.text)
    lsm6dso_long_cnt_int_value_get           0x10007f35   Thumb Code    58  lsm6dso_reg.o(.text)
    lsm6dso_fsm_number_of_programs_set       0x10007f6f   Thumb Code    22  lsm6dso_reg.o(.text)
    lsm6dso_fsm_number_of_programs_get       0x10007f85   Thumb Code    24  lsm6dso_reg.o(.text)
    lsm6dso_fsm_start_address_set            0x10007f9d   Thumb Code    60  lsm6dso_reg.o(.text)
    lsm6dso_fsm_start_address_get            0x10007fd9   Thumb Code    58  lsm6dso_reg.o(.text)
    lsm6dso_sh_read_data_raw_get             0x10008013   Thumb Code    46  lsm6dso_reg.o(.text)
    lsm6dso_sh_slave_connected_set           0x10008041   Thumb Code    82  lsm6dso_reg.o(.text)
    lsm6dso_sh_slave_connected_get           0x10008093   Thumb Code   110  lsm6dso_reg.o(.text)
    lsm6dso_sh_master_set                    0x10008101   Thumb Code    84  lsm6dso_reg.o(.text)
    lsm6dso_sh_master_get                    0x10008155   Thumb Code    62  lsm6dso_reg.o(.text)
    lsm6dso_sh_pin_mode_set                  0x10008193   Thumb Code    84  lsm6dso_reg.o(.text)
    lsm6dso_sh_pin_mode_get                  0x100081e7   Thumb Code    90  lsm6dso_reg.o(.text)
    lsm6dso_sh_pass_through_set              0x10008241   Thumb Code    84  lsm6dso_reg.o(.text)
    lsm6dso_sh_pass_through_get              0x10008295   Thumb Code    62  lsm6dso_reg.o(.text)
    lsm6dso_sh_syncro_mode_set               0x100082d3   Thumb Code    84  lsm6dso_reg.o(.text)
    lsm6dso_sh_syncro_mode_get               0x10008327   Thumb Code    86  lsm6dso_reg.o(.text)
    lsm6dso_sh_write_mode_set                0x1000837d   Thumb Code    84  lsm6dso_reg.o(.text)
    lsm6dso_sh_write_mode_get                0x100083d1   Thumb Code    90  lsm6dso_reg.o(.text)
    lsm6dso_sh_reset_set                     0x1000842b   Thumb Code   108  lsm6dso_reg.o(.text)
    lsm6dso_sh_reset_get                     0x10008497   Thumb Code    60  lsm6dso_reg.o(.text)
    lsm6dso_sh_data_rate_set                 0x100084d3   Thumb Code    84  lsm6dso_reg.o(.text)
    lsm6dso_sh_data_rate_get                 0x10008527   Thumb Code   108  lsm6dso_reg.o(.text)
    lsm6dso_sh_cfg_write                     0x10008593   Thumb Code   124  lsm6dso_reg.o(.text)
    lsm6dso_sh_slv_cfg_read                  0x1000860f   Thumb Code   184  lsm6dso_reg.o(.text)
    lsm6dso_sh_status_get                    0x100086c7   Thumb Code    24  lsm6dso_reg.o(.text)
    lsm6dso_id_get                           0x100086df   Thumb Code    50  lsm6dso_reg.o(.text)
    lsm6dso_init_set                         0x10008711   Thumb Code   354  lsm6dso_reg.o(.text)
    lsm6dso_bus_mode_set                     0x10008873   Thumb Code   402  lsm6dso_reg.o(.text)
    lsm6dso_bus_mode_get                     0x10008a05   Thumb Code   288  lsm6dso_reg.o(.text)
    lsm6dso_status_get                       0x10008b25   Thumb Code   268  lsm6dso_reg.o(.text)
    lsm6dso_pin_conf_set                     0x10008c31   Thumb Code   214  lsm6dso_reg.o(.text)
    lsm6dso_pin_conf_get                     0x10008d07   Thumb Code   162  lsm6dso_reg.o(.text)
    lsm6dso_interrupt_mode_set               0x10008da9   Thumb Code   244  lsm6dso_reg.o(.text)
    lsm6dso_interrupt_mode_get               0x10008e9d   Thumb Code   170  lsm6dso_reg.o(.text)
    lsm6dso_pin_int2_route_get               0x10008f47   Thumb Code  1060  lsm6dso_reg.o(.text)
    lsm6dso_pin_int1_route_set               0x1000936b   Thumb Code  1798  lsm6dso_reg.o(.text)
    lsm6dso_pin_int1_route_get               0x10009a71   Thumb Code  1064  lsm6dso_reg.o(.text)
    lsm6dso_pin_int2_route_set               0x10009e99   Thumb Code  1686  lsm6dso_reg.o(.text)
    lsm6dso_all_sources_get                  0x1000a52f   Thumb Code  1482  lsm6dso_reg.o(.text)
    lsm6dso_mode_set                         0x1000aaf9   Thumb Code  1552  lsm6dso_reg.o(.text)
    lsm6dso_mode_get                         0x1000b109   Thumb Code  1514  lsm6dso_reg.o(.text)
    lsm6dso_data_get                         0x1000b6f3   Thumb Code   844  lsm6dso_reg.o(.text)
    lsm6dso_embedded_sens_set                0x1000ba3f   Thumb Code   236  lsm6dso_reg.o(.text)
    lsm6dso_embedded_sens_get                0x1000bb2b   Thumb Code   200  lsm6dso_reg.o(.text)
    lsm6dso_embedded_sens_off                0x1000bbf3   Thumb Code   160  lsm6dso_reg.o(.text)
    cJSON_GetErrorPtr                        0x1000bc95   Thumb Code    12  cjson.o(.text)
    cJSON_IsString                           0x1000bca1   Thumb Code    22  cjson.o(.text)
    cJSON_GetStringValue                     0x1000bcb7   Thumb Code    20  cjson.o(.text)
    cJSON_IsNumber                           0x1000bccb   Thumb Code    22  cjson.o(.text)
    cJSON_GetNumberValue                     0x1000bce1   Thumb Code    24  cjson.o(.text)
    cJSON_Version                            0x1000bcf9   Thumb Code    22  cjson.o(.text)
    cJSON_InitHooks                          0x1000bd8f   Thumb Code    88  cjson.o(.text)
    cJSON_Delete                             0x1000be03   Thumb Code   102  cjson.o(.text)
    cJSON_SetNumberHelper                    0x1000bf97   Thumb Code    70  cjson.o(.text)
    cJSON_free                               0x1000bfdd   Thumb Code    14  cjson.o(.text)
    cJSON_SetValuestring                     0x1000bfeb   Thumb Code    96  cjson.o(.text)
    cJSON_ParseWithLengthOpts                0x1000cc13   Thumb Code   218  cjson.o(.text)
    cJSON_ParseWithOpts                      0x1000cced   Thumb Code    36  cjson.o(.text)
    cJSON_Parse                              0x1000cd11   Thumb Code    16  cjson.o(.text)
    cJSON_ParseWithLength                    0x1000cd21   Thumb Code    20  cjson.o(.text)
    cJSON_Print                              0x1000d143   Thumb Code    16  cjson.o(.text)
    cJSON_PrintUnformatted                   0x1000d153   Thumb Code    16  cjson.o(.text)
    cJSON_PrintBuffered                      0x1000d163   Thumb Code    92  cjson.o(.text)
    cJSON_PrintPreallocated                  0x1000d1bf   Thumb Code    66  cjson.o(.text)
    cJSON_GetArraySize                       0x1000d201   Thumb Code    28  cjson.o(.text)
    cJSON_GetArrayItem                       0x1000d23d   Thumb Code    24  cjson.o(.text)
    cJSON_GetObjectItem                      0x1000d2b3   Thumb Code    18  cjson.o(.text)
    cJSON_GetObjectItemCaseSensitive         0x1000d2c5   Thumb Code    18  cjson.o(.text)
    cJSON_HasObjectItem                      0x1000d2d7   Thumb Code    26  cjson.o(.text)
    cJSON_AddItemToArray                     0x1000d373   Thumb Code    16  cjson.o(.text)
    cJSON_AddItemToObject                    0x1000d417   Thumb Code    26  cjson.o(.text)
    cJSON_AddItemToObjectCS                  0x1000d431   Thumb Code    26  cjson.o(.text)
    cJSON_AddItemReferenceToArray            0x1000d44b   Thumb Code    32  cjson.o(.text)
    cJSON_AddItemReferenceToObject           0x1000d46b   Thumb Code    48  cjson.o(.text)
    cJSON_CreateNull                         0x1000d49b   Thumb Code    22  cjson.o(.text)
    cJSON_AddNullToObject                    0x1000d4b1   Thumb Code    46  cjson.o(.text)
    cJSON_CreateTrue                         0x1000d4df   Thumb Code    22  cjson.o(.text)
    cJSON_AddTrueToObject                    0x1000d4f5   Thumb Code    46  cjson.o(.text)
    cJSON_CreateFalse                        0x1000d523   Thumb Code    22  cjson.o(.text)
    cJSON_AddFalseToObject                   0x1000d539   Thumb Code    46  cjson.o(.text)
    cJSON_CreateBool                         0x1000d567   Thumb Code    32  cjson.o(.text)
    cJSON_AddBoolToObject                    0x1000d587   Thumb Code    50  cjson.o(.text)
    cJSON_CreateNumber                       0x1000d5b9   Thumb Code    82  cjson.o(.text)
    cJSON_AddNumberToObject                  0x1000d60b   Thumb Code    54  cjson.o(.text)
    cJSON_CreateString                       0x1000d641   Thumb Code    50  cjson.o(.text)
    cJSON_AddStringToObject                  0x1000d673   Thumb Code    50  cjson.o(.text)
    cJSON_CreateRaw                          0x1000d6a5   Thumb Code    50  cjson.o(.text)
    cJSON_AddRawToObject                     0x1000d6d7   Thumb Code    50  cjson.o(.text)
    cJSON_CreateObject                       0x1000d709   Thumb Code    22  cjson.o(.text)
    cJSON_AddObjectToObject                  0x1000d71f   Thumb Code    46  cjson.o(.text)
    cJSON_CreateArray                        0x1000d74d   Thumb Code    22  cjson.o(.text)
    cJSON_AddArrayToObject                   0x1000d763   Thumb Code    46  cjson.o(.text)
    cJSON_DetachItemViaPointer               0x1000d791   Thumb Code    72  cjson.o(.text)
    cJSON_DetachItemFromArray                0x1000d7d9   Thumb Code    34  cjson.o(.text)
    cJSON_DeleteItemFromArray                0x1000d7fb   Thumb Code    42  cjson.o(.text)
    cJSON_DetachItemFromObject               0x1000d825   Thumb Code    26  cjson.o(.text)
    cJSON_DetachItemFromObjectCaseSensitive  0x1000d83f   Thumb Code    26  cjson.o(.text)
    cJSON_DeleteItemFromObject               0x1000d859   Thumb Code    22  cjson.o(.text)
    cJSON_DeleteItemFromObjectCaseSensitive  0x1000d86f   Thumb Code    22  cjson.o(.text)
    cJSON_InsertItemInArray                  0x1000d885   Thumb Code    68  cjson.o(.text)
    cJSON_ReplaceItemViaPointer              0x1000d8c9   Thumb Code   108  cjson.o(.text)
    cJSON_ReplaceItemInArray                 0x1000d935   Thumb Code    38  cjson.o(.text)
    cJSON_ReplaceItemInObject                0x1000d9b5   Thumb Code    22  cjson.o(.text)
    cJSON_ReplaceItemInObjectCaseSensitive   0x1000d9cb   Thumb Code    22  cjson.o(.text)
    cJSON_CreateStringReference              0x1000d9e1   Thumb Code    34  cjson.o(.text)
    cJSON_CreateObjectReference              0x1000da03   Thumb Code    34  cjson.o(.text)
    cJSON_CreateArrayReference               0x1000da25   Thumb Code    34  cjson.o(.text)
    cJSON_CreateIntArray                     0x1000da47   Thumb Code   122  cjson.o(.text)
    cJSON_CreateFloatArray                   0x1000dac1   Thumb Code   122  cjson.o(.text)
    cJSON_CreateDoubleArray                  0x1000db3b   Thumb Code   118  cjson.o(.text)
    cJSON_CreateStringArray                  0x1000dbb1   Thumb Code   112  cjson.o(.text)
    cJSON_Duplicate                          0x1000dc21   Thumb Code   212  cjson.o(.text)
    cJSON_Minify                             0x1000ddcb   Thumb Code   156  cjson.o(.text)
    cJSON_IsInvalid                          0x1000de67   Thumb Code    22  cjson.o(.text)
    cJSON_IsFalse                            0x1000de7d   Thumb Code    20  cjson.o(.text)
    cJSON_IsTrue                             0x1000de91   Thumb Code    22  cjson.o(.text)
    cJSON_IsBool                             0x1000dea7   Thumb Code    26  cjson.o(.text)
    cJSON_IsNull                             0x1000dec1   Thumb Code    22  cjson.o(.text)
    cJSON_IsArray                            0x1000ded7   Thumb Code    22  cjson.o(.text)
    cJSON_IsObject                           0x1000deed   Thumb Code    22  cjson.o(.text)
    cJSON_IsRaw                              0x1000df03   Thumb Code    22  cjson.o(.text)
    cJSON_Compare                            0x1000df19   Thumb Code   394  cjson.o(.text)
    cJSON_malloc                             0x1000e0a3   Thumb Code    14  cjson.o(.text)
    crc16_compute                            0x1000e0b5   Thumb Code    64  crc16.o(.text)
    crc16_modbus                             0x1000e0f5   Thumb Code    52  crc16.o(.text)
    crc16_ccitt                              0x1000e129   Thumb Code    40  crc16.o(.text)
    stringLength                             0x1000e15d   Thumb Code    18  common.o(.text)
    str_cmp                                  0x1000e16f   Thumb Code    34  common.o(.text)
    BLE_SendRPPData                          0x1000e267   Thumb Code    56  main.o(.text)
    Charge_State_Judge                       0x1000e395   Thumb Code    32  main.o(.text)
    LED_State_Indicator                      0x1000e3b5   Thumb Code    72  main.o(.text)
    BLSetConnectionUpdate                    0x1000e49f   Thumb Code    92  main.o(.text)
    Connection_latency                       0x1000e4fb   Thumb Code    40  main.o(.text)
    ota_manage                               0x1000e523   Thumb Code   316  main.o(.text)
    gpio_init                                0x1000e6d5   Thumb Code   242  main.o(.text)
    nvic_priority                            0x1000e7c7   Thumb Code   188  main.o(.text)
    BLE_SendCMDData                          0x1000e9f9   Thumb Code   176  main.o(.text)
    ble_evt_callback                         0x1000eba5   Thumb Code  1268  main.o(.text)
    main                                     0x1000f11d   Thumb Code   174  main.o(.text)
    BLE_NotifyBatteryLevel                   0x1000f1cb   Thumb Code    38  main.o(.text)
    syd_nosleep                              0x1000f1f1   Thumb Code    56  main.o(.text)
    cal_battery_value                        0x1000f229   Thumb Code   346  main.o(.text)
    get_battery_value                        0x1000f383   Thumb Code    38  main.o(.text)
    rtc_event_handler                        0x1000f3a9   Thumb Code    42  main.o(.text)
    JsProtocol_Report                        0x1000f3d3   Thumb Code   666  main.o(.text)
    pack_timer_event                         0x1000f66d   Thumb Code    46  main.o(.text)
    BSP_MCU_Config                           0x1000f6d9   Thumb Code    12  mcu_bsp.o(.text)
    Timer_2_callback                         0x1000f6ed   Thumb Code    20  isr.o(.text)
    GPIO_callback                            0x1000f701   Thumb Code    64  isr.o(.text)
    SEGGER_RTT_ReadNoLock                    0x1000f893   Thumb Code   168  segger_rtt.o(.text)
    SEGGER_RTT_Read                          0x1000f93b   Thumb Code    50  segger_rtt.o(.text)
    SEGGER_RTT_WriteWithOverwriteNoLock      0x1000f96d   Thumb Code   170  segger_rtt.o(.text)
    SEGGER_RTT_WriteSkipNoLock               0x1000fa17   Thumb Code   178  segger_rtt.o(.text)
    SEGGER_RTT_WriteNoLock                   0x1000fac9   Thumb Code   170  segger_rtt.o(.text)
    SEGGER_RTT_Write                         0x1000fb73   Thumb Code    66  segger_rtt.o(.text)
    SEGGER_RTT_WriteString                   0x1000fbb5   Thumb Code    26  segger_rtt.o(.text)
    SEGGER_RTT_PutCharSkipNoLock             0x1000fbcf   Thumb Code    50  segger_rtt.o(.text)
    SEGGER_RTT_PutCharSkip                   0x1000fc01   Thumb Code    94  segger_rtt.o(.text)
    SEGGER_RTT_PutChar                       0x1000fc5f   Thumb Code   108  segger_rtt.o(.text)
    SEGGER_RTT_GetKey                        0x1000fccb   Thumb Code    32  segger_rtt.o(.text)
    SEGGER_RTT_WaitKey                       0x1000fceb   Thumb Code    14  segger_rtt.o(.text)
    SEGGER_RTT_HasKey                        0x1000fcf9   Thumb Code    38  segger_rtt.o(.text)
    SEGGER_RTT_HasData                       0x1000fd1f   Thumb Code    22  segger_rtt.o(.text)
    SEGGER_RTT_AllocDownBuffer               0x1000fd35   Thumb Code   164  segger_rtt.o(.text)
    SEGGER_RTT_AllocUpBuffer                 0x1000fdd9   Thumb Code   164  segger_rtt.o(.text)
    SEGGER_RTT_ConfigUpBuffer                0x1000fe7d   Thumb Code   142  segger_rtt.o(.text)
    SEGGER_RTT_ConfigDownBuffer              0x1000ff0b   Thumb Code   146  segger_rtt.o(.text)
    SEGGER_RTT_SetNameUpBuffer               0x1000ff9d   Thumb Code    80  segger_rtt.o(.text)
    SEGGER_RTT_SetNameDownBuffer             0x1000ffed   Thumb Code    78  segger_rtt.o(.text)
    SEGGER_RTT_SetFlagsUpBuffer              0x1001003b   Thumb Code    82  segger_rtt.o(.text)
    SEGGER_RTT_SetFlagsDownBuffer            0x1001008d   Thumb Code    80  segger_rtt.o(.text)
    SEGGER_RTT_Init                          0x100100dd   Thumb Code     8  segger_rtt.o(.text)
    SEGGER_RTT_SetTerminal                   0x100100e5   Thumb Code   140  segger_rtt.o(.text)
    SEGGER_RTT_TerminalOut                   0x10010171   Thumb Code   248  segger_rtt.o(.text)
    SEGGER_RTT_vprintf                       0x100104df   Thumb Code   646  segger_rtt_printf.o(.text)
    SEGGER_RTT_printf                        0x10010765   Thumb Code    36  segger_rtt_printf.o(.text)
    SEGGER_RTT_hexdump                       0x10010789   Thumb Code   122  segger_rtt_printf.o(.text)
    Reset_Handler                            0x10010819   Thumb Code     8  startup_armcm0.o(.text)
    NMI_Handler                              0x10010821   Thumb Code     2  startup_armcm0.o(.text)
    HardFault_Handler                        0x10010823   Thumb Code     2  startup_armcm0.o(.text)
    SVC_Handler                              0x10010825   Thumb Code     2  startup_armcm0.o(.text)
    PendSV_Handler                           0x10010827   Thumb Code     2  startup_armcm0.o(.text)
    SysTick_Handler                          0x10010829   Thumb Code     2  startup_armcm0.o(.text)
    CAP_IRQHandler                           0x1001082b   Thumb Code     0  startup_armcm0.o(.text)
    HID_IRQHandler                           0x1001082b   Thumb Code     0  startup_armcm0.o(.text)
    HPWM_IRQHandler                          0x1001082b   Thumb Code     0  startup_armcm0.o(.text)
    HTIMER_IRQHandler                        0x1001082b   Thumb Code     0  startup_armcm0.o(.text)
    I2C0_IRQHandler                          0x1001082b   Thumb Code     0  startup_armcm0.o(.text)
    I2C1_IRQHandler                          0x1001082b   Thumb Code     0  startup_armcm0.o(.text)
    IR_Rx_IRQHandler                         0x1001082b   Thumb Code     0  startup_armcm0.o(.text)
    IR_Tx_IRQHandler                         0x1001082b   Thumb Code     0  startup_armcm0.o(.text)
    ISO_7816_IRQHandler                      0x1001082b   Thumb Code     0  startup_armcm0.o(.text)
    LLC2_IRQHandler                          0x1001082b   Thumb Code     0  startup_armcm0.o(.text)
    LLC_IRQHandler                           0x1001082b   Thumb Code     0  startup_armcm0.o(.text)
    SPIM_IRQHandler                          0x1001082b   Thumb Code     0  startup_armcm0.o(.text)
    SW_IRQHandler                            0x1001082b   Thumb Code     0  startup_armcm0.o(.text)
    TIMER3_IRQHandler                        0x1001082b   Thumb Code     0  startup_armcm0.o(.text)
    TOUCH_IRQHandler                         0x1001082b   Thumb Code     0  startup_armcm0.o(.text)
    SystemCoreClockUpdate                    0x10010835   Thumb Code     8  system_armcm0.o(.text)
    SystemInit                               0x1001083d   Thumb Code     8  system_armcm0.o(.text)
    LLPingReq                                0x10010973   Thumb Code    26  main.o(.text)
    _BBGetMask                               0x10010be1   Thumb Code   158  main.o(.text)
    Lib_LLEvtCallback                        0x10010c7f   Thumb Code   186  main.o(.text)
    ConnectionLatencyMode                    0x10010d39   Thumb Code   112  main.o(.text)
    sw_timer_latency_callback                0x10010da9   Thumb Code    42  main.o(.text)
    TimerStart                               0x10010dd3   Thumb Code    10  main.o(.text)
    smart_latency_start                      0x10010ddd   Thumb Code   212  main.o(.text)
    smart_update_latency_updatersp           0x10010eb1   Thumb Code   162  main.o(.text)
    BBRFRead                                 0x10010f53   Thumb Code     4  main.o(.text)
    BBRFWrite                                0x10010f57   Thumb Code     6  main.o(.text)
    RCOSCCalibration                         0x10010f5d   Thumb Code    64  main.o(.text)
    RFSleep                                  0x10010f9d   Thumb Code    10  main.o(.text)
    UartEn                                   0x10010fa7   Thumb Code    32  main.o(.text)
    _SYS32kClockSwitch                       0x10010fc7   Thumb Code   264  main.o(.text)
    ClockSwitch                              0x100110cf   Thumb Code    10  main.o(.text)
    RFWakeup                                 0x100110d9   Thumb Code    22  main.o(.text)
    LPOCalibration                           0x100110ef   Thumb Code   242  main.o(.text)
    smart_latency_clear                      0x100111e1   Thumb Code    12  main.o(.text)
    Lib_EvtCallback                          0x100111ed   Thumb Code   248  main.o(.text)
    _BMGetNextBondDevice                     0x100112e5   Thumb Code   144  main.o(.text)
    __LLVersionIndRxHandler                  0x10011469   Thumb Code    66  main.o(.text)
    GetMasterSystem                          0x100114ab   Thumb Code     6  main.o(.text)
    TimerStop                                0x100114b1   Thumb Code    56  main.o(.text)
    smart_update_retry                       0x100114e9   Thumb Code   158  main.o(.text)
    sw_timer_update_callback                 0x10011587   Thumb Code    60  main.o(.text)
    smart_update_latency_updatareq           0x100115c3   Thumb Code   496  main.o(.text)
    Lib_ProtocolHookCallback                 0x100117b3   Thumb Code   116  main.o(.text)
    Lib_MiscCallback                         0x10011827   Thumb Code    14  main.o(.text)
    BleInit                                  0x10011835   Thumb Code   348  main.o(.text)
    DisConnect                               0x10011991   Thumb Code    10  main.o(.text)
    SetDevAddr                               0x1001199b   Thumb Code    12  main.o(.text)
    GetDevAddr                               0x100119a7   Thumb Code    12  main.o(.text)
    SetLEFeature                             0x100119b3   Thumb Code    12  main.o(.text)
    SetAdvAccCode                            0x100119bf   Thumb Code    12  main.o(.text)
    SetAdvParams                             0x100119cb   Thumb Code    12  main.o(.text)
    SetAdvData                               0x100119d7   Thumb Code    12  main.o(.text)
    StartAdv                                 0x10011c11   Thumb Code    10  main.o(.text)
    StopAdv                                  0x10011c1b   Thumb Code    24  main.o(.text)
    StopAdv_Noreset                          0x10011c33   Thumb Code    38  main.o(.text)
    SetScanParams                            0x10011c59   Thumb Code    10  main.o(.text)
    _BBSetScan                               0x10011c63   Thumb Code    46  main.o(.text)
    _GAPStartScan                            0x10011c91   Thumb Code   230  main.o(.text)
    StartScan                                0x10011d77   Thumb Code    10  main.o(.text)
    StopScan                                 0x10011d81   Thumb Code    10  main.o(.text)
    SetSecParams                             0x10011d8b   Thumb Code    12  main.o(.text)
    SetConnectionUpdate                      0x10011d97   Thumb Code    12  main.o(.text)
    GetLinkParameters                        0x10011da3   Thumb Code    12  main.o(.text)
    SetWinWideMinusCnt                       0x10011daf   Thumb Code     8  main.o(.text)
    SetPasskey                               0x10011db7   Thumb Code    12  main.o(.text)
    SecurityReq                              0x10011dc3   Thumb Code    12  main.o(.text)
    SetEvtCallback                           0x10011dcf   Thumb Code    54  main.o(.text)
    GetGATTReportHandle                      0x10011e05   Thumb Code    10  main.o(.text)
    SetGATTReadRsp                           0x10011e0f   Thumb Code    12  main.o(.text)
    CheckFIFOFull                            0x10011e1b   Thumb Code    18  main.o(.text)
    GATTDataSend                             0x10011e2d   Thumb Code    86  main.o(.text)
    ATTCSetCallback                          0x10011e83   Thumb Code     4  main.o(.text)
    ATTCMTUReq                               0x10011e87   Thumb Code    24  main.o(.text)
    ATTCFindInfoReq                          0x10011e9f   Thumb Code    28  main.o(.text)
    ATTCFindByTypeValueReq                   0x10011ebb   Thumb Code    40  main.o(.text)
    ATTCReadByTypeReq                        0x10011ee3   Thumb Code    36  main.o(.text)
    ATTCReadReq                              0x10011f07   Thumb Code    24  main.o(.text)
    ATTCReadBlobReq                          0x10011f1f   Thumb Code    28  main.o(.text)
    ATTCReadMultipleReq                      0x10011f3b   Thumb Code    28  main.o(.text)
    ATTCReadByGroupTypeReq                   0x10011f57   Thumb Code    34  main.o(.text)
    ATTCWriteReq                             0x10011f79   Thumb Code    32  main.o(.text)
    ATTCWriteCmdReq                          0x10011f99   Thumb Code    32  main.o(.text)
    ATTCPrepareWriteReq                      0x10011fb9   Thumb Code    36  main.o(.text)
    ATTCExecuteWriteReq                      0x10011fdd   Thumb Code    24  main.o(.text)
    ATTCConfirmation                         0x10011ff5   Thumb Code    20  main.o(.text)
    _SYSClockSwitch                          0x10012009   Thumb Code    86  main.o(.text)
    MCUClockSwitch                           0x1001205f   Thumb Code     2  main.o(.text)
    GetMCUClock                              0x10012061   Thumb Code    14  main.o(.text)
    GetClock                                 0x1001206f   Thumb Code    16  main.o(.text)
    WakeupConfig                             0x1001207f   Thumb Code    12  main.o(.text)
    LLSleep                                  0x1001208b   Thumb Code    12  main.o(.text)
    Rand                                     0x10012097   Thumb Code     4  main.o(.text)
    DelayUS                                  0x1001209b   Thumb Code     4  main.o(.text)
    DelayMS                                  0x1001209f   Thumb Code     6  main.o(.text)
    GetCompanyID                             0x100120a5   Thumb Code    18  main.o(.text)
    GetQFNType                               0x100120b7   Thumb Code    20  main.o(.text)
    RFRead                                   0x100120cb   Thumb Code     8  main.o(.text)
    RFWrite                                  0x100120d3   Thumb Code     8  main.o(.text)
    lib_check_ble_fsm_state                  0x100120db   Thumb Code    26  main.o(.text)
    SystemSleep                              0x100120f5   Thumb Code    20  main.o(.text)
    SystemPowerDown                          0x10012109   Thumb Code   140  main.o(.text)
    SystemReset                              0x10012195   Thumb Code    10  main.o(.text)
    CapdetEn                                 0x1001219f   Thumb Code    10  main.o(.text)
    PowerDownLPOEn                           0x100121a9   Thumb Code    12  main.o(.text)
    SetBondManagerIndex                      0x100121b5   Thumb Code    12  main.o(.text)
    GetBondDevice                            0x100121c1   Thumb Code     6  main.o(.text)
    AddBondDevice                            0x100121c7   Thumb Code    12  main.o(.text)
    DelAllBondDevice                         0x100121d3   Thumb Code    10  main.o(.text)
    DelBondDevice                            0x100121dd   Thumb Code    12  main.o(.text)
    ReadProfileData                          0x100121e9   Thumb Code     6  main.o(.text)
    WriteProfileData                         0x100121ef   Thumb Code     6  main.o(.text)
    EraseFlashData                           0x100121f5   Thumb Code    78  main.o(.text)
    ReadFlashData                            0x10012243   Thumb Code    56  main.o(.text)
    WriteFlashData                           0x1001227b   Thumb Code    56  main.o(.text)
    CodeErase                                0x100122b3   Thumb Code   100  main.o(.text)
    CodeErase_sector                         0x10012317   Thumb Code    72  main.o(.text)
    _FMCodeWrite                             0x1001235f   Thumb Code    58  main.o(.text)
    CodeWrite                                0x10012399   Thumb Code    30  main.o(.text)
    CodeUpdate                               0x100123b7   Thumb Code    10  main.o(.text)
    FlashDataUpdate                          0x100123c1   Thumb Code   124  main.o(.text)
    ble_sched_execute                        0x1001243d   Thumb Code   150  main.o(.text)
    ble_sched_finish                         0x100124d3   Thumb Code     4  main.o(.text)
    syd52832_chip_confirm                    0x100124d7   Thumb Code    26  main.o(.text)
    gap_s_smart_update_latency               0x100124f1   Thumb Code   238  main.o(.text)
    eFuseManual                              0x100125df   Thumb Code    28  main.o(.text)
    GPADC_Manual_Calibration                 0x100125fb   Thumb Code    34  main.o(.text)
    GPADC_Get_Calibration                    0x1001261d   Thumb Code    22  main.o(.text)
    GAPGetUartEn                             0x10012633   Thumb Code     6  main.o(.text)
    GAPUartEn                                0x10012639   Thumb Code     6  main.o(.text)
    GAPBBDelayUS                             0x1001263f   Thumb Code     4  main.o(.text)
    GAPBBDelayMS                             0x10012643   Thumb Code     6  main.o(.text)
    GAPGetRFAutoSleep                        0x10012649   Thumb Code     4  main.o(.text)
    GAPSetRFAutoSleep                        0x1001264d   Thumb Code     6  main.o(.text)
    Setting4kUpdate                          0x10012653   Thumb Code   114  main.o(.text)
    SetDevAddr_toflash                       0x100126c5   Thumb Code    72  main.o(.text)
    gap_s_verdor_datas_get                   0x1001270d   Thumb Code    28  main.o(.text)
    gap_s_verdor_datas_set                   0x10012729   Thumb Code    66  main.o(.text)
    gap_s_is_ll_start_enc                    0x1001276b   Thumb Code    26  main.o(.text)
    GAPBBTXFIFO0Write                        0x10012785   Thumb Code     4  main.o(.text)
    flash_peotect_key_confirm                0x10012789   Thumb Code   148  main.o(.text)
    swd_lock                                 0x1001281d   Thumb Code    36  main.o(.text)
    flash_data_offect_get                    0x10012841   Thumb Code    50  main.o(.text)
    EraseCodeB                               0x10012873   Thumb Code    56  main.o(.text)
    ReadCodeB                                0x100128ab   Thumb Code    62  main.o(.text)
    WriteCodeB                               0x100128e9   Thumb Code    62  main.o(.text)
    ble_SetTxPower                           0x10012927   Thumb Code   284  main.o(.text)
    flash_data_size_get                      0x10012a43   Thumb Code    18  main.o(.text)
    code_idx_get                             0x10012a55   Thumb Code     6  main.o(.text)
    flash_data_size_set                      0x10012a5b   Thumb Code   146  main.o(.text)
    Get_RSSI_Last_RX                         0x10012aed   Thumb Code    82  main.o(.text)
    APP_Read_Attribute_Encrypt               0x10012b3f   Thumb Code    62  main.o(.text)
    APP_Write_Attribute_Encrypt              0x10012b7d   Thumb Code    66  main.o(.text)
    APP_Read_Charact_Permission              0x10012bbf   Thumb Code    66  main.o(.text)
    smart_latency_target                     0x10012c01   Thumb Code    30  main.o(.text)
    smp_aes_encrypt                          0x10012c1f   Thumb Code     4  main.o(.text)
    gap_get_flash_data_info                  0x10012c23   Thumb Code    26  main.o(.text)
    gap_set_flash_data_info                  0x10012c3d   Thumb Code    70  main.o(.text)
    gap_check_dev_bonded                     0x10012c83   Thumb Code     6  main.o(.text)
    syd_set_chip_flash_all_size              0x10012c89   Thumb Code     6  main.o(.text)
    Xtal_trim_get                            0x10012c8f   Thumb Code   106  main.o(.text)
    Xtal_trim_set                            0x10012cf9   Thumb Code   164  main.o(.text)
    Timer_Evt_Creat                          0x10012fb5   Thumb Code    54  timer.o(.text)
    Min                                      0x10012feb   Thumb Code     8  timer.o(.text)
    TimerDelayUS                             0x10012ff3   Thumb Code    24  timer.o(.text)
    timer_0_disable                          0x1001300b   Thumb Code    48  timer.o(.text)
    timer_0_enable                           0x1001303b   Thumb Code    96  timer.o(.text)
    timer_0_start                            0x1001309b   Thumb Code    22  timer.o(.text)
    timer_0_get                              0x1001311f   Thumb Code    92  timer.o(.text)
    Timer_Evt_Stop                           0x1001317b   Thumb Code   120  timer.o(.text)
    Timer_Evt_ReSet                          0x100131f3   Thumb Code    64  timer.o(.text)
    Timer_Evt_Clr                            0x10013233   Thumb Code    10  timer.o(.text)
    Timer_Evt_Start                          0x1001323d   Thumb Code   156  timer.o(.text)
    Timer_Evt_ReStart                        0x100132d9   Thumb Code   132  timer.o(.text)
    Timer_Get_State                          0x1001335d   Thumb Code    34  timer.o(.text)
    SYD_Timer_Init                           0x1001337f   Thumb Code    58  timer.o(.text)
    timer_0_delay_32us                       0x100133b9   Thumb Code    66  timer.o(.text)
    TIMER0_IRQHandler                        0x100133fb   Thumb Code    32  timer.o(.text)
    timer_1_enable                           0x1001341b   Thumb Code    96  timer.o(.text)
    timer_1_disable                          0x1001347b   Thumb Code    48  timer.o(.text)
    TIMER1_IRQHandler                        0x100134ab   Thumb Code    32  timer.o(.text)
    timer_2_enable                           0x100134cb   Thumb Code    96  timer.o(.text)
    timer_1_get                              0x1001352b   Thumb Code    34  timer.o(.text)
    timer_2_get                              0x1001354d   Thumb Code    34  timer.o(.text)
    timer_2_disable                          0x1001356f   Thumb Code    48  timer.o(.text)
    TIMER2_IRQHandler                        0x1001359f   Thumb Code    32  timer.o(.text)
    rtc_get_calendar                         0x100135f9   Thumb Code    40  rtc.o(.text)
    RTC_RUN                                  0x10013621   Thumb Code    66  rtc.o(.text)
    rtc_set_compare                          0x10013663   Thumb Code    68  rtc.o(.text)
    RTC_SET                                  0x100136a7   Thumb Code    84  rtc.o(.text)
    RTC_Refressh                             0x100136fb   Thumb Code    76  rtc.o(.text)
    RTC_EVT_Creat                            0x10013747   Thumb Code    32  rtc.o(.text)
    Min_RTC                                  0x10013767   Thumb Code     8  rtc.o(.text)
    rtc_int_disable                          0x1001376f   Thumb Code    24  rtc.o(.text)
    RTC_EVT_Clr                              0x1001381d   Thumb Code    10  rtc.o(.text)
    RTC_EVT_Stop                             0x10013827   Thumb Code   112  rtc.o(.text)
    RTC_EVT_Start                            0x10013897   Thumb Code   146  rtc.o(.text)
    RTC_EVT_whole_minute_setid               0x10013929   Thumb Code     6  rtc.o(.text)
    RTC_EVT_whole_minute_adj                 0x1001392f   Thumb Code   132  rtc.o(.text)
    RTC_Get_State                            0x100139b3   Thumb Code    54  rtc.o(.text)
    rtc_start                                0x100139e9   Thumb Code    28  rtc.o(.text)
    rtc_set_interrupt_callback               0x10013a05   Thumb Code     6  rtc.o(.text)
    rtc_int_enable                           0x10013a0b   Thumb Code    22  rtc.o(.text)
    rtc_int_clear                            0x10013a21   Thumb Code    22  rtc.o(.text)
    rtc_set_calendar                         0x10013a37   Thumb Code    40  rtc.o(.text)
    rtc_set_prescaler                        0x10013a5f   Thumb Code    34  rtc.o(.text)
    rtc_clear                                0x10013a81   Thumb Code    18  rtc.o(.text)
    rtc_stop                                 0x10013a93   Thumb Code    30  rtc.o(.text)
    rtc_init                                 0x10013ab1   Thumb Code   126  rtc.o(.text)
    SYD_RTC_Init                             0x10013b2f   Thumb Code    40  rtc.o(.text)
    RTC_IRQHandler                           0x10013b57   Thumb Code    30  rtc.o(.text)
    rtc_status                               0x10013b75   Thumb Code     6  rtc.o(.text)
    rtc_get_compare                          0x10013b7b   Thumb Code    52  rtc.o(.text)
    __aeabi_uidiv                            0x10013bc1   Thumb Code     0  uidiv.o(.text)
    __aeabi_uidivmod                         0x10013bc1   Thumb Code    44  uidiv.o(.text)
    __aeabi_idiv                             0x10013bed   Thumb Code     0  idiv.o(.text)
    __aeabi_idivmod                          0x10013bed   Thumb Code    40  idiv.o(.text)
    tolower                                  0x10013c15   Thumb Code    12  tolower.o(.text)
    __aeabi_memcpy                           0x10013c21   Thumb Code    36  memcpya.o(.text)
    __aeabi_memcpy4                          0x10013c21   Thumb Code     0  memcpya.o(.text)
    __aeabi_memcpy8                          0x10013c21   Thumb Code     0  memcpya.o(.text)
    __aeabi_memset                           0x10013c45   Thumb Code    14  memseta.o(.text)
    __aeabi_memset4                          0x10013c45   Thumb Code     0  memseta.o(.text)
    __aeabi_memset8                          0x10013c45   Thumb Code     0  memseta.o(.text)
    __aeabi_memclr                           0x10013c53   Thumb Code     4  memseta.o(.text)
    __aeabi_memclr4                          0x10013c53   Thumb Code     0  memseta.o(.text)
    __aeabi_memclr8                          0x10013c53   Thumb Code     0  memseta.o(.text)
    _memset$wrapper                          0x10013c57   Thumb Code    18  memseta.o(.text)
    strlen                                   0x10013c69   Thumb Code    14  strlen.o(.text)
    strcmp                                   0x10013c77   Thumb Code    28  strcmp.o(.text)
    memcmp                                   0x10013c93   Thumb Code    26  memcmp.o(.text)
    strcpy                                   0x10013cad   Thumb Code    18  strcpy.o(.text)
    strncmp                                  0x10013cbf   Thumb Code    30  strncmp.o(.text)
    __aeabi_uread4                           0x10013cdd   Thumb Code    20  uread4.o(.text)
    __rt_uread4                              0x10013cdd   Thumb Code     0  uread4.o(.text)
    _uread4                                  0x10013cdd   Thumb Code     0  uread4.o(.text)
    __aeabi_uwrite4                          0x10013cf1   Thumb Code    18  uwrite4.o(.text)
    __rt_uwrite4                             0x10013cf1   Thumb Code     0  uwrite4.o(.text)
    _uwrite4                                 0x10013cf1   Thumb Code     0  uwrite4.o(.text)
    __0sscanf                                0x10013d05   Thumb Code    50  __0sscanf.o(.text)
    _scanf_real                              0x10013e5f   Thumb Code     0  scanf_fp.o(.text)
    _scanf_really_real                       0x10013e5f   Thumb Code   586  scanf_fp.o(.text)
    __aeabi_fadd                             0x100140b5   Thumb Code   162  fadd.o(.text)
    __aeabi_fsub                             0x10014157   Thumb Code     8  fadd.o(.text)
    __aeabi_frsub                            0x1001415f   Thumb Code     8  fadd.o(.text)
    __aeabi_fmul                             0x10014167   Thumb Code   122  fmul.o(.text)
    __aeabi_fdiv                             0x100141e1   Thumb Code   124  fdiv.o(.text)
    __aeabi_dadd                             0x1001425d   Thumb Code   328  dadd.o(.text)
    __aeabi_dsub                             0x100143a5   Thumb Code    12  dadd.o(.text)
    __aeabi_drsub                            0x100143b1   Thumb Code    12  dadd.o(.text)
    __aeabi_dmul                             0x100143c1   Thumb Code   202  dmul.o(.text)
    __aeabi_ddiv                             0x10014491   Thumb Code   234  ddiv.o(.text)
    __aeabi_i2f                              0x10014581   Thumb Code    22  fflti.o(.text)
    __aeabi_ui2f                             0x10014597   Thumb Code    14  ffltui.o(.text)
    __aeabi_i2d                              0x100145a5   Thumb Code    34  dflti.o(.text)
    __aeabi_ui2d                             0x100145cd   Thumb Code    24  dfltui.o(.text)
    __aeabi_f2iz                             0x100145e9   Thumb Code    50  ffixi.o(.text)
    __aeabi_d2iz                             0x1001461d   Thumb Code    62  dfixi.o(.text)
    __aeabi_d2uiz                            0x10014665   Thumb Code    50  dfixui.o(.text)
    __aeabi_f2d                              0x100146a1   Thumb Code    40  f2d.o(.text)
    __aeabi_cdcmpeq                          0x100146c9   Thumb Code     0  cdcmple.o(.text)
    __aeabi_cdcmple                          0x100146c9   Thumb Code    38  cdcmple.o(.text)
    __aeabi_cdrcmple                         0x100146f1   Thumb Code    38  cdrcmple.o(.text)
    __aeabi_d2f                              0x10014719   Thumb Code    56  d2f.o(.text)
    __aeabi_uldivmod                         0x10014751   Thumb Code    96  uldiv.o(.text)
    __aeabi_lmul                             0x100147b1   Thumb Code   122  llmul.o(.text)
    _ll_mul                                  0x100147b1   Thumb Code     0  llmul.o(.text)
    __aeabi_llsl                             0x1001482b   Thumb Code    32  llshl.o(.text)
    _ll_shift_l                              0x1001482b   Thumb Code     0  llshl.o(.text)
    __aeabi_llsr                             0x1001484b   Thumb Code    34  llushr.o(.text)
    _ll_ushift_r                             0x1001484b   Thumb Code     0  llushr.o(.text)
    __aeabi_lasr                             0x1001486d   Thumb Code    38  llsshr.o(.text)
    _ll_sshift_r                             0x1001486d   Thumb Code     0  llsshr.o(.text)
    __vfscanf_char                           0x100148a1   Thumb Code    24  scanf_char.o(.text)
    _sgetc                                   0x100148c1   Thumb Code    32  _sgetc.o(.text)
    _sbackspace                              0x100148e1   Thumb Code    36  _sgetc.o(.text)
    __strtod_int                             0x1001493b   Thumb Code    94  strtod.o(.text)
    __I$use$fp                               0x100149a9   Thumb Code     0  iusefp.o(.text)
    _float_round                             0x100149a9   Thumb Code    16  fepilogue.o(.text)
    _float_epilogue                          0x100149b9   Thumb Code   114  fepilogue.o(.text)
    _double_round                            0x10014a2b   Thumb Code    26  depilogue.o(.text)
    _double_epilogue                         0x10014a45   Thumb Code   164  depilogue.o(.text)
    __aeabi_ul2d                             0x10014ae9   Thumb Code    22  dfltul.o(.text)
    __aeabi_d2ulz                            0x10014b05   Thumb Code    54  dfixul.o(.text)
    __scatterload                            0x10014b45   Thumb Code    28  init.o(.text)
    __scatterload_rt2                        0x10014b45   Thumb Code     0  init.o(.text)
    isspace                                  0x10014b69   Thumb Code    14  isspace_c.o(.text)
    __vfscanf                                0x10014b79   Thumb Code   812  _scanf.o(.text)
    __ctype_lookup                           0x10014eb1   Thumb Code    32  ctype_c.o(.text)
    __decompress                             0x10014ed5   Thumb Code     0  __dczerorl2.o(.text)
    __decompress1                            0x10014ed5   Thumb Code    86  __dczerorl2.o(.text)
    __0sprintf                               0x10014f2d   Thumb Code    36  printfa.o(i.__0sprintf)
    __1sprintf                               0x10014f2d   Thumb Code     0  printfa.o(i.__0sprintf)
    __2sprintf                               0x10014f2d   Thumb Code     0  printfa.o(i.__0sprintf)
    __c89sprintf                             0x10014f2d   Thumb Code     0  printfa.o(i.__0sprintf)
    sprintf                                  0x10014f2d   Thumb Code     0  printfa.o(i.__0sprintf)
    __ARM_clz                                0x10014f55   Thumb Code    46  depilogue.o(i.__ARM_clz)
    __ARM_common_switch8                     0x10014f83   Thumb Code    26  main.o(i.__ARM_common_switch8)
    free                                     0x10014f9d   Thumb Code    94  mallocr.o(i.__free$realloc)
    malloc                                   0x10015001   Thumb Code    54  mallocr.o(i.__malloc$realloc)
    __scatterload_copy                       0x10015049   Thumb Code    14  handlers.o(i.__scatterload_copy)
    __scatterload_null                       0x10015057   Thumb Code     2  handlers.o(i.__scatterload_null)
    __scatterload_zeroinit                   0x10015059   Thumb Code    14  handlers.o(i.__scatterload_zeroinit)
    _is_digit                                0x100151dd   Thumb Code    14  scanf_fp.o(i._is_digit)
    realloc                                  0x10015981   Thumb Code   110  mallocr.o(i.realloc)
    strtod                                   0x100159f5   Thumb Code    28  strtod.o(i.strtod)
    adv_chn_to_freq_idx                      0x10015c20   Data           3  main.o(.constdata)
    __ctype_categories                       0x10015c48   Data          64  ctype_c.o(.constdata)
    Region$$Table$$Base                      0x10015c88   Number         0  anon$$obj.o(Region$$Table)
    Region$$Table$$Limit                     0x10015ca8   Number         0  anon$$obj.o(Region$$Table)
    PIN_CONFIG                               0x20003008   Data           4  gpio.o(.data)
    GPIO_CTRL                                0x2000300c   Data           4  gpio.o(.data)
    GPO_CTRL                                 0x20003010   Data           4  gpio.o(.data)
    GPI_CTRL                                 0x20003014   Data           4  gpio.o(.data)
    GPIO_IRQ_CTRL                            0x20003018   Data           4  gpio.o(.data)
    GPADC                                    0x20003068   Data           4  gpadc.o(.data)
    channel                                  0x2000306c   Data           1  gpadc.o(.data)
    syd_history_setting_str                  0x20003074   Data           4  rtc_handler.o(.data)
    ota_state                                0x20003078   Data           1  ota.o(.data)
    ota_writecnt                             0x20003079   Data           1  ota.o(.data)
    ota_section_size                         0x2000307a   Data           2  ota.o(.data)
    ota_receive_size                         0x2000307c   Data           2  ota.o(.data)
    ota_section_check                        0x2000307e   Data           2  ota.o(.data)
    ota_receive_check                        0x20003080   Data           2  ota.o(.data)
    ota_section_offset                       0x20003084   Data           4  ota.o(.data)
    pevt                                     0x20003090   Data           4  ota.o(.data)
    Angle                                    0x20003094   Data           4  lsm6d.o(.data)
    connect_flag                             0x200030fc   Data           1  main.o(.data)
    Adv_State                                0x200030fd   Data           1  main.o(.data)
    update_latency_mode                      0x20003102   Data           1  main.o(.data)
    start_tx                                 0x20003103   Data           1  main.o(.data)
    syd_nosleep_control                      0x20003104   Data           1  main.o(.data)
    batteryPercentage                        0x20003108   Data           4  main.o(.data)
    ADV_DATA                                 0x2000310c   Data          29  main.o(.data)
    SCAN_DATA                                0x20003129   Data          11  main.o(.data)
    SystemCoreClock                          0x20003148   Data           4  system_armcm0.o(.data)
    master_system                            0x20003151   Data           1  main.o(.data)
    p_gett_db_hdr                            0x20003168   Data           4  main.o(.data)
    Event_Num                                0x2000318c   Data           1  timer.o(.data)
    max_trigger_timer                        0x20003194   Data           4  timer.o(.data)
    TIMER_EVT                                0x20003198   Data           4  timer.o(.data)
    Timer_Evt_Trigger_Loop_now               0x2000319c   Data           4  timer.o(.data)
    sys_timer_max_p                          0x200031a0   Data           4  timer.o(.data)
    sys_timer_current_p                      0x200031a4   Data           4  timer.o(.data)
    RTC_Event_Num                            0x200031a9   Data           1  rtc.o(.data)
    max_trigger_rtc                          0x200031ac   Data           4  rtc.o(.data)
    RTC_EVT                                  0x200031b0   Data           4  rtc.o(.data)
    RTC_RTCEVT_Trigger_Loop_now              0x200031b4   Data           4  rtc.o(.data)
    RTC_second_now                           0x200031b8   Data           4  rtc.o(.data)
    sys_rtc_max_p                            0x200031bc   Data           4  rtc.o(.data)
    sys_rtc_current_p                        0x200031c0   Data           4  rtc.o(.data)
    RTCEVT_whole_minute_id                   0x200031c4   Data           4  rtc.o(.data)
    RTC_second_last                          0x200031cc   Data           4  rtc.o(.data)
    __microlib_freelist                      0x200031d0   Data           4  mvars.o(.data)
    __microlib_freelist_initialised          0x200031d4   Data           4  mvars.o(.data)
    syd_sysTimer                             0x200031d8   Data         120  timer_handler.o(.bss)
    ota_w                                    0x20003250   Data          40  ota.o(.bss)
    dev_ctx1                                 0x20003278   Data          16  lis2dh.o(.bss)
    dev_ctx                                  0x20003288   Data          16  lsm6d.o(.bss)
    tFilter                                  0x20003298   Data          12  lsm6d.o(.bss)
    PAS                                      0x200032a4   Data          14  lsm6d.o(.bss)
    dtts_tx_buffer                           0x200032c4   Data        1032  main.o(.bss)
    _SEGGER_RTT                              0x200036cc   Data          72  segger_rtt.o(.bss)
    __heap_base                              0x20003b98   Data           0  startup_armcm0.o(HEAP)
    __heap_limit                             0x20004798   Data           0  startup_armcm0.o(HEAP)
    __initial_sp                             0x20004b98   Data           0  startup_armcm0.o(STACK)



==============================================================================

Memory Map of the image

  Image Entry point : 0x100000c1

  Load Region LR_IROM1 (Base: 0x10000000, Size: 0x00015e80, Max: 0x0003f000, ABSOLUTE, COMPRESSED[0x00015d8c])

    Execution Region ER_IROM1 (Exec base: 0x10000000, Load base: 0x10000000, Size: 0x00015ca8, Max: 0x0003f000, ABSOLUTE)

    Exec Addr    Load Addr    Size         Type   Attr      Idx    E Section Name        Object

    0x10000000   0x10000000   0x000000c0   Data   RO          756    RESET               startup_armcm0.o
    0x100000c0   0x100000c0   0x00000000   Code   RO          998  * .ARM.Collect$$$$00000000  mc_p.l(entry.o)
    0x100000c0   0x100000c0   0x00000004   Code   RO         1361    .ARM.Collect$$$$00000001  mc_p.l(entry2.o)
    0x100000c4   0x100000c4   0x00000004   Code   RO         1364    .ARM.Collect$$$$00000004  mc_p.l(entry5.o)
    0x100000c8   0x100000c8   0x00000000   Code   RO         1366    .ARM.Collect$$$$00000008  mc_p.l(entry7b.o)
    0x100000c8   0x100000c8   0x00000000   Code   RO         1368    .ARM.Collect$$$$0000000A  mc_p.l(entry8b.o)
    0x100000c8   0x100000c8   0x00000008   Code   RO         1369    .ARM.Collect$$$$0000000B  mc_p.l(entry9a.o)
    0x100000d0   0x100000d0   0x00000000   Code   RO         1371    .ARM.Collect$$$$0000000D  mc_p.l(entry10a.o)
    0x100000d0   0x100000d0   0x00000000   Code   RO         1373    .ARM.Collect$$$$0000000F  mc_p.l(entry11a.o)
    0x100000d0   0x100000d0   0x00000004   Code   RO         1362    .ARM.Collect$$$$00002712  mc_p.l(entry2.o)
    0x100000d4   0x100000d4   0x000004c4   Code   RO           69    .text               uart.o
    0x10000598   0x10000598   0x00000038   Code   RO           98    .text               delay.o
    0x100005d0   0x100005d0   0x00000574   Code   RO          121    .text               gpio.o
    0x10000b44   0x10000b44   0x00000440   Code   RO          147    .text               i2c.o
    0x10000f84   0x10000f84   0x00000588   Code   RO          175    .text               gpadc.o
    0x1000150c   0x1000150c   0x000000ac   Code   RO          223    .text               timer_handler.o
    0x100015b8   0x100015b8   0x000006f0   Code   RO          291    .text               ota.o
    0x10001ca8   0x10001ca8   0x0000011c   Code   RO          322    .text               app_gpio.o
    0x10001dc4   0x10001dc4   0x00000024   Code   RO          348    .text               app_timer.o
    0x10001de8   0x10001de8   0x00000026   Code   RO          374    .text               app_adc.o
    0x10001e0e   0x10001e0e   0x00000002   PAD
    0x10001e10   0x10001e10   0x00000194   Code   RO          397    .text               lis2dh.o
    0x10001fa4   0x10001fa4   0x00000298   Code   RO          433    .text               lsm6d.o
    0x1000223c   0x1000223c   0x0000144a   Code   RO          461    .text               lis2dh12_reg.o
    0x10003686   0x10003686   0x00000002   PAD
    0x10003688   0x10003688   0x0000860a   Code   RO          473    .text               lsm6dso_reg.o
    0x1000bc92   0x1000bc92   0x00000002   PAD
    0x1000bc94   0x1000bc94   0x00002420   Code   RO          485    .text               cjson.o
    0x1000e0b4   0x1000e0b4   0x000000a8   Code   RO          533    .text               crc16.o
    0x1000e15c   0x1000e15c   0x00000034   Code   RO          553    .text               common.o
    0x1000e190   0x1000e190   0x00001528   Code   RO          570    .text               main.o
    0x1000f6b8   0x1000f6b8   0x00000034   Code   RO          626    .text               mcu_bsp.o
    0x1000f6ec   0x1000f6ec   0x0000005c   Code   RO          646    .text               isr.o
    0x1000f748   0x1000f748   0x00000b2c   Code   RO          666    .text               segger_rtt.o
    0x10010274   0x10010274   0x000005a4   Code   RO          693    .text               segger_rtt_printf.o
    0x10010818   0x10010818   0x0000001c   Code   RO          757    .text               startup_armcm0.o
    0x10010834   0x10010834   0x00000018   Code   RO          763    .text               system_armcm0.o
    0x1001084c   0x1001084c   0x00002768   Code   RO          789    .text               syd8811_ble_lib.lib(main.o)
    0x10012fb4   0x10012fb4   0x00000644   Code   RO          891    .text               Syd8811_softtimer_lib20240514_225042.lib(timer.o)
    0x100135f8   0x100135f8   0x000005c8   Code   RO          959    .text               Syd8811_softtimer_lib20240514_225042.lib(rtc.o)
    0x10013bc0   0x10013bc0   0x0000002c   Code   RO         1006    .text               mc_p.l(uidiv.o)
    0x10013bec   0x10013bec   0x00000028   Code   RO         1008    .text               mc_p.l(idiv.o)
    0x10013c14   0x10013c14   0x0000000c   Code   RO         1010    .text               mc_p.l(tolower.o)
    0x10013c20   0x10013c20   0x00000024   Code   RO         1012    .text               mc_p.l(memcpya.o)
    0x10013c44   0x10013c44   0x00000024   Code   RO         1014    .text               mc_p.l(memseta.o)
    0x10013c68   0x10013c68   0x0000000e   Code   RO         1016    .text               mc_p.l(strlen.o)
    0x10013c76   0x10013c76   0x0000001c   Code   RO         1018    .text               mc_p.l(strcmp.o)
    0x10013c92   0x10013c92   0x0000001a   Code   RO         1020    .text               mc_p.l(memcmp.o)
    0x10013cac   0x10013cac   0x00000012   Code   RO         1022    .text               mc_p.l(strcpy.o)
    0x10013cbe   0x10013cbe   0x0000001e   Code   RO         1024    .text               mc_p.l(strncmp.o)
    0x10013cdc   0x10013cdc   0x00000014   Code   RO         1317    .text               mc_p.l(uread4.o)
    0x10013cf0   0x10013cf0   0x00000012   Code   RO         1319    .text               mc_p.l(uwrite4.o)
    0x10013d02   0x10013d02   0x00000002   PAD
    0x10013d04   0x10013d04   0x0000003c   Code   RO         1321    .text               mc_p.l(__0sscanf.o)
    0x10013d40   0x10013d40   0x00000374   Code   RO         1323    .text               mc_p.l(scanf_fp.o)
    0x100140b4   0x100140b4   0x000000b2   Code   RO         1327    .text               mf_p.l(fadd.o)
    0x10014166   0x10014166   0x0000007a   Code   RO         1329    .text               mf_p.l(fmul.o)
    0x100141e0   0x100141e0   0x0000007c   Code   RO         1331    .text               mf_p.l(fdiv.o)
    0x1001425c   0x1001425c   0x00000164   Code   RO         1333    .text               mf_p.l(dadd.o)
    0x100143c0   0x100143c0   0x000000d0   Code   RO         1335    .text               mf_p.l(dmul.o)
    0x10014490   0x10014490   0x000000f0   Code   RO         1337    .text               mf_p.l(ddiv.o)
    0x10014580   0x10014580   0x00000016   Code   RO         1339    .text               mf_p.l(fflti.o)
    0x10014596   0x10014596   0x0000000e   Code   RO         1341    .text               mf_p.l(ffltui.o)
    0x100145a4   0x100145a4   0x00000028   Code   RO         1343    .text               mf_p.l(dflti.o)
    0x100145cc   0x100145cc   0x0000001c   Code   RO         1345    .text               mf_p.l(dfltui.o)
    0x100145e8   0x100145e8   0x00000032   Code   RO         1347    .text               mf_p.l(ffixi.o)
    0x1001461a   0x1001461a   0x00000002   PAD
    0x1001461c   0x1001461c   0x00000048   Code   RO         1349    .text               mf_p.l(dfixi.o)
    0x10014664   0x10014664   0x0000003c   Code   RO         1351    .text               mf_p.l(dfixui.o)
    0x100146a0   0x100146a0   0x00000028   Code   RO         1353    .text               mf_p.l(f2d.o)
    0x100146c8   0x100146c8   0x00000028   Code   RO         1355    .text               mf_p.l(cdcmple.o)
    0x100146f0   0x100146f0   0x00000028   Code   RO         1357    .text               mf_p.l(cdrcmple.o)
    0x10014718   0x10014718   0x00000038   Code   RO         1359    .text               mf_p.l(d2f.o)
    0x10014750   0x10014750   0x00000060   Code   RO         1376    .text               mc_p.l(uldiv.o)
    0x100147b0   0x100147b0   0x0000007a   Code   RO         1378    .text               mc_p.l(llmul.o)
    0x1001482a   0x1001482a   0x00000020   Code   RO         1380    .text               mc_p.l(llshl.o)
    0x1001484a   0x1001484a   0x00000022   Code   RO         1382    .text               mc_p.l(llushr.o)
    0x1001486c   0x1001486c   0x00000026   Code   RO         1384    .text               mc_p.l(llsshr.o)
    0x10014892   0x10014892   0x00000002   PAD
    0x10014894   0x10014894   0x0000002c   Code   RO         1388    .text               mc_p.l(scanf_char.o)
    0x100148c0   0x100148c0   0x00000044   Code   RO         1390    .text               mc_p.l(_sgetc.o)
    0x10014904   0x10014904   0x000000a4   Code   RO         1392    .text               mc_p.l(strtod.o)
    0x100149a8   0x100149a8   0x00000000   Code   RO         1394    .text               mc_p.l(iusefp.o)
    0x100149a8   0x100149a8   0x00000082   Code   RO         1396    .text               mf_p.l(fepilogue.o)
    0x10014a2a   0x10014a2a   0x000000be   Code   RO         1398    .text               mf_p.l(depilogue.o)
    0x10014ae8   0x10014ae8   0x0000001c   Code   RO         1402    .text               mf_p.l(dfltul.o)
    0x10014b04   0x10014b04   0x00000040   Code   RO         1404    .text               mf_p.l(dfixul.o)
    0x10014b44   0x10014b44   0x00000024   Code   RO         1406    .text               mc_p.l(init.o)
    0x10014b68   0x10014b68   0x0000000e   Code   RO         1408    .text               mc_p.l(isspace_c.o)
    0x10014b76   0x10014b76   0x00000002   PAD
    0x10014b78   0x10014b78   0x00000338   Code   RO         1410    .text               mc_p.l(_scanf.o)
    0x10014eb0   0x10014eb0   0x00000024   Code   RO         1412    .text               mc_p.l(ctype_c.o)
    0x10014ed4   0x10014ed4   0x00000056   Code   RO         1422    .text               mc_p.l(__dczerorl2.o)
    0x10014f2a   0x10014f2a   0x00000002   PAD
    0x10014f2c   0x10014f2c   0x00000028   Code   RO         1263    i.__0sprintf        mc_p.l(printfa.o)
    0x10014f54   0x10014f54   0x0000002e   Code   RO         1400    i.__ARM_clz         mf_p.l(depilogue.o)
    0x10014f82   0x10014f82   0x0000001a   Code   RO          810    i.__ARM_common_switch8  syd8811_ble_lib.lib(main.o)
    0x10014f9c   0x10014f9c   0x00000064   Code   RO         1293    i.__free$realloc    mc_p.l(mallocr.o)
    0x10015000   0x10015000   0x00000048   Code   RO         1294    i.__malloc$realloc  mc_p.l(mallocr.o)
    0x10015048   0x10015048   0x0000000e   Code   RO         1416    i.__scatterload_copy  mc_p.l(handlers.o)
    0x10015056   0x10015056   0x00000002   Code   RO         1417    i.__scatterload_null  mc_p.l(handlers.o)
    0x10015058   0x10015058   0x0000000e   Code   RO         1418    i.__scatterload_zeroinit  mc_p.l(handlers.o)
    0x10015066   0x10015066   0x00000002   PAD
    0x10015068   0x10015068   0x00000174   Code   RO         1268    i._fp_digits        mc_p.l(printfa.o)
    0x100151dc   0x100151dc   0x0000000e   Code   RO         1325    i._is_digit         mc_p.l(scanf_fp.o)
    0x100151ea   0x100151ea   0x00000002   PAD
    0x100151ec   0x100151ec   0x000006ec   Code   RO         1269    i._printf_core      mc_p.l(printfa.o)
    0x100158d8   0x100158d8   0x00000020   Code   RO         1270    i._printf_post_padding  mc_p.l(printfa.o)
    0x100158f8   0x100158f8   0x0000002c   Code   RO         1271    i._printf_pre_padding  mc_p.l(printfa.o)
    0x10015924   0x10015924   0x0000000a   Code   RO         1273    i._sputc            mc_p.l(printfa.o)
    0x1001592e   0x1001592e   0x00000002   PAD
    0x10015930   0x10015930   0x00000050   Code   RO         1295    i.internal_alloc    mc_p.l(mallocr.o)
    0x10015980   0x10015980   0x00000074   Code   RO         1296    i.realloc           mc_p.l(mallocr.o)
    0x100159f4   0x100159f4   0x0000001c   Code   RO          995    i.strtod            m_ps.l(strtod.o)
    0x10015a10   0x10015a10   0x00000200   Data   RO          534    .constdata          crc16.o
    0x10015c10   0x10015c10   0x00000010   Data   RO          694    .constdata          segger_rtt_printf.o
    0x10015c20   0x10015c20   0x00000028   Data   RO          791    .constdata          syd8811_ble_lib.lib(main.o)
    0x10015c48   0x10015c48   0x00000040   Data   RO         1413    .constdata          mc_p.l(ctype_c.o)
    0x10015c88   0x10015c88   0x00000020   Data   RO         1415    Region$$Table       anon$$obj.o


    Execution Region RW_IRAM1 (Exec base: 0x20003000, Load base: 0x10015ca8, Size: 0x00001b98, Max: 0x00005000, ABSOLUTE, COMPRESSED[0x000000e4])

    Exec Addr    Load Addr    Size         Type   Attr      Idx    E Section Name        Object

    0x20003000   COMPRESSED   0x00000008   Data   RW           70    .data               uart.o
    0x20003008   COMPRESSED   0x00000048   Data   RW          122    .data               gpio.o
    0x20003050   COMPRESSED   0x00000018   Data   RW          148    .data               i2c.o
    0x20003068   COMPRESSED   0x0000000c   Data   RW          176    .data               gpadc.o
    0x20003074   COMPRESSED   0x00000004   Data   RW          265    .data               rtc_handler.o
    0x20003078   COMPRESSED   0x0000001c   Data   RW          293    .data               ota.o
    0x20003094   COMPRESSED   0x00000027   Data   RW          435    .data               lsm6d.o
    0x200030bb   COMPRESSED   0x00000001   PAD
    0x200030bc   COMPRESSED   0x00000014   Data   RW          487    .data               cjson.o
    0x200030d0   COMPRESSED   0x00000067   Data   RW          572    .data               main.o
    0x20003137   COMPRESSED   0x00000011   Data   RW          668    .data               segger_rtt.o
    0x20003148   COMPRESSED   0x00000004   Data   RW          764    .data               system_armcm0.o
    0x2000314c   COMPRESSED   0x00000040   Data   RW          792    .data               syd8811_ble_lib.lib(main.o)
    0x2000318c   COMPRESSED   0x0000001c   Data   RW          893    .data               Syd8811_softtimer_lib20240514_225042.lib(timer.o)
    0x200031a8   COMPRESSED   0x00000028   Data   RW          960    .data               Syd8811_softtimer_lib20240514_225042.lib(rtc.o)
    0x200031d0   COMPRESSED   0x00000004   Data   RW         1386    .data               mc_p.l(mvars.o)
    0x200031d4   COMPRESSED   0x00000004   Data   RW         1387    .data               mc_p.l(mvars.o)
    0x200031d8        -       0x00000078   Zero   RW          224    .bss                timer_handler.o
    0x20003250        -       0x00000028   Zero   RW          292    .bss                ota.o
    0x20003278        -       0x00000010   Zero   RW          398    .bss                lis2dh.o
    0x20003288        -       0x0000002a   Zero   RW          434    .bss                lsm6d.o
    0x200032b2        -       0x0000000f   Zero   RW          486    .bss                cjson.o
    0x200032c1   COMPRESSED   0x00000003   PAD
    0x200032c4        -       0x00000408   Zero   RW          571    .bss                main.o
    0x200036cc        -       0x00000458   Zero   RW          667    .bss                segger_rtt.o
    0x20003b24        -       0x00000068   Zero   RW          790    .bss                syd8811_ble_lib.lib(main.o)
    0x20003b8c        -       0x0000000c   Zero   RW          892    .bss                Syd8811_softtimer_lib20240514_225042.lib(timer.o)
    0x20003b98        -       0x00000c00   Zero   RW          755    HEAP                startup_armcm0.o
    0x20004798        -       0x00000400   Zero   RW          754    STACK               startup_armcm0.o


==============================================================================

Image component sizes


      Code (inc. data)   RO Data    RW Data    ZI Data      Debug   Object Name

        38          0          0          0          0        461   app_adc.o
       284          6          0          0          0       1038   app_gpio.o
        36          8          0          0          0        668   app_timer.o
      9248        216          0         20         15      43288   cjson.o
        52          0          0          0          0        919   common.o
       168         12        512          0          0       1901   crc16.o
         0          0          0          0          0      46288   debug.o
        56          0          0          0          0        652   delay.o
      1416         44          0         12          0      10727   gpadc.o
      1396         44          0         72          0       4662   gpio.o
      1088         24          0         24          0       3457   i2c.o
        92          8          0          0          0        613   isr.o
       404         46          0          0         16      15183   lis2dh.o
      5194         38          0          0          0      35000   lis2dh12_reg.o
       664         78          0         39         42      48259   lsm6d.o
     34314        442          0          0          0     115768   lsm6dso_reg.o
      5416       1110          0        103       1032      11261   main.o
        52          0          0          0          0        749   mcu_bsp.o
      1776        432          0         28         40       5773   ota.o
         0          0          0          4          0       2155   rtc_handler.o
      2860         56          0         17       1112      15827   segger_rtt.o
      1444         34         16          0          0       4838   segger_rtt_printf.o
        28          8        192          0       4096        616   startup_armcm0.o
        24          8          0          4          0        781   system_armcm0.o
       172         30          0          0        120       3243   timer_handler.o
      1220         22          0          8          0      10960   uart.o

    ----------------------------------------------------------------------
     67448       2666        752        332       6476     385087   Object Totals
         0          0         32          0          0          0   (incl. Generated)
         6          0          0          1          3          0   (incl. Padding)

    ----------------------------------------------------------------------

      Code (inc. data)   RO Data    RW Data    ZI Data      Debug   Library Member Name

      1480         38          0         40          0      17883   rtc.o
      1604         36          0         28         12      46732   timer.o
        28          0          0          0          0         72   strtod.o
        60         10          0          0          0         84   __0sscanf.o
        86          0          0          0          0          0   __dczerorl2.o
       824         12          0          0          0         84   _scanf.o
        68          0          0          0          0         76   _sgetc.o
        36          4         64          0          0         60   ctype_c.o
         0          0          0          0          0          0   entry.o
         0          0          0          0          0          0   entry10a.o
         0          0          0          0          0          0   entry11a.o
         8          4          0          0          0          0   entry2.o
         4          0          0          0          0          0   entry5.o
         0          0          0          0          0          0   entry7b.o
         0          0          0          0          0          0   entry8b.o
         8          4          0          0          0          0   entry9a.o
        30          0          0          0          0          0   handlers.o
        40          0          0          0          0         72   idiv.o
        36          8          0          0          0         68   init.o
        14          0          0          0          0         68   isspace_c.o
         0          0          0          0          0          0   iusefp.o
       122          0          0          0          0         84   llmul.o
        32          0          0          0          0         68   llshl.o
        38          0          0          0          0         68   llsshr.o
        34          0          0          0          0         68   llushr.o
       368         36          0          0          0        308   mallocr.o
        26          0          0          0          0         72   memcmp.o
        36          0          0          0          0         60   memcpya.o
        36          0          0          0          0        100   memseta.o
         0          0          0          8          0          0   mvars.o
      2270         94          0          0          0        472   printfa.o
        44          8          0          0          0         84   scanf_char.o
       898         12          0          0          0        184   scanf_fp.o
        28          0          0          0          0         68   strcmp.o
        18          0          0          0          0         60   strcpy.o
        14          0          0          0          0         60   strlen.o
        30          0          0          0          0         72   strncmp.o
       164         16          0          0          0        120   strtod.o
        12          0          0          0          0         60   tolower.o
        44          0          0          0          0         72   uidiv.o
        96          0          0          0          0         84   uldiv.o
        20          0          0          0          0         60   uread4.o
        18          0          0          0          0         60   uwrite4.o
        40          2          0          0          0         68   cdcmple.o
        40          2          0          0          0         68   cdrcmple.o
        56          0          0          0          0         68   d2f.o
       356          4          0          0          0        140   dadd.o
       240          6          0          0          0         84   ddiv.o
       236          0          0          0          0        216   depilogue.o
        72         10          0          0          0         72   dfixi.o
        60         10          0          0          0         68   dfixui.o
        64         10          0          0          0         68   dfixul.o
        40          6          0          0          0         68   dflti.o
        28          4          0          0          0         68   dfltui.o
        28          6          0          0          0         68   dfltul.o
       208          6          0          0          0         88   dmul.o
        40          0          0          0          0         60   f2d.o
       178          0          0          0          0        108   fadd.o
       124          0          0          0          0         72   fdiv.o
       130          0          0          0          0        144   fepilogue.o
        50          0          0          0          0         60   ffixi.o
        22          0          0          0          0         68   fflti.o
        14          0          0          0          0         68   ffltui.o
       122          0          0          0          0         72   fmul.o
     10114        482         40         64        104     111445   main.o

    ----------------------------------------------------------------------
     20952        830        104        140        116     180724   Library Totals
        16          0          0          0          0          0   (incl. Padding)

    ----------------------------------------------------------------------

      Code (inc. data)   RO Data    RW Data    ZI Data      Debug   Library Name

      3084         74          0         68         12      64615   Syd8811_softtimer_lib20240514_225042.lib
        28          0          0          0          0         72   m_ps.l
      5562        208         64          8          0       2796   mc_p.l
      2148         66          0          0          0       1796   mf_p.l
     10114        482         40         64        104     111445   syd8811_ble_lib.lib

    ----------------------------------------------------------------------
     20952        830        104        140        116     180724   Library Totals

    ----------------------------------------------------------------------

==============================================================================


      Code (inc. data)   RO Data    RW Data    ZI Data      Debug   

     88400       3496        856        472       6592     561575   Grand Totals
     88400       3496        856        228       6592     561575   ELF Image Totals (compressed)
     88400       3496        856        228          0          0   ROM Totals

==============================================================================

    Total RO  Size (Code + RO Data)                89256 (  87.16kB)
    Total RW  Size (RW Data + ZI Data)              7064 (   6.90kB)
    Total ROM Size (Code + RO Data + RW Data)      89484 (  87.39kB)

==============================================================================

